:1000000000800020BD01000095CB00004DCB00001A
:100010004DCB00004DCB00004DCB00004DCB000080
:100020004DCB00004DCB00004DCB000095CB000028
:1000300095CB00004DCB000015C2000019C3000095
:1000400095CB000095CB000095CB000095CB000030
:1000500095CB000095CB000095CB000095CB000020
:1000600095CB000095CB000095CB000095CB000010
:1000700095CB000095CB000095CB000095CB000000
:1000800095CB000095CB000095CB000095CB0000F0
:1000900095CB000095CB000095CB000095CB0000E0
:1000A00051A700005DA7000095CB000095CB000094
:1000B00095CB000095CB000095CB000095CB0000C0
:1000C00095CB000095CB000095CB000095CB0000B0
:1000D00095CB000095CB000095CB000095CB0000A0
:1000E00095CB000095CB000095CB000095CB000090
:1000F00095CB000001EC000095CB00002DED000039
:1001000095CB00006DD5000095CB000095CB00008D
:1001100095CB000095CB000095CB000095CB00005F
:1001200095CB000095CB000095CB000095CB00004F
:1001300095CB000095CB000095CB000095CB00003F
:1001400095CB000095CB000095CB000095CB00002F
:1001500005C4000019C400002DC4000041C4000003
:1001600095CB000089D8000095CB000095CB00000E
:1001700095CB000095CB000095CB000095CB0000FF
:1001800095CB000095CB000095CB000095CB0000EF
:1001900095CB000095CB000095CB000095CB0000DF
:1001A00095CB000095CB000095CB000095CB0000CF
:1001B00095CB000095CB000095CB0000564B4CF240
:1001C000205210B51A804DF628121A8000BF00BFC9
:1001D0000CF0E4FC514B4FF010621A60504A9A60E8
:1001E000504ADA60504A136813F4807304D14F49BF
:1001F0000B604FF4A85313604D4B1A78110703D5C9
:100200001A7842F008021A704A4B4B492A221A7097
:100210004A4A4B4B8B4204D252F8040F43F8040B6A
:10022000F8E7484B484900228B4202D243F8042B9E
:10023000FAE74649464A002352F8230041F82300D2
:1002400001336F2BF8D1434B434A802103F8011B44
:100250009342FBD1414B3D4A1A60414B8A221A70AE
:10026000A3F5805324225A70A0221A709A7992071B
:10027000FCD59A79D406FCD43A4A937903F00C035E
:10028000082B384BF9D103221A7140225A719A79FE
:100290009006FCD5334A9179324B4906FBD5324A58
:1002A000324911600221516020221A709A7902F0BD
:1002B0000C020C2AFAD12E4B2E4A1A602E4B2F4AD2
:1002C0001A6000225A60072243F8042C2C4AC3F813
:1002D0000C2D62B60DF012F8144B1B68DA0705D529
:1002E00028480CF0DFFD284B284A1A60284B1B7861
:1002F0005B0609D5244C254B22689A4204D121483B
:100300000CF0D0FD002323600FF0CAFF0CF04CFC72
:100310000CF07AFBFEE700BF0E2005403080044061
:10032000823F04000100002B10D0034014D0034092
:1003300002D0074000E00740C49BFF1FCC3A0100F9
:100340004088FF1FC49BFF1FD0A3FF1F0082FF1F19
:100350000000000000E400E05FE400E008ED00E0E1
:100360000050064000400640448004400000030165
:1003700004800440C010050014E000E0FF76010096
:10038000000020209E3B185F1CE00340A5C3945A48
:1003900000F00740FFFFFFFFFFFFFFFFFFFFFFFF32
:1003A000FFFFFFFFFFFFFFFFFFFFFFFFFFFFFFFF5D
:1003B000FFFFFFFFFFFFFFFFFFFFFFFFFFFFFFFF4D
:1003C000FFFFFFFFFFFFFFFFFFFFFFFFFFFFFFFF3D
:1003D000FFFFFFFFFFFFFFFFFFFFFFFFFFFFFFFF2D
:1003E000FFFFFFFFFFFFFFFFFFFFFFFFFFFFFFFF1D
:1003F000FFFFFFFFFFFFFFFFFFFFFFFFFFFFFFFF0D
:10040000FFFFFFFFFFFFFFFFFFFFFFFFDEF9FFFF23
:1004100010B5054C237833B9044B13B10448AFF33E
:1004200000800123237010BDC49BFF1F000000004B
:10043000D03A0100084B10B51BB108490848AFF38A
:1004400000800848036803B910BD074B002BFBD0A0
:10045000BDE81040184700BF00000000C89BFF1F08
:10046000D03A0100C49BFF1F0000000038B50446CD
:10047000104621700A491D460FF0F4FC01464FF06A
:100480007E500FF0A3FD07490FF0ECFCE5606060C3
:10049000256165610CF0C2FEE061204638BD00BFF9
:1004A000DB0FC9400024744938B50446104621705A
:1004B00009491D460FF0D6FC01464FF07E500FF063
:1004C00085FD06490FF0CEFCE56060602561656141
:1004D0000CF0A4FEE06138BDDB0FC9400024744974
:1004E00038B503780446032B20D8DFE803F01A1848
:1004F0001002C16840690FF0ABFB0D49054660680A
:100500000FF064FD014628460FF060FD38BD084934
:1005100040680FF05BFDE1680FF0A4FC38BDC068D7
:1005200038BDC16840690FF093FB38BD002038BD6D
:100530000024744970B504460E460CF06FFE054663
:10054000E069281A0FF03AFCE3682361E56166610F
:10055000A061014660680FF039FD0146A0601048B7
:100560000FF034FD0FF00AF80EF0AAFC0FF01CFBA0
:10057000054601464FF07E500FF06AFB61690FF0AF
:1005800071FC2169064628460FF06CFC0146304696
:100590000FF060FBE0602046BDE87040FFF7A0BFB1
:1005A000000080BF38B50E201C4C0CF007F92188E4
:1005B0001B4B884205461A881DDA0023511AB1F5F3
:1005C000805FAABF1B03C3EB03330131142093FBED
:1005D000F1F10CF079FC134B1988F1B923889D4295
:1005E00010DAC3F57F630F33282091FBF3F1BDE8E8
:1005F00038400CF069BC9042D4BFC1EB0003C1EBA2
:100600000203DBE740F6FF718D42D4BFC3EB050167
:10061000C3EB0101C1EB0131E3E738BDB49CFF1F1F
:100620006A9EFF1F1C9EFF1F10B504460BF0C8FEFC
:10063000204610BD70B44C88A04220D9012301335C
:10064000DBB21CB2660031F8144084421D46F6D37A
:10065000A04211D005F10045013D965B31F815101F
:1006600032F81530401AF21A00FB02F0641A90FBBF
:10067000F4F4E01870BC7047905B70BC70470226C1
:100680000125E5E700280CDA064A434282FB0320F5
:10069000DA17C2EB600000EB4000A3EB8000C0F172
:1006A0000C007047ABAAAA2A2DE9F0470C200CF0E9
:1006B00051F80C200CF006FDBB4914200CF012FD83
:1006C000BA49BB4809F04AFD022103200CF0A0FD05
:1006D000022104200CF09CFD022105200CF098FD65
:1006E000022106200CF094FD01210A200CF090FD5F
:1006F000012109200CF08CFD01210D200CF088FD5A
:10070000012128200CF084FD012114200CF080FD33
:10071000012116200CF07CFD172001210CF078FD42
:1007200004200CF067FD00283BD005200CF062FD92
:10073000054600283CD0002528469E4C207006F037
:1007400069FF24784CBB284608F06AFB9A4B9B490A
:100750001B889B4D098829709A4A9B4EA3F5AF715F
:1007600040F23A7303FB01F382FB0312DB17A3EBA6
:100770006213323301210D2033600CF035FD64200B
:100780000CF06EFD4FF416710A200CF09DFB5D21FC
:100790008E480AF08DF890B9FEE7BDE8F04709F001
:1007A000EDBB06200CF026FD0028BED10125C4E7D4
:1007B00003200CF01FFDB0FA80F04009BDE7642073
:1007C0000CF04EFD21460A200CF07EFB4FF4967192
:1007D00009200CF079FB5C217D480AF069F800B92A
:1007E000FEE764200CF03CFD214609200CF06CFB78
:1007F0004FF4967116200CF067FB5B2175480AF0E8
:1008000057F800B9FEE764200CF02AFD21461620B7
:100810000CF05AFB4FF4967117200CF055FB642036
:100820000CF01EFD214617200CF04EFB64200CF04E
:1008300017FD21460D200CF0D7FC674A6748126867
:10084000DFF8E8A1DFF8A091654EDFF8E481654F9D
:1008500000230121FFF728FE0123C9F8004034607E
:10086000C8F800408AF8003004240F200CF0EAFE9B
:10087000D8F8003003440E20C8F800300BF09EFF7B
:10088000D9F800309AF800200344C9F80030152048
:10089000002A78D00BF092FF33681844306004F0DF
:1008A000010080F0010005F0D5FB3B88002B14BF50
:1008B0004B20DC200CF0D4FC013CD6D1D8F8003021
:1008C000D9F80020484930683C88DFF868E1474F94
:1008D000002BB8BF0333002AB8BF033292100A605E
:1008E0004349444A098812880028B8BF03309B1046
:1008F000801030605E1A19443E60CEF800103E4F02
:100900003E4E3F49C8F80030C2EB000E0244C7F823
:1009100000E032600B605CB94FF4FA7005F0AAFB9E
:1009200005F094FB07F072F94FF4AF600CF098FCFF
:10093000344B012404201C600CF05CFC10B9324BD9
:1009400028701C70314B1B881C2B23D0304C04F1B9
:10095000C80523200BF032FF44F8040F01200CF0EF
:100960007FFCA542F5D12B4A2B4B1078187008F06C
:1009700061F905F067FB45F6BF5228492848BDE8F4
:10098000F0470BF0D3BC11200CF05CFE3368184428
:10099000306084E7234B18880028D7D0224BC0B2A0
:1009A000197808F08FF8D1E7001B374640420F0056
:1009B000D090FF1F209CFF1F649EFF1F7A9EFF1F89
:1009C0007C9CFF1FB5814E1B048AFF1F1C9CFF1FD0
:1009D000AC9CFF1F509CFF1F2489FF1FE09DFF1F41
:1009E000E09BFF1F0E9EFF1FFC9BFF1F389EFF1FFB
:1009F000168AFF1F5C89FF1F449CFF1F809CFF1FFE
:100A00007C9EFF1F409EFF1F0B9CFF1F469EFF1FEB
:100A1000C09CFF1FD09DFF1FAF9DFF1FA5050000BD
:100A20005C9EFF1F849CFF1F3E9CFF1FD49DFF1FE9
:100A3000349EFF1FB49DFF1FF0B40E8886420DD276
:100A400003F10043013B31F81350854202D9F0BC59
:100A5000FFF7F0BD32F81300F0BC70471088F0BC0F
:100A6000704700BF094B1B880C2B09D8084A80B27D
:100A700052F8232028B143F6FE73984203D9108C14
:100A80007047108870470349FFF7D4BD189CFF1FBB
:100A9000A01501003C170100374A38491088384A30
:100AA000F8B5384B12881B68834248DB9342A8BFD5
:100AB000134698420B60C8BF002342DD101AB0F500
:100AC000804FAABF9B03C3EB8333013093FBF0F04D
:100AD000FFF7C8FF2C4B2D4F1C883B68C0F3C61591
:100AE00005FB04F47F2CA8BF7F249D42064608D056
:100AF000274B1B88002B38D1264B1B88002B30D16D
:100B00003D60254D2B689E4205D0214B1B885A1F06
:100B1000032A1DD92E60214D2B689C420ED0204BFC
:100B2000188848B11A4B1F4A1B88D35C834203D0F4
:100B3000C0B2E1B207F0C6FF2C60F8BDF8BD0346B5
:100B400008609A42D4BFC0EB0203C0EB0303B5E7D1
:100B5000144AD05C2030C0B206F07F0107F0B2FF2B
:100B6000D8E7284608F022F8CAE70E4A2946D05CA2
:100B700007F0A8FFC0E700BFB49CFF1FE89BFF1F62
:100B80006A9EFF1F189EFF1F009CFF1F5C9CFF1F9B
:100B9000049EFF1FA69CFF1F749EFF1FA89CFF1FA3
:100BA000129EFF1F088AFF1F2DE9F04F012089B018
:100BB0000CF048FDAF4B186000200CF043FDAE4B2D
:100BC000AE4A1B8810600C2B00F03B81AC4BAD4A49
:100BD00019880093AC4B52F8214000221A70AB4B9D
:100BE000AB4D1B88AB4A2E88013B32F91370002EA7
:100BF0005CD0A94BA94A1B88A9491278013B31F95D
:100C00001380002A40F0DF8011200CF01BFDA54B63
:100C10000193D3F800A00646B24540F3DF80A24B13
:100C2000DFF8A4921B88A14A012BD9F80030B2F852
:100C300000B09F4A02922046C8EB030800F09A8257
:100C40000FF0BCF8029A52F82B100FF00BF9014686
:100C500000200EF0FDFF0FF0CBFACAEB0802B04502
:100C6000B8BFB0469042CAEB080880F2968200FBFB
:100C70000888013298FBF2F08E4BDFF85082029325
:100C8000D8F80030034403EBD3735B10C8F800308E
:100C90002B88012B12D1884BDFF834B20393874B9A
:100CA000DBF8005004934FF0000A47E07D4B0193BE
:100CB000DFF814927F4BDFF8148202937E4B03938C
:100CC0001D460F200CF0BEFC2B689842824641DA8C
:100CD000754A1288012A00F01D82744A0593128811
:100CE000734D049220460FF069F8049ADFF8E0B1E2
:100CF00055F82210DBF800500FF0B4F80146002040
:100D00000EF0A6FF0FF074FAEF1B059B5745A7EBFB
:100D10000302B8BF5746FF1A9042BABF013200FB28
:100D20000777474397FBF2F7D8F80020634B04930B
:100D3000BB1803EBD3735B10C8F80030604B1B8803
:100D4000013B032B00F2B082DFE813F06301A9013D
:100D5000C4008601594B04931B68984240F3C2813A
:100D6000514A1288012A00F0A682504A079311883E
:100D70004F4A0691204605920FF020F8059A0699F1
:100D8000DFF84CB152F82110DBF800500FF06AF890
:100D90000FF02EFA079B2F445745A7EB0302A8BF7D
:100DA0005746FF1AD8F800309042BABF00FB0777C9
:100DB0000132474397FBF2F73B4403EBD3735B10DD
:100DC000C8F80030BAE715200BF0F8FC354B01935A
:100DD000D3F800A00646B2453FF721AF354B02934A
:100DE000D3F800A0B24580F289812F4BDFF8D8906C
:100DF0001B882E4A012BD9F80030B2F800B02C4ADB
:100E000003922046984400F070820EF0D7FF039AB8
:100E100052F82B100FF026F80FF0EAF9B045CAEBA4
:100E20000802A8BFB046CAEB08089042B6BF00FB54
:100E3000088800FB08F8013298FBF2F0DFF88C809C
:100E40001EE7204B1B78002B3FF4C0AE0C4B0D4A25
:100E5000198800930C4B52F8210001221A700EF0F1
:100E6000ADFF4FF07C510EF0FDFF0FF0C1F90446CD
:100E7000B5E600BF4C9CFF1F469EFF1F889EFF1FCC
:100E8000529CFF1F8889FF1FF29BFF1F148AFF1FC0
:100E9000C09DFF1F841A0100648AFF1FD49DFF1F9D
:100EA000F4160100449CFF1F929CFF1F149CFF1F1F
:100EB0009C1A0100809CFF1F389EFF1FB49DFF1FDE
:100EC0005E89FF1F0A9CFF1FE09BFF1F4C9EFF1FB8
:100ED000349EFF1F28460EF071FFB2490EF0C2FF8C
:100EE000054650460EF06AFFAF490EF0BBFF0146C3
:100EF00028460EF0AFFE0FF07BF90546CBF8005008
:100F0000D9F800000EF05AFFA6490EF0ABFF0746D5
:100F100030460EF053FFA4490EF0A4FF01463846B8
:100F20000EF098FE0FF064F9C9F800009F4AA04B3C
:100F3000168819889F4AA04B12681B889F4FC6EBE2
:100F4000050E3544039EC6F800E0461A084404998D
:100F50000D6001990E6002993E8808609A4280F205
:100F600089810025C3EB060E954974450F6880F210
:100F70007681611C9F4205FB01F50EF1010E95FB88
:100F8000FEF5C0F2BE81BE42A8BF3E46F61A01FB86
:100F900006F494FBFEF49A4200F33681BB42C0F2A1
:100FA0003381884C20680EF009FF87490EF05AFF04
:100FB00086490EF04FFE0FF01BF9A0F5FF531C3BC6
:100FC000082B98BF4FF40050D8F800301844002880
:100FD0002060C0F24281B0F5804F80F252817C4B9C
:100FE0001B781BB1B0F5005F40F05381794D2B7831
:100FF000002B40F05481784D20682B68714C98424A
:1010000004D080B207F03CFE23682B6009B0BDE835
:10101000F08F28460EF0D2FE70490EF023FF0546F1
:1010200050460EF0CBFE6E490EF01CFF01462846DE
:101030000EF010FE0FF0DCF80546CBF80050D9F8A2
:1010400000000EF0BBFE65490EF00CFF074630466F
:101050000EF0B4FE62495FE728460EF0AFFE5A4933
:101060000EF000FF054650460EF0A8FE5D490EF05A
:10107000F9FE014628460EF0EDFD0FF0B9F80546E1
:10108000CBF80050D9F800000EF098FE4E490EF053
:10109000E9FE074630460EF091FE52493CE72846ED
:1010A0000EF08CFE50490EF0DDFE054650460EF067
:1010B00085FE4E490EF0D6FE014628460EF0CAFDCA
:1010C0000FF096F80546CBF80050D9F800000EF066
:1010D00075FE45490EF0C6FE074630460EF06EFE20
:1010E000424919E7D8F80030DFF810B103EBD373A9
:1010F0005B10DBF80050C8F800301FE6DFF8008115
:10110000DFF80091D8F8003003EBD3735B10C8F818
:101110000030BDE5364A06931188364A05912046CF
:101120000492DFF8D8B00EF049FE049A0599DBF876
:10113000005052F821100EF095FE0FF059F8EF1BF9
:10114000069B5745A7EB0302B8BF5746FF1AD8F8CE
:1011500000309042BABF013200FB0777474397FB4C
:10116000F2F73B4403EBD373234A04925B10C8F8B5
:101170000030E3E50EF022FE029A52F82B100EF03A
:1011800071FE0FF035F8CAEB0802B045B8BFB046A3
:101190008242CAEB08083FF76AAD00FB08F898FBEB
:1011A000F2F069E5CDCC4C3FCDCC4C3E168AFF1F0A
:1011B0005C89FF1F4C9CFF1F149EFF1F309CFF1F6C
:1011C000889EFF1FBC89FF1F9A99193FCDCC4C45C3
:1011D0003A9FFF1FA49CFF1F2089FF1F3333733FDB
:1011E000CDCC4C3DCDCCCC3E6666663FCDCCCC3D27
:1011F000149CFF1F9C1A0100B49DFF1F349EFF1F0B
:101200004C9EFF1FE09BFF1F009B1B88002B3FF4A1
:10121000C8AE2B1B002BB8BF5B42092B47DD05F581
:1012200000500130001B0EF0C9FD3B493B4C0EF055
:1012300019FE054620680EF0C1FD39490EF012FE78
:10124000014628460EF006FD0EF0D2FFD8F8003019
:10125000184400282060BFF6BEAE002213E09F4273
:1012600005FB04F5B8BF002195FBFEF54BDA91FBB9
:10127000FEF490E6B242D4BFC3EB0205C3EB060511
:1012800070E643F6FF72274B22601B78002B3FF479
:10129000ADAE04F0DBFE244B01221A70ABE604F085
:1012A000D1FE00232B70A6E6D9F800003EE64FF4ED
:1012B00000501A4C88E61D491D4A069320460D88A9
:1012C00005920EF07BFD059ADFF868B052F8251004
:1012D000DBF800500EF0C6FD014600200EF0B8FC11
:1012E0000EF086FF2F44069B56E50EF067FD039A2D
:1012F00052F82B100EF0B6FD014600200EF0A8FCAF
:101300008AE51E4642E6B742D4BFC3EB0701C3EBF2
:10131000060104FB01F1AAE7CDCCCC3EBC89FF1F3E
:101320009A99193F3A9FFF1FA49CFF1F149CFF1F0F
:101330009C1A0100349EFF1F08B5244B1B88FBB18B
:10134000234B1B78FBB1234B1B78E3B1224B1B785B
:10135000CBB1224B1B78B3B1214B22481A78C2B9CA
:10136000214A22490088128809680244B1EB620FC1
:1013700009DD01221A706420BDE8084004F07ABE3D
:10138000174A117801B908BD1370BDE8084007F08D
:1013900041BC154A16490088128809680244B1EB1D
:1013A000620FF0DD00221A7007F034FC642004F0B4
:1013B00061FE642004F05EFE642004F05BFE4FF4E6
:1013C0001670BDE808400BF04BBF00BFC29DFF1F69
:1013D000669EFF1F679EFF1F689EFF1F699EFF1F7F
:1013E000169CFF1F309CFF1F149EFF1F4C9CFF1F6D
:1013F000889EFF1F38B5114C232025780BF0DEF9AD
:101400000F4A42F82500131F02F1C400002253F8CE
:10141000041F83420A44FAD123780A4907480A4C38
:101420000133DBB2322B81FB025108BF0023D217FC
:10143000C2EB21120370226038BD00BF029CFF1F67
:10144000C49CFF1F1F85EB51309EFF1F2DE9F04FFD
:10145000B84CB94D2068B94F83B00EF0AFFCB84915
:101460000EF000FD064610200CF0ECF80EF0A6FC85
:10147000B4490EF0F7FC31460EF0ECFB0EF0B8FE6E
:101480002988206088423B8843DA9E465B1A7F2B7E
:101490004FF0000247DDD2015E1C92FBF6F2AA4E2D
:1014A000DFF8C882B6F800C0C8F80020BCF1190FF8
:1014B00000F0DF80BCF11A0F00F01781BCF11E0FA5
:1014C00000F020810126B146A04A1288002A00F0CF
:1014D0009D808842C0F207817045D4BFC1EB0000F7
:1014E000C1EB0E009A42BABF02FB00000133504329
:1014F00090FBF3F3964A1360964B1888C0B9964A4E
:101500001288AAB9954B197801B11A7003B0BDE8D9
:10151000F08F9842D4BFC1EB0002C1EB03029E469C
:101520005B1A7F2BB7DCC2EBC21292FBF3F2B6E779
:101530002988D4F800E0DFF80082DFF8F8A17145CF
:101540006CDCDFF818C29CF80020002A2ED14FF086
:10155000010B04288CF800B028D1002E40F09481B3
:101560007D4B18880028D1D0B9F1000FCED0236868
:101570002C883A88A34280F265810023141B7E2CBC
:10158000774DD5BFC3EB8313C3EBC3135B000134AB
:1015900093FBF4F42B680134A34203D0C0B2E1B250
:1015A00007F090FA2C6003B0BDE8F08F012800F03E
:1015B000F680022800F0EB800328D1D1694B1B880C
:1015C000092BCDD0002ECBD023682E883A88B34289
:1015D00080F27B810023961B7E2EDFF88CA1D5BF85
:1015E000C3EB8313C3EBC3135B00013693FBF6F627
:1015F000DAF800300136B34203D0F1B24A2007F0E6
:1016000061FACAF80060ABE716469146BCF11E0FBE
:101610007FF472AF0022DFF858817EE04F4B1A78DA
:10162000002A3FF473AF002401281C7000F0A4804E
:10163000022840F00E81002E00F0A3804A4D2B6856
:10164000002B00F09E800420214607F03BFA424B1D
:101650002C60188800283FF459AFB9F1000F3FF40F
:1016600055AFC0B2002107F02DFA3D4B00221A60A1
:101670004CE7DFF8FC8098F80020C2B1DFF8D89082
:10168000B9F800A0BAF1000F11D0DFF8E89099F88E
:1016900000B0934578D05FFA8AF07F2107F012FA04
:1016A00098F80030B6F800C089F8003010E0DFF894
:1016B000C49099F800A0924566D0274B0021187875
:1016C00007F000FA98F80030B6F800C089F800304A
:1016D0001E4B1A88002A97D0BCF11E0F40F00681DD
:1016E0000026B14619E00020FCE6DFF8848098F877
:1016F0000020002A0BBF012600264FF000094FF002
:101700000109E1E6DFF86880104B98F800601A885C
:10171000B6FA86F676094FF0000998F80030002BEB
:101720003FF4E8AE2988B7F800E02068C1EB0E036B
:10173000CFE600BF409CFF1FC89DFF1FC49DFF1F39
:101740009A99193FCDCCCC3E469EFF1F709EFF1F3D
:10175000BC9CFF1F4A9CFF1F529EFF1F4B9EFF1FFA
:10176000249CFF1F049EFF1FC09CFF1F2C9EFF1F79
:101770000A9CFF1F069CFF1F1EB1614D2B68002BAA
:101780007BD1604B188865E70026B1469CE6002EA9
:101790003FF4E6AEDFF868A1DAF800202EE0002E74
:1017A0003FF4DEAEB7F80080F045D4BFC1EB0802CD
:1017B000C1EB0E02C1EB0808B8F17E0FDFF840A1C3
:1017C000D5BFC2EB8212C2EBC212520008F101086F
:1017D00092FBF8F8DAF8002008F10108424506D03B
:1017E0005FFA88F10120009307F06CF9009B1888DC
:1017F000CAF8008002287FF4DFAE42462168B5F8BF
:1018000000803888414559DA0021C8EB0008B8F15A
:101810007E0FD3BFC1EB8111C1EBC11108F10108EB
:10182000490091FBF8F808F10108904506D05FFAED
:1018300088F10420009307F045F9009B1888CAF846
:101840000080B9E69342D4BFC4EB0303C4EB0203A8
:1018500094E6032827D12C4B1B88092B91D0002E0E
:101860008FD0274D2B68002B8BD04A20214607F0C4
:1018700029F9244B2C601888ECE6214607F022F960
:10188000204B2C601888E5E640207F218DE80C0075
:1018900007F018F9019B009A188858451CD00228B7
:1018A0007FF48AAE76E704287FF46BAF002E3FF416
:1018B00068AF2146402007F005F962E78142D4BFB6
:1018C000C8EB0101C8EB00019FE79342D4BFC6EB10
:1018D0000303C6EB02037EE6B8F80010DAF800E076
:1018E000B7F800808E45FFF665AF5DE72988B7F849
:1018F00000E020680026C1EB0E03B146E9E500BF19
:10190000C09CFF1F529EFF1F049EFF1F08B50F4B78
:101910001B88022B0FD0032B12D0042B03D00C4BAF
:1019200001221A7008BD7F21092007F0CBF8084B6F
:1019300001221A7008BD7F21412007F0C3F8EEE7AD
:101940004021092007F0BEF8E9E700BFB89CFF1F5F
:101950006E9CFF1F38B51C4B1B881D2B26D01B4BC4
:101960001B88012B25D01A4A1A4B14881B681A4A67
:10197000A342128818DB9342D4BFC4EB0303C4EB29
:101980000203141B7F2CC6BFDB010134C3EBC3135E
:1019900093FBF4F4114D2B689C4203D0E1B2052077
:1019A00007F090F82C6038BD0023EAE70C4B1C8848
:1019B000F0E70C4B0C4A0D491B6812680C689B1A27
:1019C0001C1B84F30704E5E7469EFF1FC09DFF1F15
:1019D0006A9CFF1FF89BFF1F449EFF1FEC9BFF1F8D
:1019E0003E9CFF1F7C9EFF1F2889FF1FCC9DFF1F71
:1019F00010B50F4C23685BB90E4B1B88022B11D01E
:101A0000033B012B09D90C4A00231370236010BD3E
:101A10000021052007F056F8EEE70021092007F025
:101A200051F8F0E70021412007F04CF8EBE700BF48
:101A3000EC9BFF1FB89CFF1F6E9CFF1F08B5274B38
:101A40001B78ABB115200AF0B9FE254A254B128848
:101A500018601D2A15D0244A1288EAB1012A25D01F
:101A6000224B1B78002B34D0BDE80840FFF7C0BFE5
:101A700011200BF0E7FD1A4A1A4B128818601D2A34
:101A8000E9D11B4B1B78002BEAD0184B1B780BB30A
:101A9000BDE80840FFF75EBF164A1288002ADFD073
:101AA000154A1B6812889A42DADCEEE70F200BF029
:101AB000C9FD104B114A1B88106033B1104B114AFD
:101AC0001B6812689B1A9842DFDD084B1B78002BBD
:101AD000CAD108BDFFF71AFFDAE700BFD49DFF1F88
:101AE000469EFF1FF89BFF1FC09DFF1F6E9CFF1FA0
:101AF0000A9CFF1FB89CFF1F6A9CFF1FCC9DFF1F05
:101B00007C9EFF1F2889FF1F2DE9F04FAC4C2678E3
:101B1000012E95B000F04582C0F0FB81022E00F04E
:101B2000CB80A849A84A91F800801178A74ADFF82D
:101B30002CE3A74DA74FA848A84B0292A84A0092B1
:101B4000A84A9EF800B001922D78A74A3F7890F8F5
:101B500000E01B78DFF80CA3DFF80CC3DFF80C9370
:101B60000392012E84BF00222270A04AA048137065
:101B7000A04A80F800B015709F48A04A077082F80C
:101B800000809F489F4A03709CBF013626701170E9
:101B9000BEF1000F40F009819B4A10880D2800F02B
:101BA000A9819A4C00202070024604462DB1964827
:101BB0000088002840F0AA810546954806882544FB
:101BC000002E40F057819348934C019E0078367860
:101BD00024780130A0EB4600002C40F04682039CA4
:101BE00094F800E0CEEB0004BEF1000F40F06682F6
:101BF0000026DFF864E202989EF800E00078A41B5B
:101C0000A4EB4E043C44CBEB040410B1B7FA87F0CC
:101C100040099CF800602718BC1B1EB11EF100068D
:101C200018BF0126009F99F8000097F800909AF8D5
:101C300000C07A4FC6EB040EC0EB0E00A0EB4900CB
:101C40008044C3EB0803A3EB41010C2313FB0C11ED
:101C50003960734B734C744E1B8874482488376802
:101C60000088734E033B03EB4303C4EBC40401EB56
:101C700083033C4403440C3B56F824001D440544B4
:101C80000AB16C4B19606C4B1A68954200F02E81BA
:101C90006A4A6B48116807910799016012680892B7
:101CA0006848089A00881D60521A824284BF664ABA
:101CB000156015B0BDE8F08FDFF8B481634E08AF52
:101CC0000025E9B2624808F0B7FD58F8043BC3F5B7
:101CD000967300FB03F086FB00230135C017C0EBB1
:101CE00063100C2D47F8040BEBD15A4B3D4D019579
:101CF0003D4DB3F800C00395109D09980F99464ECD
:101D0000DFF8D4A0DFF8C890DFF8D080654511AACD
:101D10008CCAAE46ACBF4FF0000E4FF0010E8445AA
:101D2000D4BF0020012030708C452E480B9D254EDD
:101D30008AF800E0D4BF00210121017094452A49AE
:101D4000DFF820A1D4BF002201220A709C45424A3C
:101D5000D4BF00230123BC45AB46D4BF00270127D5
:101D60001370AC451B4B0C9D1F70D4BF4FF0000B84
:101D70004FF0010B394B154A0292AC45DFF848C0D1
:101D8000174A83F800B0D4BF0025012589F8005018
:101D900098F800309CF8001096F80080DFF8C8C072
:101DA0002678DFF8C8900092DBE62D4A17481488A1
:101DB0000122182C027040F260810024F6E600BF78
:101DC000AE9DFF1F009EFF1F029EFF1F949CFF1FE2
:101DD000909EFF1F6C9CFF1F959EFF1F019EFF1F83
:101DE000499EFF1F559EFF1F569EFF1F8F9EFF1F80
:101DF000C79DFF1F919EFF1F929EFF1F939EFF1F77
:101E0000949EFF1F4A9EFF1F969EFF1F0A9CFF1F66
:101E1000F09BFF1F188AFF1F809EFF1F089EFF1F59
:101E2000209EFF1F3C9EFF1FBC9CFF1F049CFF1FAA
:101E3000B4180100389CFF1F649CFF1F7C9FFF1F8C
:101E4000549CFF1F509EFF1F849EFF1FB5814E1B99
:101E5000AC9CFF1F649EFF1F579EFF1F6D9CFF1FC2
:101E6000469EFF1FB99DFF1F8E9EFF1F489EFF1FAE
:101E70002C89FF1F012E00F08F81022E00F0EE81D1
:101E8000032EA74B00F01F811E78009B9CF800E0FA
:101E90001C78019B99F800C01878029B93F8008089
:101EA000039B1F78A6EB4E03A4EB8404CCEB030C3E
:101EB000C0EB80760CEB0403C0EB8600034403EB1D
:101EC000480303EB810327B196490978002940F0C4
:101ED000608201269AF800109348C1F1060101EBD7
:101EE0004101334403EB81010160B2E68F49904A1E
:101EF0000968D3E6002D3FF454AE8E4A8E4E148806
:101F00000122182C327040F2B8807446A0F10D0501
:101F100053E6DFF87092894F0DF120080025E9B2F1
:101F2000874808F089FC59F8043BC3F5967300FB19
:101F300003F087FB00230135C017C0EB6310062DAB
:101F400048F8040BEBD17F4BDFF83CA219880D9BBE
:101F500000228B428AF8002080F2A2807A4B8AF815
:101F600000507A497A4A7B4891F8008011787A4A81
:101F70001D7002920378794ADFF810C2DFF81092E0
:101F80000092774A774E784D784892F800E0784A88
:101F90000192784A96F800B02D7807782678039257
:101FA000DFE5DFF8F081654E08AF0025E9B2724841
:101FB00008F042FC58F8043BC3F5967300FB03F0AD
:101FC00086FB00230135C017C0EB63100C2D47F8CA
:101FD000040BEBD15B4B0C9D1F885F4B02935F4B57
:101FE00000930B9B0A98099ADFF8A0C1089EDFF8BE
:101FF000A0910F99BB429E46ACBF4FF0000E4FF030
:10200000010EAF42D4BF002501258742109B8CF8FA
:102010000050D4BF00200120504D89F800009742A5
:10202000D4BF00220122B742D4BF4FF000084FF0C6
:1020300001082A709F42474A4448474E80F8008072
:10204000D4BF002301231370129A414886F800E0A0
:102050008F42D4BF00210121974201701ADC002277
:102060004648DFF824A102708BE7039C46B126782E
:10207000002E40F06081441EBBE50C3C012295E53A
:1020800094F800E00138CEEB0004BEF1000F7FF4BD
:10209000B0ADADE5119A9742D4BF00220122DFE72F
:1020A0000C9A374B9142CCBF012200221A7040F3A8
:1020B000458105258AF80050234B52E7002E3FF456
:1020C00097AD012695E51C78009B029893F8008057
:1020D000019B9CF800601B7890F800C099F8007094
:1020E0000398A4EB4604E71B90F800E0C3EB83746D
:1020F000A8EB88003844C3EB8403034403EB4C0390
:1021000003EB8103BEF1000F40F0488101269AF8ED
:102110000010054833440C2414FB0131016098E59C
:10212000188AFF1F579EFF1F089EFF1F549CFF1F0A
:102130007C9FFF1F469EFF1F0A9CFF1FB5814E1B01
:102140001C9CFF1F649EFF1FC69DFF1F009EFF1F5C
:10215000029EFF1F019EFF1F949CFF1F499EFF1FB1
:10216000959EFF1F6D9CFF1F909EFF1F6C9CFF1F85
:10217000559EFF1F569EFF1F509CFF1F369CFF1F42
:10218000699EFF1F4C8AFF1FB99DFF1F8E9EFF1F78
:10219000489EFF1F1C8AFF1FA34CDFF89CE220789B
:1021A00005909EF8004001980494059C00780190E9
:1021B0000134A4EB40040498002840F0AF80039859
:1021C00090F800E00498261ACEEB06000390BEF1CA
:1021D000000F40F09E8074460298944E0078029062
:1021E000039836780496041BA4EB460402983C44FA
:1021F000CBEB0404002800F08780B7FA87F0400991
:102200009CF800602044871B1EB10498061C18BF70
:102210000126009C99F800002478BE1B301AA0EB20
:10222000440080440198C3EB0803A3EB410300285A
:1022300067D1BEF1000F40F0BB807344002C5ED12B
:1022400000290CBF00206FF009009AF80010784CAC
:1022500003440C2010FB01312160FAE4039E019C31
:1022600036780396009E2478019434786F4E714836
:1022700099F800E0009496F800906F4C9DF80C607F
:1022800086709DF80460067080F806E09DF8006096
:1022900080F803909CF800C02478DFF8B491DDF852
:1022A00004E080F80880077180F805C0C6714172AB
:1022B00044704FF000080120009500215D4C0D4650
:1022C0005FFA88FC4F46764607E0022809D00A29C3
:1022D0000BD014F8016F17F8010F864201F10101CC
:1022E000F3D101350A29EDB2F3D1092D72D808F1E5
:1022F0000108B8F1100F36D019F80A0FDDE70020F9
:10230000A3E74FF0000E98E7029879E7CEEB0400C0
:1023100003900198041C18BF01245DE70198002870
:102320004ED0039890F800E0BEF1000FEED1601E91
:102330000390744650E7841B01265AE40B9A3F4BE6
:102340009142CCBF012200221A703EDC0A9A3C4B1B
:102350009142CCBF012200221A7052DD03258AF877
:102360000050384BFDE5304837490478C86B029976
:10237000009D097801342044CBEB00000844002183
:102380009AF800402A4B401A0C2111FB04011960F5
:102390005FE41BF1000618BF01269BE5234909787D
:1023A00000293FF4B3AE1BF1000618BF0126AEE6CC
:1023B000049800280CBF4FF0000E4FF0090E3CE7C8
:1023C000039890F800E03046FDE604258AF80050B6
:1023D0001C4BC6E514481C49047851F828000299A2
:1023E000009D097801342044CBEB00006646084488
:1023F000002BC4D0002EC2D1BBF1000FBFD00121F1
:10240000BEE7099A114B9142CCBF012200221A70FB
:1024100004DD02258AF800500A4BA2E5089B994288
:1024200018DD01259AE500BF188AFF1F579EFF1F80
:10243000089EFF1F889CFF1F809EFF1F689EFF1F36
:10244000679EFF1FC69DFF1FC489FF1F669EFF1F5B
:1024500060170100134B1D78012D21D9124A8AF80B
:1024600000501288002A3FF47CAD104A1288013ACD
:1024700092B2062A3FF675AD0D4A1278002A3FF453
:1024800070AD0C4A1268012A7FF46BAD0A4A0B4EFC
:1024900010680C2290FBF2F102FB1102328060E521
:1024A00035465EE5C69DFF1F8C9EFF1FD29DFF1F18
:1024B000B69CFF1F409EFF1F849EFF1F0C9EFF1FA8
:1024C0002DE9F04F3A4B1B788BB0002B6AD10E20D0
:1024D0000AF074F90DF072FC01463648364E374D5D
:1024E000FEF728F83348FDF7FBFF0DF081FE80F37F
:1024F0000C003060FFF708FB2C68012C7AD0022C0E
:1025000000F09F82032C00F0AD832D4E33682D4ADE
:102510002D4E0993099B316812882C4C591A013AA7
:102520009142236000F28882294E32689A1A0D2A5D
:1025300000F27B82274E32689A1A132A00F27082C8
:10254000254E32689A1A252A1AD9244B1B88002B4B
:1025500040F05F81224B1B78002B40F05A81FEF740
:1025600049FF204B1B881B3B9BB2022B04D81E4B00
:102570001B78002B40F0508103F08EFD2368336000
:102580001A4D2A689B1A502B00F20682184B1B88A2
:10259000012B00F01E8206F029FB06F057F90BB064
:1025A000BDE8F08F07F072FB0BB0BDE8F08F00BF05
:1025B000209CFF1FE09DFF1F189EFF1F409EFF1FD6
:1025C0007C9FFF1FC089FF1FB09CFF1FDC9DFF1F6A
:1025D0009C9CFF1F749CFF1F789CFF1FC29DFF1FC8
:1025E000169CFF1F469EFF1F0A9CFF1FBC9DFF1FDE
:1025F0001C9EFF1FDFF810939E4AB9F80000137865
:10260000834204D0C3B21846137006F02BFADFF8E9
:10261000F482994AB8F800301178994204D0974F63
:102620003978002940F0F186954A33681288954E32
:102630009A42C0F2F680944A1278002A40F0F18063
:10264000DFF8C8A2BAF8003023B9904B1B88002BE2
:1026500000F0EF848E4A8F4B11881B888E4A0B4402
:1026600012685B1093428D4A126880F291840021B7
:102670009342B4BF01230B4604910093ACBF4FF0CB
:10268000010B8B4605910E200AF098F8844B854A81
:102690001B68176803930133A7F25232002B84465C
:1026A000029240F3C386802BA8BF80237E4A7F49D5
:1026B00012780191002A00F0BE800978914200F062
:1026C000BA80B8F80010DFF83CE2994201F09B8034
:1026D0006A49AEF80030764B4FF0010E81F800E009
:1026E0001978DFF82CE2019B8EF800101A70009B1D
:1026F000002B00F00F81BAF80030002B00F00A81A7
:102700006C4B1B685A1C002A40F39486802A00F305
:102710009086694C69496A48248809880068214480
:10272000B0EB610FC1F2E282A3F148020F2A02D896
:10273000473BA9F800300E200AF040F86FF45473BC
:102740001F44874202DC5F4B00221A705E4B1B88DD
:10275000002B00F015845D4B5D4A1B78117899427F
:1027600040D0002B3ED05B490C78002C00F0148741
:10277000594991F800C0BCF1000F40F00B87574F4A
:102780000097574F57480297544F007887F800C07A
:10279000534F4FF0010E87F800C081F800E0002889
:1027A00041F0B18050490978002900F0D5874F49A0
:1027B00003910C460978002940F0CB874C48484FDC
:1027C0000078397001210297217058B1434842497D
:1027D0000090002008700099029F0870039901245E
:1027E0003C7008701370434B1B88A3F11B02012A35
:1027F00040F2E6851D2B7FF489AE3D4F3B78002BE0
:1028000041F048803C4C2378002B40F086842370B4
:102810007CE6FEF791FDA2E62B68012B7FF4ACAEBF
:10282000ACE63168354A06910698354910600222B7
:102830000B602A6004E71E49DFF8D4E0097800291C
:102840003FF451AF9EF8000081423FF44CAF039833
:102850004B2840F39F871833802BB8F80000A8BF9F
:10286000802398423FF43FAF26480380034801236A
:10287000037038E7AF9DFF1F7C9CFF1F0B9CFF1F61
:10288000B49CFF1F7C9FFF1F169CFF1FA29CFF1F75
:10289000309CFF1F149EFF1F4C9CFF1F889EFF1F34
:1028A000389CFF1FFC9BFF1F789EFF1F609CFF1F33
:1028B000799EFF1F089EFF1FC89DFF1FC49DFF1F1D
:1028C000409CFF1FB89DFF1FD29DFF1F369CFF1F1E
:1028D000E49BFF1F929EFF1F109EFF1F549EFF1F31
:1028E000B69CFF1F939EFF1F8F9EFF1FE59BFF1F40
:1028F0000A9CFF1F469EFF1F069CFF1F709CFF1F28
:10290000D89DFF1F7A9EFF1FD09DFF1F689CFF1F51
:10291000619CFF1F029B9C45BFF60DAF864B1B8839
:10292000002B3FF408AFBBF1000F7FF4E9AE834BFF
:102930001B881BB1059B002B7FF4E2AE049B002B90
:102940003FF4F9AE7E4B1A78002A7FF4F4AEDFF83C
:10295000649299F8004001221A70002C40F03683EE
:10296000784B1B78002B02F03780774B1B78002BBD
:1029700002F00283754B1B78002B7FF4DCAE744BA6
:102980001B78002B3FF4D7AEB8F8003071490A3BF2
:10299000A8F800300A70CEE604F084FE6E4B1B7877
:1029A00073B96E4B1B785BB96D4B1B7843B96D4B9C
:1029B0001B782BB96C4B1B7813B903F043FB01E078
:1029C00003F04CFB23682B60684B1B88012B7FF4C2
:1029D000E2AD674A674B116867481A78A1F118039E
:1029E0002A2101FB03F10160002A00F0B382634C4D
:1029F0002368994200F35C8310DA61480278002A68
:102A000040F03E875F4A1068D0F17F0048BF033036
:102A1000801001301B1A994242F3428621609BE2EA
:102A2000FFF70CF8236833608AE5FEF7BDF8FEF780
:102A30000DFD236833607DE5FEF72EF823683360D3
:102A400072E5514A34681188A14204DB464B1B7879
:102A5000002B00F05D834D4E4D48336807934D4B7E
:102A6000079A00681B88121A9A4200F2A980002B6C
:102A700000F0A680484B1A88002A3FF447AD474B28
:102A800047481B680088A342B8BF2346994241F3D8
:102A90002681444B1960DFF8208188F80020344FEC
:102AA000FDF7FAFF38687F2840F370853E4B7F388A
:102AB00083FB0032C317C3EB620303EB4303A0EBBA
:102AC00083007330394B01931B883860002B40F032
:102AD0008C86234B00931B78002B00F0CD83344C65
:102AE0002378002B00F0C883DFF8D090DFF8B8A07F
:102AF0004FF0000B0CE003F17300C0B298F8001027
:102B000006F008F823780BF1010B5B4540F3B48322
:102B10003B6859F8040F1844A0F17F038AFB032196
:102B2000DA17C2EB610202EB42027F28A3EB8203B9
:102B3000E1DCFDF7A7FDE0E7A29CFF1FD69DFF1F8C
:102B4000B89DFF1F8F9EFF1FC79DFF1F919EFF1FF8
:102B5000929EFF1F0B9CFF1FB69CFF1F109EFF1F26
:102B6000549EFF1FE59BFF1F169CFF1F1C9EFF1F0F
:102B7000849EFF1F6E9CFF1F6C9EFF1F109CFF1FFB
:102B8000589EFF1FEC9BFF1FB49CFF1F7C9FFF1FE5
:102B9000709CFF1FA09CFF1F089CFF1FD89DFF1F5C
:102BA0006A9EFF1FE89BFF1FABAAAA2A489CFF1F33
:102BB0008489FF1FB99DFF1F959CFF1F5C89FF1F24
:102BC000554B564A1B681088554AA342B8BF234646
:102BD000994200F38482534C12888342A8BF034673
:102BE0002360002A7FF457AF9942C8BF134640F3D1
:102BF0007D82401AB0F5804FAABF9B03C3EB83339D
:102C0000013093FBF0F0FDF72DFFC0F3C6100DF07F
:102C1000D5F8454B044618880DF0D0F843490746CF
:102C200020460DF01FF9014638460DF01BF92146EC
:102C30000DF010F84FF07E5104460DF0B1FA002867
:102C400041F031803A4920460DF0C8FA002840F0A2
:102C5000548620460DF0F2FAC0B2DFF8F48088F80E
:102C600000001CE7334B34681988A14274DD324BF5
:102C70001B78002B70D1DFF8DC9099F800007F28DA
:102C800040F3FA85A3F155337F3803F1004383FB0A
:102C90000032C317C3EB620303EB4303A0EB8300D3
:102CA0007330264B01931B88C0B289F80000002BBB
:102CB00040F0EB87224B00931B78002B00F09984A7
:102CC000204C2378002B00F094841F4FDFF87C8089
:102CD0004FF0000A0AE003F17300C0B205F042FFB2
:102CE00023780AF1010A534540F3838457F8043FDF
:102CF00099F800001844A0F17F0388FB0321DA173C
:102D0000C2EB610202EB42027F28A3EB8203E2DC0A
:102D1000FDF7B8FCE1E700BFD89DFF1F6A9EFF1FCB
:102D2000089CFF1FE89BFF1FF49BFF1FCDCCCC3DF1
:102D30000000FE42B49CFF1F169CFF1F489CFF1F13
:102D4000549EFF1F8489FF1F5C89FF1FABAAAA2A1C
:102D5000959CFF1F069EFF1FB84F38687F2840F3E1
:102D6000CC81B74B7F3883FB0032C317C3EB6203C0
:102D700003EB4303A0EB83007330DFF8249399F84F
:102D800000A0824500F01F82AE4B1B88002B43D170
:102D9000AD4AAE4812680088914205DC8242D4BF39
:102DA000C1EB0203C1EB0003411AB1F5804FA6BF8E
:102DB0009B030131C3EB833393FBF1F0FDF752FE2C
:102DC000C0F3C6100CF0FAFFA14B044618880CF0B3
:102DD000F5FFA049804620460DF044F801464046E4
:102DE0000DF040F821460CF035FF4FF07E510446BF
:102DF0000DF0D6F9002840F0C286974920460DF024
:102E0000EDF9002840F0768520460DF017FAC0B2A3
:102E1000DFF8908288F80000BAF17F0F40F3B283A8
:102E20008748AAF17F0A80FB0A304FEAEA73C3EBB6
:102E3000600000EB4000AAEB80007330874B0093EA
:102E40001B78C0B289F80000002B40F01283844B3D
:102E500003931B78002B40F0F584824B02931B7880
:102E6000002B40F03487804B0193029B1B78FBB111
:102E70007E4B1B88012B00F00086022B00F0598747
:102E8000032B01F0EB80042B01F0EB82052B01F00A
:102E90000784062B01F06085072B01F0D185082BF4
:102EA00002F02A80092B02F02F810A2B02F0828285
:102EB000009B1B78002B00F05F84019B6A4C1988F3
:102EC000002900F0B58438687F2840F3CF825C4B3E
:102ED0007F3883FB0032C317C3EB620303EB43036A
:102EE000A0EB830073303860002940F06484009BBD
:102EF0001B78002B00F072815D4C2378002B00F0D2
:102F00006D81DFF8A4A1DFF89C814FF0000B0CE08D
:102F100003F17300C0B298F8001005F0FBFD2378B0
:102F20000BF1010B5B4540F359813B685AF8040FE4
:102F3000434A1844A0F17F0382FB0321DA17C2EB56
:102F4000610202EB42027F28A3EB8203E0DCFDF783
:102F500099FBDFE7474B1960474B1B68A92202FB2F
:102F600003F3002BBCBF03F57F533F339B13543B4C
:102F7000194481F30C01282009F0A6FFFFF70BBBD1
:102F8000384C3E483549364A237003700B7029E4AB
:102F900093424FF0000B80F2B3800123CDF800B0D4
:102FA000CDF814B00493FFF76EBB354B1B78002BA4
:102FB0007FF4C1AB039B334A243B83F34703D9B26D
:102FC0005B20136005F07EFD99F80040032C30D1A2
:102FD000DFF8D88098F80030002B42F022812A4F89
:102FE0003B78002B42F01081254C2378002B42F0D7
:102FF000FE80264B1B78002B42F0EC80244A138085
:10300000244B1B78002B42F018810E4B7F221A8034
:1030100098F800306BB93B785BB923784BB91E4AFE
:103020007F210720138005F04DFD7F210B2005F047
:1030300049FD1A4B1F68FFF77EBB00BF849EFF1F30
:10304000ABAAAA2A089CFF1FE89BFF1F6A9EFF1FCE
:10305000F49BFF1FCDCCCC3D0000FE42549EFF1FD1
:10306000E59BFF1FB69CFF1F489CFF1FD29DFF1FC3
:103070008489FF1F109CFF1FBC89FF1F109EFF1F2C
:10308000929EFF1F2C9CFF1F919EFF1FC79DFF1F3D
:10309000A69CFF1F939EFF1F049EFF1FFC9BFF1F0C
:1030A000069EFF1F959CFF1F5C89FF1F8F9EFF1FC1
:1030B000B04A1078002840F04383AF4A1268D2F13A
:1030C0007F0248BF033203EBA202531CAB4A2360CA
:1030D0009942B8BF1160FFF63FAF19463CE7A84BD5
:1030E00012881960002A7FF4D6AC0B469842D4BFF0
:1030F000C1EB0003C1EB03037BE5FDF7C3FA3CE63C
:103100000123CDF810B0CDF800B00593FFF7BBBA9E
:1031100001232B609B4EFFF7F9B99B4B6A2019885E
:1031200005F054FE3B782370FFF7F0B9029B1B7843
:10313000FBB1964B1B88012B00F01884022B00F08A
:103140007686032B01F00080042B01F0AF81052B64
:1031500001F02A82062B01F01484072B01F0C085B0
:10316000082B01F07D86092B01F0EF870A2B02F076
:10317000B281019B1B88002B00F02683009B1B78EB
:103180003BB9039B1B7823B9029B1B78002B00F0F3
:1031900054877F4B1B78002B00F035817D490B78DD
:1031A000082B00F230817C483A6800687B4C013380
:1031B000DBB25F1E101A44F827000B70784B34689E
:1031C000198889F800208C426E4E7FF79FA93268DB
:1031D000744B0892089A1A60FFF798B9039B1B7802
:1031E000002BA3D03B68A3F10C007F2840F327837A
:1031F0006D488B3B80FB0320DA17C2EB600000EBCD
:103200004000A3EB800303F17300DFF8AC81C0B290
:1032100098F8001005F07EFC009B1B78002B85D0F1
:103220005C4C2378002B81D0DFF890A14FF0000B8D
:103230000CE003F17300C0B298F8001005F06AFCCE
:1032400023780BF1010B5B457FF770AF3B685AF8B1
:10325000040F554A1844A0F18B0382FB0321DA17AF
:10326000C2EB61020C3802EB42027F28A3EB82031F
:10327000DFDCFDF707FADEE7454B1B78002B40F05B
:10328000A9823B68494A1278002A45D0A3F10C0074
:103290007F2840F3EE82444A8B3B82FB0321DA17FE
:1032A000C2EB610202EB4202A3EB820303F1730063
:1032B000C0B298F8001005F02DFC009B1B7853B3AA
:1032C000344C23783BB3DFF8F490DFF8DCA04FF008
:1032D000000B0BE003F17300C0B298F8001005F08A
:1032E00019FC23780BF1010B5B4514DD3B6859F8A1
:1032F000040F1844A0F18B038AFB0321DA17C2EBF9
:1033000061020C3802EB42027F28A3EB8203E1DC6E
:10331000FDF7B8F9E0E73B68254A1278FAB11B4A95
:103320001288012A00F02E84022A00F00186032A66
:1033300000F08387042A01F0E080052A01F018825A
:10334000062A01F02A83072A01F01984082A01F0CD
:103350005786092A01F09B860A2A02F08880019A82
:103360001288002A00F04882124903220B702A605A
:10337000FFF7CCB8589EFF1FEC9BFF1F109CFF1F50
:10338000E89BFF1F7C9FFF1F3E9CFF1FD29DFF1FDE
:10339000109EFF1F8489FF1F0C9CFF1F6089FF1F69
:1033A000B49CFF1F249FFF1FABAAAA2AE59BFF1F07
:1033B000B69CFF1F069EFF1F959CFF1F5C89FF1F89
:1033C000B04F3B78002B3FF41DAAAF4C207802F0A1
:1033D000CDFEAE4B1B78002B00F0748223887E2B31
:1033E00000F27082AA4A0133108899B22180002825
:1033F00000F07882C9B2C0B2A64C05F063FB3B78FE
:103400002370FFF783B83A68D8E6DBB2184613702A
:1034100005F036FBA04BA1491A46A14B18460023E4
:103420000B703B7013700370FFF7FEB80123FFF7BA
:103430003DB980249B499C4B9C4A09881B88126893
:103440000B44B2EB630FBFF676A98E4B1B78002BB3
:1034500040F0DF81B8F80030954AA3423FF46BA9F1
:10346000944B148001221A70FFF765B9FDF70AF931
:1034700039E5914B01931B88002B42F00B81884B5F
:1034800003938E4B02938E4C23786BB3DFF840820C
:10349000DFF830A24FF0000B09E003F17300C0B277
:1034A00005F060FB23780BF1010B5B451CDD58F840
:1034B000043F99F800001844A0F17F038AFB032120
:1034C000DA17C2EB610202EB42027F28A3EB820310
:1034D000E3DCFDF7D7F8E2E7784B029305F042FB17
:1034E000009B1B78002BCED1039B1B78002B3FF455
:1034F000BCAC99F80030A3F10C007F2840F3B681F2
:1035000070488B3B80FB0320DA17C2EB600000EBB6
:103510004000A3EB800303F17300C0B205F022FB6F
:10352000009B1B78002B00F09681654C2378002BC4
:1035300001F04B82DFF89881DFF888A14FF0000B93
:103540000AE003F17300C0B205F00CFB23780BF125
:10355000010B5B457FF789AC58F8043F99F80000F0
:103560001844A0F18B038AFB0321DA17C2EB610236
:103570000C3802EB42027F28A3EB8203E1DCFDF76B
:1035800081F8E0E75046FDF77DF857E4FDF77AF85B
:10359000FFF798BA002008704B49087840B13E49BF
:1035A00000910978002900F0AB81009F002139705B
:1035B0004649097800297FF4FAA8002C40F0CC8015
:1035C000002840F0C9802F4C334F94F800E0344C71
:1035D00003943A4C0294324C30492070374C009797
:1035E000087038702070BEF1000F7FF4F2A8FFF76A
:1035F000F9B82B4B1B78002B6CD099F80030A3F155
:103600000C007F2840F37B832E4A8B3B82FB0321F7
:10361000DA17C2EB610202EB4202A3EB820303F171
:103620007300C0B205F09EFA009B1B78002B51D0AE
:10363000234C2378002B4DD0254FDFF888804FF0A6
:10364000000A09E003F17300C0B205F08BFA237899
:103650000AF1010A53453DDD57F8043F99F800008F
:103660001844A0F18B0388FB0321DA17C2EB610237
:103670000C3802EB42027F28A3EB8203E2DCFDF769
:1036800001F8E1E70A9CFF1F3E9CFF1F949EFF1F6D
:10369000849CFF1F069CFF1F549EFF1F109EFF1F50
:1036A000E59BFF1FC89DFF1FC49DFF1F409CFF1F80
:1036B0007A9EFF1F0B9CFF1F489CFF1FB69CFF1F9D
:1036C0008489FF1FABAAAA2A939EFF1F8F9EFF1F0C
:1036D0005C89FF1F924B1B78FBB1924B1B88012B1F
:1036E00000F03886022B00F03287032B01F0AB800C
:1036F000042B01F05D81052B01F09783062B01F06F
:103700003084072B01F0BC85082B01F07B86092B48
:1037100001F088870A2B01F06587019B1B88002B2D
:1037200000F0BC82804B1B78002B40F0B2827F4BB4
:103730007F4A198834680020012310602B6042E51D
:103740000130C0B2022886BF0021117010701946E6
:1037500002E40398002101707649097800293FF4BA
:1037600041A86F4902910978002900F01687029854
:1037700000210170FFF736B8039B1B78002B7FF404
:103780009CAB029B1B78002B7FF497AB019B1988A5
:10379000FFF799BB243B002BB8F8000040F34784A7
:1037A00098423EF4A0AF9BB26348A8F800300123D2
:1037B0000370FEF798BFDFF88481C0B298F800105C
:1037C00005F0A8F9FFF793BB5C4B3878197805F042
:1037D000A1F9D3E47F21402005F074F95849594AF2
:1037E0003B680B60002111704CE5C0B298F80010E6
:1037F00005F090F9FFF76DB9D8B298F8001005F010
:1038000089F93B68B0E5504BDFF85CE11978FEF7C9
:103810006ABF4B2C40F34A821834802CB8F8003031
:103820004A4AA8BF8024A3427FF41AAEFEF783BFA2
:1038300099F8000005F096F92188FFF744BBFCF7E2
:1038400021FFE2E4424B01931B88002B7FF444AE3E
:10385000334B02934DE6029B1B78002B7FF408ABA1
:10386000039B1B78002B7FF428AB8FE7FCF70AFF44
:1038700053E6FCF707FF1BE5FCF704FFFFF711BA5F
:103880000132D2B2022A40F23D8200220270194671
:10389000FFF762BB2F4C207802F068FC2E4B1B78A0
:1038A0001BB123887E2B41F23B802C4B1B7823B12C
:1038B0002388284A002B41F05880294C3B782370FC
:1038C000FEF724BE254B1B78002BF6D02388214A17
:1038D000002BF2D02349013B088899B211800028BF
:1038E0007FF488ADC8B21E4C05F060F93B782370B8
:1038F000FEF70CBE7F20FFF78BBA7F20FFF7ADB934
:10390000074F094902974FF0000C81F800C0009F53
:1039100002994FF0010E87F800E081F800C047E6F9
:10392000B69CFF1FD29DFF1F109EFF1FB49CFF1F60
:10393000E89BFF1F0A9CFF1F0B9CFF1F959CFF1F0E
:103940000C9CFF1F8489FF1F799EFF1F7A9EFF1F1B
:10395000489CFF1F3E9CFF1F949EFF1F939EFF1FCE
:10396000069CFF1F849CFF1F619CFF1FDFF8B0A314
:103970003868BAF80030E54AE54CC31A82FB031EEA
:10398000D917C1EB6E0101EB4101A3EB810303EBFE
:10399000430354F8233018447F2840F3C9847F3808
:1039A00082FB0032C317C3EB620303EB4303A0EBBC
:1039B00083007330DFF86C83DFF86CB398F8001085
:1039C000C0B205F0A7F8BBF80030022B7FF6D1ABF0
:1039D0003968BAF80030CD4ACB1A82FB030ED817EB
:1039E000C0EB6E0000EB4000A3EB800303EB43034E
:1039F00004EB8303586808447F2840F320877F380E
:103A000082FB0032C317C3EB620202EB4202A0EB5F
:103A100082007330C0B298F8001005F07BF8BBF854
:103A20000030032B7FF6A5AB3968BAF80030B74AEF
:103A3000CB1A82FB030ED817C0EB6E0000EB4000E0
:103A4000A3EB800303EB430304EB8304A068084467
:103A50007F2840F36B817F3882FB0032C317C3EBB2
:103A6000620202EB4202A0EB8200733098F8001071
:103A7000C0B205F04FF8FFF77CBBDFF8A4A299F8BD
:103A80000000BAF80030A14AA14CC31A82FB031E01
:103A9000D917C1EB6E0101EB4101A3EB810303EBED
:103AA000430354F8233018447F2840F33D847F3883
:103AB00082FB0032C317C3EB620303EB4303A0EBAB
:103AC00083007330DFF860B2C0B205F04BF8BBF88A
:103AD0000030022B7FF6ECA999F80010BAF80030FC
:103AE0008A4ACB1A82FB030ED817C0EB6E0000EB9C
:103AF0004000A3EB800303EB430304EB830358680C
:103B000008447F2840F397867F3882FB0032C31732
:103B1000C3EB620202EB4202A0EB82007330C0B240
:103B200005F020F8BBF80030032B7FF6C1A999F807
:103B30000010BAF80030754ACB1A82FB030ED81772
:103B4000C0EB6E0000EB4000A3EB800303EB4303EC
:103B500004EB8304A06808447F2840F3CA807F38C0
:103B600082FB0032C317C3EB620202EB4202A0EBFE
:103B700082007330C0B204F0F5FFFFF799B901205D
:103B8000FFF746B9DFF898A16049BAF80020604C09
:103B90009A1A81FB020ED017C0EB6E0000EB4000BA
:103BA000A2EB800202EB420254F8220018447F2864
:103BB00040F3C283A0F17F0381FB0321DA17C2EB3C
:103BC000610000EB4000A3EB80007330DFF858B1D8
:103BD00098F80010C0B204F09DFFBBF80030022B33
:103BE00050D93968BAF80030484ACB1A82FB030E24
:103BF000D817C0EB6E0000EB4000A3EB800303EB93
:103C0000430304EB8303586808447F2840F37E860F
:103C10007F3882FB0032C317C3EB620202EB420221
:103C2000A0EB82007330C0B298F8001004F072FF6D
:103C3000BBF80030032B25D93868BAF80030334A76
:103C4000C31A82FB031ED917C1EB6E0101EB4101C0
:103C5000A3EB810303EB430304EB8304A368184441
:103C60007F2849DD7F3882FB0032C317C3EB620235
:103C700002EB4202A0EB82007330C0B298F8001051
:103C800004F048FF3B68FFF76ABB04F06BFFFFF7E7
:103C900011B80021402004F015FF48E599F8000014
:103CA00004F060FF3EE50120FEF7D7BF243C002C66
:103CB000B8F8003040F35685A3423EF43CADA4B2C0
:103CC000144BA8F8004001221A70FEF734BD124BC5
:103CD00001931B88002B7FF401ACFFF7C6B80F4996
:103CE0008342A8BF03460B60FEF7D5BE1446FFF71C
:103CF000ACBBFCF7C7FC3DE7FCF7C4FCBDE7FCF739
:103D0000C1FC8EE402701946FFF726B9ABAAAA2AB5
:103D1000641601000B9CFF1F489CFF1FE89BFF1FC0
:103D20000C9EFF1F959CFF1F1E9CFF1FFCF7AAFC0B
:103D30009CE6DFF81CA399F80000BAF80030C24AEC
:103D4000C24CC31A82FB031ED917C1EB6E0101EBF3
:103D50004101A3EB810303EB430354F823301844E0
:103D60007F2840F3C7837F3882FB0032C317C3EB41
:103D7000620303EB4303A0EB83007330DFF8D4B29C
:103D8000C0B204F0EFFEBBF80030022B7FF690A823
:103D900099F80010BAF80030AB4ACB1A82FB030E38
:103DA000D817C0EB6E0000EB4000A3EB800303EBE1
:103DB000430304EB8303586808447F2840F30186DB
:103DC0007F3882FB0032C317C3EB620303EB43036C
:103DD000A0EB83007330C0B204F0C4FEBBF8003027
:103DE000032B7FF665A899F80010BAF80030964AC0
:103DF000CB1A82FB030ED817C0EB6E0000EB40001D
:103E0000A3EB800303EB430304EB8304A0680844A3
:103E10007F287FF76EAF7F3882FB0032C317C3EB7A
:103E2000620303EB4303A0EB83007330A2E6DFF8E9
:103E300020A23868BAF80030834A844CC31A82FB47
:103E4000031ED917C1EB6E0101EB4101A3EB810306
:103E500003EB430354F8233018447F2840F3718365
:103E60007F3882FB0032C317C3EB620303EB4303CB
:103E7000A0EB83007330DFF8E081DFF8D8B198F869
:103E80000010C0B204F046FEBBF80030022B7FF6F3
:103E900070A93968BAF800306B4ACB1A82FB030E5E
:103EA000D817C0EB6E0000EB4000A3EB800303EBE0
:103EB000430304EB8303586808447F2840F3748568
:103EC0007F3882FB0032C317C3EB620303EB43036B
:103ED000A0EB83007330C0B298F8001004F01AFE13
:103EE000BBF80030032B7FF644A93868BAF80030DD
:103EF000554AC31A82FB031ED917C1EB6E0101EBB1
:103F00004101A3EB810303EB430304EB8304A368A8
:103F100018447F287FF70AAF7F3882FB0032C3172F
:103F2000C3EB620303EB4303A0EB830073309DE517
:103F3000DFF81CA14449BAF80020444C9A1A81FBCE
:103F4000020ED017C0EB6E0000EB4000A2EB800227
:103F500002EB420254F8220018447F2840F3F48216
:103F6000A0F17F0381FB0321DA17C2EB610000EBB4
:103F70004000A3EB80007330DFF8D8B098F8001051
:103F8000C0B204F0C7FDBBF80030022B7FF67AAE5A
:103F90003968BAF800302C4ACB1A82FB030ED817C6
:103FA000C0EB6E0000EB4000A3EB800303EB430388
:103FB00004EB8303586808447F2840F3EA847F3881
:103FC00082FB0032C317C3EB620303EB4303A0EB96
:103FD00083007330C0B298F8001004F09BFDBBF86A
:103FE0000030032B7FF64EAE3868BAF80030164A20
:103FF000C31A82FB031ED917C1EB6E0101EB41010D
:10400000A3EB810303EB430304EB8304A36818448D
:104010007F287FF771AE7F3882FB0032C317C3EB76
:10402000620303EB4303A0EB8300733025E6012812
:104030003EF459AB0123FFF7B7BB99F8000004F039
:1040400091FDFFF7A6B800BFABAAAA2A401901004C
:104050000C9EFF1F1E9CFF1F959CFF1FDFF8E8A210
:1040600099F80000BAF80030B54AB64CC31A82FB82
:10407000031ED917C1EB6E0101EB4101A3EB8103D4
:1040800003EB430354F8233018447F2840F3DD81C9
:104090007F3882FB0032C317C3EB620202EB42029D
:1040A000A0EB82007330DFF8A4B2C0B204F05AFD76
:1040B000BBF80030022B7EF6FBAE99F80000BAF890
:1040C00000309F4AC31A82FB0321DA17C2EB610258
:1040D00002EB4202A3EB820303EB430304EB8303F3
:1040E0005B6818447F2840F327847F380C2290FBBC
:1040F000F2F302FB13007330C0B204F033FDBBF8DF
:104100000030032B7EF6D4AE99F80000BAF80030E8
:104110008B4AC31A82FB0321DA17C2EB610202EB5E
:104120004202A3EB820303EB430304EB8304A36883
:1041300018447F287FF7DDAD7F380C2290FBF2F327
:1041400002FB1300733015E5DFF8FCA13868BAF8FC
:1041500000307B4A7B4CC31A82FB031ED917C1EB8C
:104160006E0101EB4101A3EB810303EB430354F820
:10417000233018447F2840F365817F3882FB00326A
:10418000C317C3EB620202EB4202A0EB8200733062
:10419000DFF8BC81DFF8B4B198F80010C0B204F0C9
:1041A000B9FCBBF80030022B7EF6E3AF3868BAF8F2
:1041B0000030634AC31A82FB0321DA17C2EB6102A3
:1041C00002EB4202A3EB820303EB430304EB830302
:1041D0005B6818447F2840F3A0837F380C2290FB53
:1041E000F2F302FB13007330C0B298F8001004F031
:1041F00091FCBBF80030032B7EF6BBAF3868BAF8F1
:1042000000304F4AC31A82FB0321DA17C2EB610266
:1042100002EB4202A3EB820303EB430304EB8304B0
:10422000A36818447F287FF781AD7F380C2290FB6C
:10423000F2F302FB1300733018E4DFF80CA14049DD
:10424000BAF800203F4C9A1A81FB020ED017C0EB3F
:104250006E0000EB4000A2EB800202EB420254F839
:10426000220018447F2840F3F380A0F17F0381FBF4
:104270000321DA17C2EB610101EB4101A3EB8100DD
:104280007330DFF8C8B098F80010C0B204F042FCF8
:10429000BBF80030022B7FF6F5AC3868BAF8003076
:1042A000274AC31A82FB0321DA17C2EB610202EB31
:1042B0004202A3EB820303EB430304EB83035B683B
:1042C00018447F2840F345837F380C2290FBF2F39B
:1042D00002FB13007330C0B298F8001004F01AFC0F
:1042E000BBF80030032B7FF6CDAC3868BAF800304D
:1042F000134AC31A82FB0321DA17C2EB610202EBF5
:104300004202A3EB820303EB430304EB8304A368A1
:1043100018447F287FF7F0AC7F380C2290FBF2F333
:1043200002FB13007330A8E4FCF7ACF9FFF7CABB3B
:10433000FCF7A8F9FFF73EBBFCF7A4F946E400BF81
:10434000ABAAAA2AD01901000C9EFF1F1E9CFF1FBA
:10435000959CFF1FDFF83CA399F80000BAF80030E5
:10436000C44AC54CC31A82FB0317D917C1EB6701B6
:1043700001EB4101A3EB810303EB430354F823302A
:1043800018447F286ADD7F3882FB0032C317C3EBF5
:10439000620202EB4202A0EB82007330DFF8F8B257
:1043A000C0B204F0DFFBBBF80030022B7FF6B5A9EA
:1043B00099F80000BAF80030AE4AC31A82FB032114
:1043C000DA17C2EB610202EB4202A3EB820303EBBA
:1043D000430304EB83035B6818447F2840F3B682F1
:1043E0007F380C2290FBF2F302FB13007330C0B253
:1043F00004F0B8FBBBF80030032B7FF68EA999F8C8
:104400000000BAF800309B4AC31A82FB0321DA1776
:10441000C2EB610202EB4202A3EB820303EB430314
:1044200004EB8304A36818447F2814DD7F380C2232
:1044300090FBF2F302FB13007330C0B204F092FB66
:10444000FFF76BB9FCF71EF9A2E6FCF71BF92AE6A9
:10445000FCF718F915E7FCF715F9EEE7FCF712F988
:104460009CE7DFF830A299F80000BAF80030814AE2
:10447000824CC31A82FB031ED917C1EB6E0101EBFC
:104480004101A3EB810303EB430354F823301844A9
:104490007F28DADD7F3882FB0032C317C3EB62036B
:1044A00003EB4303A0EB83007330FCE5DFF8E4A1EA
:1044B0003868BAF800306F4A704CC31A82FB031E8A
:1044C000D917C1EB6E0101EB4101A3EB810303EBB3
:1044D000430354F8233018447F28B3DD7F3882FB30
:1044E0000032C317C3EB620303EB4303A0EB83006B
:1044F00073304DE6FCF7C6F840E4DFF898A15D495B
:10450000BAF800205D4C9A1A81FB020ED017C0EB5E
:104510006E0000EB4000A2EB800202EB420254F876
:10452000220018447F2893DDA0F17F0381FB032143
:10453000DA17C2EB610000EB4000A3EB80007330A0
:104540009FE6FCF79FF896E4FCF79CF814E5DFF88B
:1045500044A199F80000BAF80030464A484CC31A02
:1045600082FB0317D917C1EB670101EB4101A3EBF4
:10457000810303EB430354F8233018447F287FF76B
:104580006DAF7F3882FB0032C317C3EB620303EBCE
:104590004303A0EB8300733000E73A4800903A48A9
:1045A0003A490390FEF715B9DFF8E8A03868BAF881
:1045B0000030304A364CC31A82FB0321DA17C2EBB3
:1045C000610202EB4202A3EB820303EB430354F8C4
:1045D000233018447F2840F3B6817F380C2290FBAB
:1045E000F2F302FB13007330DFF8B080DFF8A8B0FD
:1045F00098F80010C0B204F08DFABBF80030022B1E
:104600001AD93868BAF800300C22C11A91FBF2F3BB
:1046100002FB131302FB03435B6818447F2840F33B
:1046200067847F3890FBF2F302FB13007330C0B253
:1046300098F8001004F06EFABBF80030032B7EF6F9
:1046400098ADBAF8003038680C22C11A91FBF2F329
:1046500002FB131302FB0344A36818447F287FF76F
:1046600065AB7F3890FBF2F302FB13007330FFF76A
:10467000FDB900BFABAAAA2A64160100541B0100B1
:1046800040190100549EFF1FE59BFF1F109EFF1F56
:10469000001801000C9EFF1F1E9CFF1F959CFF1F12
:1046A000DFF894A399F80000BAF80030D84AD94C42
:1046B000C31A82FB0321DA17C2EB610202EB42024A
:1046C000A3EB820303EB430354F8233018447F2801
:1046D00040F320817F380C2290FBF2F302FB1300A1
:1046E0007330DFF858B3C0B204F03CFABBF80030C6
:1046F000022B19D999F80000BAF800300C22C11A1F
:1047000091FBF2F302FB131302FB03435B681844B3
:104710007F2840F322847F3890FBF2F302FB1300E2
:104720007330C0B204F01EFABBF80030032B7EF6E3
:10473000BFABBAF8003099F800000C22C11A91FB07
:10474000F2F302FB131302FB0344A36818447F280F
:104750007FF7CFAA7F3890FBF2F302FB1300733090
:10476000FFF708BA012B3DF4E6AF0124FFF7A8BA22
:10477000DFF8C4A2A649BAF80020A64C9A1A81FB19
:104780000210D117C1EB600101EB4101A2EB8102E4
:1047900002EB420254F8220018447F2840F3D080F4
:1047A000A0F17F030C2093FBF0F200FB123073307A
:1047B000DFF888B298F80010C0B204F0ABF9BBF88B
:1047C0000030022B1AD93868BAF800300C22C11A0E
:1047D00091FBF2F302FB131302FB03435B681844E3
:1047E0007F2840F382837F3890FBF2F302FB1300B3
:1047F0007330C0B298F8001004F08CF9BBF80030A8
:10480000032B7FF63FAABAF8003038680C22C11A91
:1048100091FBF2F302FB131302FB0344A368184459
:104820007F287FF769AA7F3890FBF2F302FB130021
:104830007330FFF722BAFBF725FFFFF770B9FBF7DC
:1048400021FFFFF7E7B8DFF8F0A199F80000BAF808
:1048500000306F4A704CC31A82FB0321DA17C2EB97
:10486000610202EB4202A3EB820303EB430354F821
:10487000233018447F2846DD7F380C2290FBF2F36A
:1048800002FB13007330DFF8B4B1C0B204F06AF970
:10489000BBF80030022B19D999F80000BAF80030A3
:1048A0000C22C11A91FBF2F302FB131302FB034328
:1048B0005B6818447F2840F3A7807F3890FBF2F3B1
:1048C00002FB13007330C0B204F04CF9BBF80030A7
:1048D000032B7EF622AFBAF8003099F800000C22C4
:1048E000C11A91FBF2F302FB131302FB0344A3680A
:1048F00018447F287FF7AFAD7F3890FBF2F302FBBF
:104900001300733099E5FBF7BDFEBCE7FBF7BAFE79
:10491000FFF789B9FBF7B6FEE3E6FBF7B3FE63E406
:1049200001339BB22380D9B205203C4C04F0CAF875
:104930003B782370FDF7EABDFBF7A4FEFFF7DCBB75
:10494000FBF7A0FE34E7FBF79DFE4DE6FBF79AFE72
:104950004DE5FBF797FEBEE4DFF8DCA099F8000018
:10496000BAF800302A4A2E4CA2E6013B9BB2D9B2DB
:1049700005202A4C138004F0A5F83B782370FDF73E
:10498000C5BDDFF8B4A03868BAF80030204A244C1E
:1049900011E6FBF777FEFFF71DBBDFF89CA01C4973
:1049A000BAF800201E4CE9E6FBF76CFEFFF793BA5D
:1049B000DFF884A099F80000BAF80030144A194CC6
:1049C00049E7FBF75FFEFFF706BA029B1B78002B57
:1049D0007EF44EAAFEF771BA134B1B78002B00F041
:1049E000DE82124B1B78002B7DF4A5AE104B1B789A
:1049F000002B3DF4A0AEB8F800300E490A33A8F8F9
:104A000000300A70FDF797BEFBF73CFE5BE700BF86
:104A1000ABAAAA2A00180100D0190100069CFF1FAA
:104A2000C41A0100541B0100C79DFF1F919EFF1F68
:104A3000929EFF1F0B9CFF1F0C9EFF1F1E9CFF1FC3
:104A4000A14C2388002B40F05483DFF890B29F499B
:104A50009F4A098899F80000B2F800E0DFF87882F0
:104A6000C1EB000C0C229CFBF2F102FB11C14FF0D8
:104A7000900C0CFB0EFE02FB01E16FF00B0E58F8E0
:104A8000011008440EFB03007F2840F3EC84A0F1E2
:104A90007F0393FBF2F002FB10307330C0B204F0DE
:104AA00061F8BBF8002023881344022B22DD874ADB
:104AB000874B118899F80000B3F800C0DFF818E2BE
:104AC000411A0C2291FBF2F302FB1311902303FB1A
:104AD0000CF302FB013373445B6818447F2840F3F6
:104AE00050857F3890FBF2F302FB13007330C0B2A5
:104AF00004F038F8BBF8002023881344032B22DD90
:104B0000724A734B118899F80000B3F800C0DFF8BF
:104B1000C8E1411A0C2291FBF2F302FB131190231E
:104B200003FB0CF302FB013373449B6818447F289A
:104B300040F338857F3890FBF2F302FB13007330AB
:104B4000C0B204F00FF8BBF8002023881344042BF4
:104B50007EF7AEA95F4B1B88012B7EF4A9A999F8BB
:104B60000020A2F10C007F287FF7C3A88B3A0C200D
:104B700092FBF0F300FB13207330FEF7FBBF524CA7
:104B80002288002A00F018835249DFF850B10988C2
:104B9000BBF800000331884227DD4C484C490088AF
:104BA000B1F800E0DFF830C1181A0C2190FBF1F9E0
:104BB00001FB19004FF0900909FB0EFE01FB00E01C
:104BC0006FF00B0E5CF8000003440EFB02307F28F0
:104BD00040F311847F3890FBF1F301FB1300733035
:104BE000C0B298F8001003F095FFBBF800202388AE
:104BF0001344022B23DD354B354A38681B88B2F845
:104C000000C0DFF8D4E0C31A0C2193FBF1F201FBE2
:104C10001232902303FB0CF301FB023373445B68F5
:104C200018447F2840F3A5847F3890FBF1F301FB03
:104C300013007330C0B298F8001003F06BFFBBF89C
:104C4000002023881344032B23DD204B204A38689F
:104C50001B88B2F800C0DFF880E0C31A0C2193FB78
:104C6000F1F201FB1232902303FB0CF301FB023340
:104C700073449B6818447F2840F37F847F3890FBFF
:104C8000F1F301FB13007330C0B298F8001003F089
:104C900041FFBBF8002023881344042B7EF7F2AFBA
:104CA0000C4B1B88012B7EF4EDAF3A68A2F10C008F
:104CB0007F287FF721A88B3A0C2092FBF0F300FBB2
:104CC00013207330FEF7D9BF989CFF1F0C9EFF1F67
:104CD000BA9DFF1F3C9CFF1F601301001E9CFF1F1D
:104CE000B84C2388002B40F06A82DFF810B3B64935
:104CF000B64A0988D7F80080B2F800E0B448C1EBA2
:104D0000080C0C229CFBF2F102FB11C14FF0900C3D
:104D10000CFB0EFE02FB01E16FF00B0E40588044CD
:104D20000EFB03807F2840F36A83A0F17F0393FB8F
:104D3000F2F002FB10307330A64BC0B2197803F0CA
:104D4000E9FEBBF8002023881344022B23DD9E4A92
:104D50009E4B11883868B3F800C0DFF874E2411A3E
:104D60000C2291FBF2F302FB1311902303FB0CF3D3
:104D700002FB013373445B6818447F2840F30B84C3
:104D80007F3890FBF2F302FB13007330914BC0B2FB
:104D9000197803F0BFFEBBF8002023881344032BCF
:104DA00023DD894A894B11883868B3F800C0DFF8E1
:104DB00020E2411A0C2291FBF2F302FB1311902323
:104DC00003FB0CF302FB013373449B6818447F28F8
:104DD00040F3DE837F3890FBF2F302FB1300733065
:104DE0007C4BC0B2197803F095FEBBF800202388F5
:104DF0001344042B7EF7BDA9774B1B88012B7EF44F
:104E0000B8A93A68A2F10C007F2840F3B2808B3A2F
:104E10000C2092FBF0F300FB132073306D4BC0B2FB
:104E2000197803F077FEFEF7A4B9DFF89CA199F892
:104E30000000BAF80030694CC11A0C2291FBF2F361
:104E400002FB131302FB03F3E35818447F287FF798
:104E50005AAD7F3890FBF2F302FB1300733012E57A
:104E60005F4B1A88182A13D03B681344A3F118002B
:104E70007F2840F37B830C20973B93FBF0F200FBF1
:104E8000123303F17300534BC0B2197803F042FEA2
:104E9000544B55491A78022A94BF013200221A70E5
:104EA0001A7831F81200182810D10424022A02F1CD
:104EB0000100C2B288BF002231F81200182804D1C4
:104EC000013CF3D11A70FEF754B91A703B680344E1
:104ED000A3F118007F284CDD0C20973B93FBF0F2E8
:104EE00000FB123303F1730098E7FBF7CBFB80E480
:104EF000FBF7C8FBFFF79BBB394B1B88182B12D065
:104F000099F800201344A3F118007F2840F33D8353
:104F10000C20973B93FBF0F200FB123303F173007C
:104F2000C0B203F01FFE2F4A2F4B127833F8123015
:104F3000182B3DF4BDAF99F800201344A3F11800DD
:104F40007F287EF7D6AE0C20973B93FBF0F200FB58
:104F5000123303F17300FEF70DBEFBF793FBFFF76F
:104F6000E0BBDFF864A099F80000BAF800301F4CED
:104F700062E7FBF787FB51E71D4B1B78002B7DF4A5
:104F8000DAAB1C4B1B78002B3DF4D5ABB8F80030E6
:104F90001949013BA8F800300A70FDF7CCBB144B4F
:104FA0001B78002B7EF401A8124B1B78002B3DF4DC
:104FB000C2ABB8F8003010490133A8F800300A70CD
:104FC000FDF7B9BB989CFF1F0C9EFF1FBA9DFF1FEA
:104FD00060130100959CFF1F3C9CFF1F00180100FF
:104FE0002A9CFF1F969CFF1F249EFF1FC41A0100CE
:104FF000919EFF1F929EFF1F0B9CFF1F1E9CFF1F79
:10500000944A1288182A12D01344A3F118007F285A
:1050100040F3CC820C20973B93FBF0F200FB123361
:1050200003F17300C0B298F8001003F073FD8A4BCF
:105030008A491A78022A94BF013200221A701A781B
:1050400031F81200182811D10424022A02F10100BB
:10505000C2B288BF002231F81200182805D1013CE5
:10506000F3D11A703B68FEF77AB91A703B680344B3
:10507000A3F118007F287EF73FAE0C20973B93FBEF
:10508000F0F200FB123303F17300FEF7F6BD744A31
:105090001288182A12D01344A3F118007F2840F375
:1050A0007E820C20973B93FBF0F200FB123303F15E
:1050B0007300C0B298F8001003F02CFD664B6949EC
:1050C0001A78022A94BF013200221A701A7831F835
:1050D00012001828CAD10424022A02F1010294BF46
:1050E000D2B2002231F812001828BED1013CF3D10F
:1050F000B7E75D4ADFF884B11288BBF800100332CD
:1051000091427FF7CEACA2E4554B1B88182B12D0EE
:1051100099F800201344A3F118007F2840F323825C
:105120000C20973B93FBF0F200FB123303F173006A
:10513000C0B203F017FD484A4A4B127833F81230D8
:10514000182B7FF4F8AEFDF7B3BE454B1A88182A2A
:1051500013D03B681344A3F118007F2840F3F28179
:105160000C20973B93FBF0F200FB123303F173002A
:105170003E4BC0B2197803F0CDFC374B39491A7851
:10518000022A94BF013200221A701A7831F81200F4
:1051900018287FF49BAE0424022A02F1010294BF76
:1051A000D2B2002231F8120018287FF48EAE013CF2
:1051B000F2D11A70FDF7DDBFDFF8C0B0EDE42A4A86
:1051C000DFF8B8B01288BBF80010033291427FF7C5
:1051D000B8AD8CE5264B01227F2107201A8003F011
:1051E00071FC7F210B2003F06DFCFDF709BF214B03
:1051F00004227F2107201A8003F064FC00210B2089
:1052000003F060FCFDF7F5BE1A4B02227F21072058
:105210001A8003F057FC7F210B2003F053FCFDF7AD
:10522000E3BE144B002107201C8003F04BFC7F21C0
:105230000B2003F047FCFDF7D2BE0F4B00227F216D
:1052400007201A8003F03EFC7F210B2003F03AFC7C
:10525000FDF7DEBE2A9CFF1F969CFF1F249EFF1FAA
:10526000329CFF1F9C9DFF1F3C9CFF1F959CFF1FB6
:10527000A69CFF1F049EFF1F089CFF1F1E9CFF1F74
:10528000CC4C2388002B40F06381DFF854B3CA492B
:1052900099F80000C94A09881788DFF824E3411A01
:1052A0000C2291FBF2FC02FB1C114FF0900C0CFB4A
:1052B00007F702FB01716FF00B075EF80110014464
:1052C00007FB03107F2840F340817F3890FBF2F307
:1052D00002FB13007330C0B203F044FCBBF80020A3
:1052E00023881344022B21DDB34BB44A99F8000004
:1052F0001B88B2F800E0B24FC31A0C2193FBF1F205
:1053000001FB1232902303FB0EF301FB02333B44FB
:105310005B6818447F2840F3B1817F3890FBF1F33C
:1053200001FB13007330C0B203F01CFCBBF800207B
:1053300023881344032B21DD9F4BA04A99F80000DA
:105340001B88B2F800E09E4FC31A0C2193FBF1F2C8
:1053500001FB1232902303FB0EF301FB02333B44AB
:105360009B6818447F2840F386817F3890FBF1F3D7
:1053700001FB13007330C0B203F0F4FBBBF8002054
:1053800023881344042B7EF7C8A98E4B1B88012B5E
:105390007EF4C3A999F80020A2F10C007F287FF7C2
:1053A0005AA88B3A0C2092FBF0F300FB13207330C9
:1053B000FFF743B8844B1B88182B12D099F80020B4
:1053C0001344A3F118007F2840F35B810C20973B26
:1053D00093FBF0F200FB123303F17300C0B203F051
:1053E000C1FB7A4A7A4B127833F81230182B7FF4CB
:1053F000A2ADFDF75DBDFBF745F9FFF7F1BBFBF78C
:1054000041F999E4734B1B88182B12D099F80020AE
:105410001344A3F118007F2840F339810C20973BF7
:1054200093FBF0F200FB123303F17300C0B203F000
:1054300099FB664A684B127833F81230182B3EF409
:105440006CA999F800201344A3F118007F287FF776
:1054500002A80C20973B93FBF0F200FB123303F100
:105460007300FEF7EABFFBF70DF9FFF717BB564ACB
:105470001288182A12D01344A3F118007F2840F391
:1054800003810C20973B93FBF0F200FB123303F1F6
:105490007300C0B298F8001003F03CFB4B4B4C4932
:1054A0001A78022A94BF013200221A701A7831F851
:1054B000120018287FF4DAAD0424022A02F1010256
:1054C00094BFD2B2002231F8120018287FF4CDAD7B
:1054D000013CF2D1C5E53C4B1A88182A13D03B6831
:1054E0001344A3F118007F2840F3C2800C20973B9F
:1054F00093FBF0F200FB123303F17300374BC0B2A1
:10550000197803F007FB314B31491A78022A94BF0E
:10551000013200221A701A7831F8120018287FF42C
:10552000D5AC0424022A02F1010294BFD2B20022B7
:1055300031F8120018287FF4C8AC013CF2D11A707F
:10554000FDF717BEFBF79EF812E6FBF79BF8C2E6E5
:105550001C4ADFF88CB01288BBF80010033291426D
:105560007FF7BCAE93E6FBF78DF8E1E5FBF78AF831
:1055700089E4FBF787F8FFF75DBBFBF783F8FFF7DC
:1055800083BBFBF77FF8FFF7B2BAFBF77BF8C7E402
:10559000FBF778F824E4FBF775F8FFF7F7BBFBF7A8
:1055A00071F886E5FBF76EF8FFF7CABAFBF76AF801
:1055B00038E500BF989CFF1F0C9EFF1FBA9DFF1F80
:1055C000601301003C9CFF1F349CFF1F969CFF1F33
:1055D000A49DFF1F2A9CFF1F249EFF1F959CFF1F59
:1055E0001E9CFF1F304B1B88182B11D099F80020F0
:1055F0001344A3F118007F2834DD0C20973B93FB64
:10560000F0F200FB123303F17300C0B203F0AAFA08
:10561000264A274B127833F81230182B7FF411AF3B
:10562000FEF77BB8234B1B88182B11D099F800206C
:105630001344A3F118007F2817DD0C20973B93FB40
:10564000F0F200FB123303F17300C0B203F08AFAE8
:10565000164A194B127833F81230182B7FF4F1AE3A
:10566000FEF75BB8FBF70EF8CFE7FBF70BF8ECE7BC
:10567000FBF708F842E7FBF705F87CE6FBF702F8D2
:1056800051E6FAF7FFFFA9E6FAF7FCFF01E7FAF7A0
:10569000F9FFCBE6094B0393094B0293FDF71EBFBD
:1056A00023601946FDF758BC349CFF1F969CFF1FD2
:1056B000A49DFF1F329CFF1F9C9DFF1FE59BFF1FAA
:1056C000B69CFF1F38B507F015F90E4805F04CF8E9
:1056D0000D4805F049F80D4805F046F800234FF055
:1056E0007E5201210A48FAF7C1FE0A4B0A4A0B49C9
:1056F000802400251C7118461D60BDE838400AF062
:10570000BDBD00BF1C9CFF1F509CFF1FAC9CFF1F1A
:10571000E09DFF1F5C9EFF1F1C89FF1F29060000E4
:1057200043682A20198803F051BB00BF10B5044616
:1057300022206368198803F049FBE3682420198854
:10574000BDE8104003F042BB10B504460A20636870
:10575000198803F03BFBE3680C201988BDE8104072
:1057600003F034BB10B5044606206368198803F0C3
:105770002DFBE36808201988BDE8104003F026BB24
:1057800010B5044602206368198803F01FFBE36824
:1057900004201988BDE8104003F018BB70B50E4C0A
:1057A00084B012250422012306460390029320466A
:1057B0008DE824001423102106F0DAF906220923CB
:1057C000029303960195204600921423102106F0BF
:1057D000CFF904B070BD00BFC09EFF1F2DE9F0419E
:1057E000224D82B0012602B284B200922846019670
:1057F0007823192106F002F904F10C0212B28DE8A7
:1058000044002846A7197823192104F1020806F05C
:10581000F5F83FB20FFA88F819233A462846194698
:105820000196CDF8008006F0E9F878233A4628463C
:105830001946CDF80080019604F10A070B3406F0F2
:10584000DDF83FB224B278233A46284619468DE85F
:10585000500006F0D3F8192300943A4601962846E2
:10586000194606F0CBF802B0BDE8F081C09EFF1FDC
:105870002DE9F0411E4682B01446002A6AD0099BE9
:105880004D4A00EBC305012C6F8929896868A7EB95
:10589000010382FB03E21A444FEAE373C3EBA21352
:1058A00002887BD0042C38D112FA83F3994203DCAE
:1058B0009F423946A8BF1946089A0180B6F90030C0
:1058C000BDF920803D48971D4FF0000E3FB21946AC
:1058D00042460097CDF804E006F090F829896A89DD
:1058E0006B68521A1B885C2AA3EB010359DD03EB9A
:1058F00043030132C3EB431393FBF2F303F11B02A7
:1059000013B20120328019464246019000972B487D
:1059100006F074F82A4B00221A702A4B022CB3F9B5
:10592000001045D0082C31D100221A8091422DD090
:10593000089AB6F9003021480632012412B20092CA
:1059400019460194BDF9202006F058F8204602B00F
:10595000BDE8F0811C4D1D4A2B681268CB1A93429A
:105960000F4617D9164A338811781448012918BFF1
:1059700001241470089A06321BB212B28DE814008A
:105980001946BDF9202006F039F82F60012002B039
:10599000BDE8F081204602B0BDE8F0819BB2D31A89
:1059A00084E75C2101FB03F393FBF2F21B32A7E7D0
:1059B0004A1C12B21A80B9E7C94216B2C09EFF1F34
:1059C000399FFF1FA29EFF1F249FFF1F7C2B0100FA
:1059D00030B583B000230C4605B2009326225B232A
:1059E0001C210C4805F05AFD2946012326220948AE
:1059F00005F064F8002C24B205DB214601232622A1
:105A0000044805F05BF8044A044B15801C8003B081
:105A100030BD00BFC09EFF1F668AFF1F688AFF1F40
:105A20002DE9F041AA4C237882B01BB1A94B4FF667
:105A3000FF721A80A84BB3F90030CBB9A74AA54B27
:105A40001068B3F9002080F30C005B2303FB00F027
:105A500000131C30824269D04FF0FF31FFF7B8FFCE
:105A60009F4805F07FFD0023237002B0BDE8F08160
:105A7000012B40D0022B78D0032B5DD0042BF2D128
:105A8000252200258DE8240076231C219448954E7C
:105A9000954FDFF8888205F0B1FF17E0B0F5AF7FD2
:105AA000A8BF4FF4AF70323802FB00F088FB003122
:105AB000C017C0EB61111C3109B201231D4425221E
:105AC000874804F0FBFF0C2D00F08C80E9B287487A
:105AD00004F0B2FE56F8043BC3F5967300FB03F0E6
:105AE00087FB0013C017C0EB631031284FF05B0237
:105AF000D4DC1C21E1E77E4B1A68B2F52F7F32DB44
:105B000041F25C239342A8BF1346A3F52F735B2297
:105B1000784802FB03F380FB0320DB17C3EBA020D4
:105B20001C306C4BB3F90030834295D1724BB3F902
:105B30000030013390D196E7704B1B68B3F5FA7FC4
:105B400011DBB3F57A6FA8BF4FF47A63A3F5FA724D
:105B50006B485B2303FB02F380FB0320DB17C3EBE3
:105B600020201C30DDE71C20DBE7664B1B68B3F50B
:105B7000FA7F33DBB3F57A6FA8BF4FF47A63A3F5EE
:105B8000FA725F485B2303FB02F380FB0320DB1701
:105B9000C3EB20201C305C4B1B68B3F5FA7F1FDB86
:105BA000B3F57A6FA8BF4FF47A63A3F5FA7254493C
:105BB0005B2303FB02F381FB0321DB17C3EB2121F2
:105BC0001C31444BB3F9003083427FF447AF4A4B5A
:105BD000B3F900308B427FF441AF44E71C20DAE791
:105BE0001C21EEE7262200258DE8240076231C21C7
:105BF0003B48464E3C4FDFF8248105F0FFFE16E09F
:105C0000B0F5AF7FA8BF4FF4AF70323802FB00F0A1
:105C100088FB0031C017C0EB61111C3109B20123B0
:105C20001D4426222E4804F049FF0C2D14D0E9B261
:105C3000374804F001FE56F8043BC3F5967300FBA9
:105C400003F087FB0013C017C0EB631031284FF03F
:105C50005B02D5DC1C21E2E7272200258DE8240029
:105C600076231C211E482B4E1F4FDFF8B08005F015
:105C7000C5FE17E0B0F5AF7FA8BF4FF4AF70323864
:105C800002FB00F088FB0031C017C0EB61111C3132
:105C900009B201231D442722114804F00FFF062DED
:105CA0003FF4DEAEE9B21C4804F0C6FD56F8043BF2
:105CB000C3F5967300FB03F087FB0013C017C0EB1E
:105CC000631031284FF05B02D4DC1C21E1E700BFF8
:105CD000989EFF1F668AFF1F9E9EFF1F189EFF1F34
:105CE000C09EFF1F1C8AFF1FB5814E1B509CFF1FCB
:105CF000F89BFF1FD3058541688AFF1F409CFF1F4B
:105D0000011FB8124C9CFF1F889EFF1F2C89FF1F8C
:105D1000AC9CFF1F4C8AFF1F1C9CFF1F4B48371B6E
:105D20002DE9F04FDFF8EC82B74CB8F900604D7800
:105D300054F8264087B08246039305B10D78DFF80A
:105D4000FCB2002A34D19BF800308BBBAF4EB6F9C1
:105D50000000002800F0CE80012800F024810120FE
:105D600032232A46019000935146A94B2046FFF763
:105D70007FFD00250746B6F90030022B40F3F48082
:105D800000233380B8F90030A24A002BC0F2F8801B
:105D9000042BC4BF00231380039B002B40F0F6802C
:105DA000002D0CBF38464FF0FF3007B0BDE8F08F34
:105DB000964EE3682268984804930027059237803E
:105DC0008BF8007005F0C2FA1120FFF707FD4FF0C5
:105DD000010919232821CDF80490009124221946A5
:105DE0008D4805F00BFE782328212422CDF804905D
:105DF00000918948194605F001FE4946864806F09B
:105E000093F902221921844806F08AF9DDF81490EA
:105E100048460AF0F5FF494602467F4806F01AFB5D
:105E20007D4806F02DFB394614227B4806F078F9B0
:105E300003227A49784806F00DFB774806F020FBEC
:105E400039462322744806F06BF9032274497248DC
:105E500006F000FB704806F013FB049B002B72D188
:105E60000123704A18461370FFF798FC2089638954
:105E70006768191A5C293A885BDC131A5C2202FBFA
:105E800003F292FBF1F31B33674A63481380012747
:105E90001BB21A2219468DE88400142205F0AEFDCB
:105EA000049BDBB1218A638AE768581A5C283A8828
:105EB0006FDD521A02EB4202C2EB4212431C92FB0C
:105EC000F3F31B33524A54481380012738221BB284
:105ED0008DE884001946322205F090FD534A544B58
:105EE000B6F90000012111704FF6FF721A800028E8
:105EF0007FF432AFDFF848914E4AD9F8003012688B
:105F0000C3EB0A0393424CD9464B1A78012A18BFB7
:105F1000012018700127FFF741FCC9F800A0012DEE
:105F20004ED0042D59D0022D60D0082D64D000250C
:105F300021E7121A02EB4202C2EB42124B1C92FB07
:105F4000F3F31B33A0E72F20FFF748FC394632223A
:105F5000314806F0E5F8032237492F4806F07AFA6F
:105F60002D4806F08DFA7BE77FF40CAFE368002B39
:105F70003FF406AFB8F90030264A002BBFF608AF51
:105F800004231380039B002B3FF40AAFFFF748FD67
:105F900006E7511A5C2202FB01F292FBF0F31B337D
:105FA00090E70746BBE7002714238DE888002A46C0
:105FB00051461D4B2046FFF75BFC3D460746DAE69F
:105FC000B8F800308BF800500133A8F8003063694E
:105FD00083B1002520469847CDE6B8F8003001226D
:105FE000013BA8F800308BF80020F0E70123338054
:105FF0000025C7E61D46BEE66369002232804FF0E9
:10600000FF35002BE6D1BDE66C8AFF1FA29EFF1F65
:106010009C9EFF1F9E9EFF1FC09EFF1FA41C010091
:10602000A81C0100399FFF1F9A9EFF1F989EFF1F0B
:10603000668AFF1F7C2B0100AC1C0100A09EFF1F85
:10604000249FFF1F01210D2007F0CEB800210D2055
:1060500007F0CAB801460D2007F0C6B808B50D20F4
:1060600007F0C8F8B0FA80F149090D20BDE80840F2
:1060700007F0BAB810B5002144080D2007F0B4F8B5
:10608000204607F0EDF80D20012107F0ADF820467D
:10609000BDE8104007F0E4B82D4A2E4B10881B686D
:1060A000984210B549DA2C4A1288141A9A42A8BFAD
:1060B0001A46B4F5157F36DA121A40F2532303FB61
:1060C00002F393FBF4F105310A2006F0FDFE234BA9
:1060D0001978C9B3224B23491B6840F2271283F376
:1060E000070302FB03F381FB03211944DB17C3EB16
:1060F000A1110531092006F0E7FE1B4B1968F1B12B
:1061000081F3070140F22712164802FB01F380FBDE
:1061100003211944DB17C3EBA11105311620BDE89B
:10612000104006F0D1BE131A4FF41572611C02FB29
:1061300003F393FBF1F10531C6E70021C4E7162014
:10614000BDE8104006F0C0BE092006F0BDFED4E751
:10615000B49CFF1FE89BFF1F6A9EFF1F6E9CFF1FE2
:10616000EC9BFF1F090402812C9EFF1F7F2838B57E
:10617000A8BF7F200F4C4FF4167202FB00F284FB85
:1061800002311144D2170546C2EBA1110A2006F0D4
:106190009BFE7F3D4FF4967303FB05F384FB0321C5
:1061A0001944DB17A3EBA1110920BDE8384006F024
:1061B0008BBE00BF09040281C368B3F9003030B55B
:1061C00083EAE374A4EBE374002BA0B218DB012391
:1061D00000E0134603EB830252009442F9DA0A4DC1
:1061E00090FBF3F285FB03E403FB1200DB17303274
:1061F000D3EBA40380B201F8012BF1D10B7030BDB9
:106200002D230B700131E2E76766666638B5094DEC
:106210008224204602F0F4FD35F8021B00B28842C9
:10622000204601D002F0D2FD0234A4B28A2CF0D173
:1062300038BD00BFA49DFF1F024B8020198802F0CB
:10624000C5BD00BF349CFF1F38B5094D78242046DA
:1062500002F0D6FD35F8021B00B28842204601D07C
:1062600002F0B4FD0234A4B2802CF0D138BD00BFDE
:106270009C9DFF1F024B7620198802F0A7BD00BF2E
:10628000329CFF1F38B5094D4624204602F0B8FD68
:1062900035F8021B00B28842204601D002F096FD7C
:1062A0000234A4B24E2CF0D138BD00BF249EFF1F93
:1062B000024B4420198802F089BD00BF2A9CFF1FB1
:1062C000024B4E20198802F081BD00BF489CFF1F81
:1062D000024B9A20198802F079BD00BF989CFF1FDD
:1062E000024B9820198802F071BD00BF3C9CFF1F33
:1062F000024B8C20198802F069BD00BFBA9DFF1FB8
:10630000024B9C20198802F061BD00BF1E9CFF1F3C
:10631000024BA020198802F059BD00BF8C9EFF1FC0
:10632000024B9620198802F051BD00BF0C9EFF1F42
:10633000024B8A20198802F049BD00BFD29DFF1F81
:1063400008B5034B1020198802F040FD012008BD5C
:10635000D09DFF1F024B1020198802F037BD00BFEF
:10636000D09DFF1F024B2C20198802F02FBD00BFCB
:10637000189CFF1F024B1E20198802F027BD00BF8A
:10638000149CFF1FC3680E20198802F01FBD00BFB8
:10639000024B2820198802F019BD00BF209EFF1F64
:1063A000024B6420198802F011BD00BF1C9EFF1F24
:1063B000024B5A20198802F009BD00BF009CFF1F44
:1063C000024B1620198802F001BD00BF089CFF1F78
:1063D000024B2E20198802F0F9BC00BFA09CFF1FC1
:1063E000024B3020198802F0F1BC00BFF49BFF1F64
:1063F000024B9E20198802F0E9BC00BFC089FF1F34
:10640000024B1820198802F0E1BC00BFB89CFF1FA6
:10641000024B1A20198802F0D9BC00BF529CFF1F02
:10642000024B1C20198802F0D1BC00BF4A9CFF1F00
:10643000024B6620198802F0C9BC00BF529EFF1FA4
:10644000024B7220198802F0C1BC00BF709EFF1F72
:10645000024B2020198802F0B9BC00BF509EFF1FDC
:10646000024B3220198802F0B1BC00BF469EFF1FCC
:10647000024B6820198802F0A9BC00BF849CFF1F52
:10648000024B6C20198802F0A1BC00BFF09BFF1FDB
:10649000024B6E20198802F099BC00BF969EFF1F28
:1064A000024B5220198802F091BC00BF5E89FF1F89
:1064B000024B5020198802F089BC00BF148AFF1FCC
:1064C000024B5420198802F081BC00BF168AFF1FBE
:1064D000024B5C20198802F079BC00BF648AFF1F60
:1064E000024B5E20198802F071BC00BF5C89FF1F5F
:1064F000024B6020198802F069BC00BFC09DFF1FDD
:10650000024B5620198802F061BC00BF929CFF1F0D
:10651000244B1B880B2B43D8DFE803F00B10151A14
:106520001F24292E33383D06084604221E490AF04E
:1065300025BD084604221D490AF020BD0846042254
:106540001B490AF01BBD084604221A490AF016BD71
:106550000846042218490AF011BD084604221749CA
:106560000AF00CBD0846042215490AF007BD08468A
:10657000042214490AF002BD0846042212490AF016
:10658000FDBC0846042211490AF0F8BC0846042262
:106590000F490AF0F3BC084604220E490AF0EEBC8B
:1065A000704700BF0C9EFF1F5428010028260100E1
:1065B000DC240100C4250100E02401006029010061
:1065C000E4240100E824010060270100EC2401001C
:1065D00060280100F0240100064B074A10B41C8813
:1065E000064B0846002C14BF11461946042210BC65
:1065F0000AF0C4BC689CFF1FF4240100F8240100C9
:10660000064B074A10B41C88064B0846002C14BFE2
:1066100011461946042210BC0AF0B0BCA29CFF1F10
:10662000F4240100F8240100064B074A10B41C882A
:10663000064B0846002C14BF11461946042210BC14
:106640000AF09CBCC29DFF1FF4240100F824010045
:10665000064B074A10B41C88064B0846002C14BF92
:1066600011461946042210BC0AF088BC0E9EFF1F7A
:10667000F4240100F8240100064B074A10B41C88DA
:10668000064B0846002C14BF11461946042210BCC4
:106690000AF074BCA69CFF1FF4240100F82401003A
:1066A0001B4B1B880A2B0AD8DFE803F00A0E1216D0
:1066B0001A1E22262A2E0600164B186808607047FC
:1066C000154B186808607047144B186808607047CD
:1066D000134B186808607047124B186808607047C1
:1066E000114B186808607047104B186808607047B5
:1066F0000F4B1868086070470E4B186808607047A9
:106700000D4B1868086070470C4B1868086070479C
:10671000D29DFF1F20250100F8240100FC24010068
:106720000025010004250100082501000C250100B9
:106730001025010014250100182501001C25010069
:10674000F0B52B4E2B4FDFF8C4E005460FCE87B0D7
:106750006C460FC496E803003B68274A274F44F86D
:10676000040B40F6CC308342C8BF3A46BEF8006006
:106770002180012E11889278ADF80D108DF80F2030
:106780002AD032D340F6CA02022E18BF00229A4203
:1067900026DCA3F698031A491A4AC3EB031381FBBC
:1067A00003011944DB17C3EB6123243382FB03216C
:1067B000DA17C2EBA10202EB8201A3EB41033033F3
:1067C00030328DF813308DF8112069462846162294
:1067D0000AF0D4FB07B0F0BD40F698029A42D8DD2B
:1067E000094B1868CDF81100EFE740F6FC02CEE740
:1067F00034250100309EFF1F2825010024250100BB
:106800003B773B98676666662C250100AC9DFF1FB1
:10681000F8B5174C174E2278174D33782F888E46CF
:10682000003218BF012201467046FFF779FA0023B3
:1068300098423370237015DB14BF012000202B8891
:106840009F420ED040F23A72A3F5AF730B490C4C45
:1068500002FB03F381FB0312DB17A3EB621332335A
:106860002360F8BD0749012218460A702270E6E746
:10687000108BFF1FB19EFF1F649EFF1FB5814E1B33
:10688000048AFF1F389FFF1F014B187802F036BAA9
:10689000209FFF1F014B187802F04ABAB490FF1FE7
:1068A000134BB3F9003030B583EAE374A4EBE3741F
:1068B000002BA0B218DB012300E0134603EB830298
:1068C00052009442F9DA0B4D90FBF3F285FB03E49E
:1068D00003FB1200DB173032D3EBA40380B201F8C4
:1068E000012BF1D10B7030BD2D230B700131E2E78C
:1068F000B490FF1F67666666144BB3F9003070B53D
:1069000083EAE375A5EBE375002BACB21ADB012338
:1069100000E0034603EB830040008542F9DA0C4EA9
:1069200094FBF3F086FB03E503FB1044DB173030E8
:10693000D3EBA503A4B201F8010BF1D105480B700C
:10694000106070BD2D230B700131E0E7009CFF1F2C
:10695000676666664C250100134BB3F9003030B50D
:1069600083EAE374A4EBE374002BA0B218DB0123E9
:1069700000E0134603EB830252009442F9DA0B4D18
:1069800090FBF3F285FB03E403FB1200DB173032CC
:10699000D3EBA40380B201F8012BF1D10B7030BD11
:1069A0002D230B700131E2E7C089FF1F6766666621
:1069B000134BB3F9003030B583EAE374A4EBE3740E
:1069C000002BA0B218DB012300E0134603EB830287
:1069D00052009442F9DA0B4D90FBF3F285FB03E48D
:1069E00003FB1200DB173032D3EBA40380B201F8B3
:1069F000012BF1D10B7030BD2D230B700131E2E77B
:106A00005E89FF1F67666666134BB3F9003030B5C9
:106A100083EAE374A4EBE374002BA0B218DB012338
:106A200000E0134603EB830252009442F9DA0B4D67
:106A300090FBF3F285FB03E403FB1200DB1730321B
:106A4000D3EBA40380B201F8012BF1D10B7030BD60
:106A50002D230B700131E2E7148AFF1F676666661B
:106A6000134BB3F9003030B583EAE374A4EBE3745D
:106A7000002BA0B218DB012300E0134603EB8302D6
:106A800052009442F9DA0B4D90FBF3F285FB03E4DC
:106A900003FB1200DB173032D3EBA40380B201F802
:106AA000012BF1D10B7030BD2D230B700131E2E7CA
:106AB000168AFF1F67666666134BB3F9003030B560
:106AC00083EAE374A4EBE374002BA0B218DB012388
:106AD00000E0134603EB830252009442F9DA0B4DB7
:106AE00090FBF3F285FB03E403FB1200DB1730326B
:106AF000D3EBA40380B201F8012BF1D10B7030BDB0
:106B00002D230B700131E2E7648AFF1F676666661A
:106B1000134BB3F9003030B583EAE374A4EBE374AC
:106B2000002BA0B218DB012300E0134603EB830225
:106B300052009442F9DA0B4D90FBF3F285FB03E42B
:106B400003FB1200DB173032D3EBA40380B201F851
:106B5000012BF1D10B7030BD2D230B700131E2E719
:106B60005C89FF1F6766666608B5702002F048F909
:106B7000044B1988884204D07020BDE8084002F018
:106B800025B908BDAC9DFF1F08B5742002F038F987
:106B9000044B1988884204D07420BDE8084002F0F4
:106BA00015B908BD3C9EFF1F054B1B8808460422F3
:106BB00013B904490AF0E2B903490AF0DFB900BF8A
:106BC000489CFF1F54250100502501000E4B1B88D7
:106BD000032B17D8DFE803F0110C07020846042244
:106BE0000A490AF0CBB90846042209490AF0C6B995
:106BF0000846042207490AF0C1B90846042206499A
:106C00000AF0BCB9704700BFBA9DFF1F64250100A0
:106C1000602501005C2501005825010010B40A4BD5
:106C20000A4C0A4693E8030083B0238802AC04E9C7
:106C3000030004EB8303104653F8081C052203B03D
:106C400010BC0AF09BB900BF341D01001C9EFF1F41
:106C500030B40A4B0A4D0C4693E8070084B02B88E9
:106C600004AD05E9070005EB8303204653F80C1C2F
:106C7000042204B030BC0AF081B900BF3C1D010001
:106C8000AC9DFF1FF0B40C4D0C4F0E460FCD8CB0D9
:106C900001AC0FC40FCD0FC495E807003B8884E812
:106CA00007000CAA02EB8303304653F82C1C042285
:106CB0000CB0F0BC0AF062B9481D0100049EFF1F31
:106CC000F0B40A4D0A4F0E460FCD86B001AC0FC48A
:106CD0002A683B88226006AA02EB8303304653F8F9
:106CE000141C042206B0F0BC0AF048B9741D01005F
:106CF000B89CFF1FF0B40A4D0A4F0E460FCD86B068
:106D000001AC0FC42A683B88226006AA02EB830309
:106D1000304653F8141C0C2206B0F0BC0AF02EB911
:106D2000881D01004A9CFF1FF0B40A4D0A4F0E4611
:106D30000FCD86B001AC0FC42A683B88226006AA3A
:106D400002EB8303304653F8141C042206B0F0BC57
:106D50000AF014B99C1D01003C9EFF1F164B1B88B6
:106D60000BB31BB283EAE370A0EBE370002B30B5EA
:106D700084B21DDB012300E0134603EB83025200C3
:106D80009042F9DA0D4894FBF3F280FB03E503FB34
:106D90001244DB173032D3EBA503A4B201F8012B68
:106DA000F1D10B7030BD0846042205490AF0E6B85F
:106DB0002D230B700131DDE7849CFF1F676666663B
:106DC00068250100F0B40A4D0A4F0E460FCD86B07B
:106DD00001AC0FC42A683B88226006AA02EB830339
:106DE000304653F8141C042206B0F0BC0AF0C6B8B2
:106DF000B01D0100F09BFF1F054B1B881BB9054B05
:106E00001868086070470846042203490AF0B6B8BB
:106E1000989CFF1FF8240100F4240100164B1B88E6
:106E20000BB31BB230B583EAE374A4EBE374002B1D
:106E3000A0B21CDB012300E0134603EB83025200E7
:106E40009442F9DA0D4D90FBF3F285FB03E403FB6A
:106E50001200DB173032D3EBA40380B201F8012B10
:106E6000F1D10B7030BD064B1868086070472D23B8
:106E70000B700131DEE700BF149CFF1F676666667A
:106E8000F8240100164B1B880BB31BB230B583EA04
:106E9000E374A4EBE374002BA0B21CDB012300E03D
:106EA000134603EB830252009442F9DA0D4D90FB36
:106EB000F3F285FB03E403FB1200DB173032D3EB64
:106EC000A40380B201F8012BF1D10B7030BD064B49
:106ED0001868086070472D230B700131DEE700BF92
:106EE000129EFF1F67666666F8240100164B1B881A
:106EF0000BB31BB230B583EAE374A4EBE374002B4D
:106F0000A0B21CDB012300E0134603EB8302520016
:106F10009442F9DA0D4D90FBF3F285FB03E403FB99
:106F20001200DB173032D3EBA40380B201F8012B3F
:106F3000F1D10B7030BD064B1868086070472D23E7
:106F40000B700131DEE700BF089CFF1F67666666B5
:106F50006C250100174B1B881BB31BB270B583EA6D
:106F6000E375A5EBE375002BACB21EDB012300E05B
:106F7000034603EB830040008542F9DA0E4E94FB92
:106F8000F3F086FB03E503FB1044DB173030D3EB53
:106F9000A503A4B201F8010BF1D108480B701060F1
:106FA00070BD074B1868086070472D230B700131C6
:106FB000DCE700BFA09CFF1F6766666670250100C6
:106FC000F8240100164B1B880BB31BB230B583EAC3
:106FD000E374A4EBE374002BA0B21CDB012300E0FC
:106FE000134603EB830252009442F9DA0D4D90FBF5
:106FF000F3F285FB03E403FB1200DB173032D3EB23
:10700000A40380B201F8012BF1D10B7030BD064B07
:107010001868086070472D230B700131DEE700BF50
:10702000F49BFF1F67666666F8240100164B1B88F9
:107030000BB31BB230B583EAE374A4EBE374002B0B
:10704000A0B21CDB012300E0134603EB83025200D5
:107050009442F9DA0D4D90FBF3F285FB03E403FB58
:107060001200DB173032D3EBA40380B201F8012BFE
:10707000F1D10B7030BD064B1868086070472D23A6
:107080000B700131DEE700BF529EFF1F6766666628
:10709000F8240100164B1B880BB31BB230B583EAF2
:1070A000E374A4EBE374002BA0B21CDB012300E02B
:1070B000134603EB830252009442F9DA0D4D90FB24
:1070C000F3F285FB03E403FB1200DB173032D3EB52
:1070D000A40380B201F8012BF1D10B7030BD064B37
:1070E0001868086070472D230B700131DEE700BF80
:1070F000709EFF1F67666666F8240100174B1B88A9
:107100001BB31BB270B583EAE375A5EBE375002BE7
:10711000ACB21EDB012300E0034603EB830040001A
:107120008542F9DA0E4E94FBF3F086FB03E503FB90
:107130001044DB173030D3EBA503A4B201F8010BE8
:10714000F1D108480B70106070BD074B18680860DB
:1071500070472D230B700131DCE700BF509EFF1FED
:107160006766666670250100F8240100074B1B88DE
:10717000022B06D0012B0CBF054B064B186808608C
:107180007047054B18680860704700BFC09DFF1F1F
:10719000782501007C25010074250100054B1B8822
:1071A0001BB1054B186808607047044B18680860ED
:1071B000704700BF929CFF1F8425010080250100BD
:1071C000184B1A8852B3184A128830B50A80B3F99E
:1071D0000030002B83EAE374A4EBE374BCBF2D23DF
:1071E0008B70A0B2ACBF02310331012300E0134623
:1071F00003EB830252009442F9DA0C4D90FBF3F258
:1072000085FB03E403FB1200DB173032D3EBA4034E
:1072100080B201F8012BF1D10B7030BD044B18681E
:1072200008607047529CFF1F8825010067666666EC
:10723000F824010070B53C4D2B780646002B35D163
:107240001C4673780BB9204670BDFAF75DFC374ACF
:10725000374B3848127831781B78007802EB4303BB
:107260004A1E03EB80030E2AEDD801A050F822F04D
:10727000D9720000FB72000047720000D972000052
:10728000477200004772000047720000C77200009A
:10729000477200004772000047720000477200000A
:1072A0004772000047720000C3720000AE212248FE
:1072B00003F0FCFD204804F049F800232B70012462
:1072C000BFE706F0DFFAAF211B4803F0EFFD1B4AD2
:1072D000012313702B70B6E783B91948038804297A
:1072E0004FF6FF7103F1FF320CBF01230B4613442D
:1072F00003F07F03013303800FE073B1013B114AB8
:1073000032F813304BB10E4E0F481049104A3380FB
:107310000123002606700B701370084A0221012316
:1073200011702B70204670BD108BFF1F559EFF1FE4
:10733000569EFF1F579EFF1FC09EFF1F389FFF1FB7
:107340007A9EFF1F8C9DFF1F7C9CFF1F0B9CFF1FC5
:107350003B9FFF1F10B5064B064C1A8820460121A3
:1073600001F022FD21884220BDE8104001F02EBD31
:10737000689CFF1F289CFF1F10B5064B064C1A88FF
:107380002046022101F010FD21884220BDE8104076
:1073900001F01CBDA29CFF1F289CFF1F10B5064BCF
:1073A000064C1A882046042101F0FEFC2188422068
:1073B000BDE8104001F00ABDC29DFF1F289CFF1FC1
:1073C00010B5064B064C1A882046002101F0ECFC53
:1073D00021884220BDE8104001F0F8BC0E9EFF1F3E
:1073E000289CFF1F08B5122001F00AFD054B1988E3
:1073F000884206D0122001F0E9FCBDE8084001F007
:10740000FDBB08BD049EFF1F08B5582001F0F8FC25
:10741000054B1988884206D0582001F0D7FCBDE8FA
:10742000084001F0EBBB08BD129EFF1F08B51420F9
:1074300001F0E6FC054B1988884206D0142001F0C3
:10744000C5FCBDE8084001F0D9BB08BDA69CFF1FE4
:10745000F0B480EAE075A5EBE0750028ACB21FDB64
:107460001DBF2B230B704E1C0E46012300E013465C
:1074700003EB830252009542F9DA0B4F94FBF3F2CF
:1074800087FB030503FB1244DB173032D3EBA50364
:10749000A4B206F8012BF1D133700846F0BC704756
:1074A0002D230B704E1CE0E767666666084B188854
:1074B00028B10D2807D00D3800B2FFF7C9BF054A23
:1074C000106808607047044A10680860704700BF81
:1074D000969EFF1FF82401008C250100174B188889
:1074E0000C2813D0192815D01A2817D01B2819D00A
:1074F0001C281BD01D281DD01E2803D00C3800B21C
:10750000FFF7A6BF0E4A1068086070470D4A106862
:10751000086070470C4A1068086070470B4A106892
:10752000086070470A4A106808607047094A106886
:1075300008607047084A106808607047469EFF1F41
:10754000A82501009025010094250100982501003F
:107550009C250100A0250100A4250100034B1888EB
:10756000A0EB8000400000B2FFF772BF209FFF1F1A
:10757000024B1888033800B2FFF76ABF209EFF1F36
:10758000024B18880C3800B2FFF762BF049CFF1F43
:10759000024B1888183800B2FFF75ABF349CFF1FFF
:1075A000024B1888183800B2FFF752BF329CFF1FF9
:1075B000024B1888183800B2FFF74ABF2A9CFF1FF9
:1075C000C3681888183800B2FFF742BF054B1B8804
:1075D0001BB9054B18680860704708460422034928
:1075E00009F0CCBC8C9EFF1FF8240100F42401009C
:1075F000054B1B881BB9054B186808607047084687
:107600000422034909F0BABC3C9CFF1FF824010086
:10761000F424010030B5134C85B001252B463C22E3
:1076200002212046009503F0B7FC204603F08EFEB1
:1076300000224021802320460191009311460A4BED
:10764000029504F031FB204603F08CFF07480849FF
:10765000084A0023036083800B608B801360938053
:1076600005B030BDC09EFF1F60200100A49EFF1F1B
:10767000B89EFF1F289FFF1F10B500EBC00000F150
:107680000F02D2B293B284B09C1E981C3D2303918A
:107690008DE819003921024804F06AFA04B010BDDF
:1076A000C09EFF1F014B01221A707047B19EFF1F41
:1076B000F0B5664B664C674F674E684D85B0042247
:1076C0008DE80C0002932046654B4022802103F098
:1076D0006BFA2046634A6449644C08F0CFFD644B62
:1076E00064489F61644FDF61644FB761644FF76125
:1076F000644FAF61644FEF61644FA761644FE7610E
:10770000644F87616449654FC761654F8F61654A02
:10771000654FCF61654F9761654B664FD761664F87
:107720009F61664E664FDF61664FB761664D674F7A
:10773000F761674F674CAF61674FEF61674F68480C
:10774000A761684FE761684F68498761684FC76103
:10775000684F694A8F61694FCF61694F694B976183
:10776000694FD761694F6A4E9F616A4FDF616A4F07
:107770006A4DB7616A4FF7616A4FAF616A4C6B4FF0
:10778000EF616B4FA7616B486B4FE7616B4F876190
:107790006B496C4FC7616C4F8F616C4A6C4FCF6106
:1077A0006C4F97616C4B6D4FD7616D4F9F616D4E04
:1077B0006D4FDF616D4FB7616D4D6E4FF7616E4F6D
:1077C000AF616E4C6E4FEF616E4FA7616E486F4FA9
:1077D000E7616F4F87616F496F4FC7616F4F704AA5
:1077E0008F61704FCF61704F704B9761704FD76151
:1077F000704F714E9F61714FDF61714F714DB76175
:10780000714FF761714F724CAF61724F724873499B
:10781000EF61734F734DA761E561734F734D744C06
:10782000DFF8F0E1734A744B8761744EC561744FA1
:107830008C61744D744CC1F81CE0744874499761B4
:10784000D5619C61D861B16005B0F0BD40420F00C8
:10785000C09EFF1F81750000108FFF1F808EFF1FCD
:10786000D090FF1F1C89FF1F01AC0000788CFF1F08
:10787000988DFF1F348FFF1F856300007175000016
:1078800091630000D9650000557300000166000097
:107890007973000029660000748DFF1F9D7300003E
:1078A0001D6C0000E48CFF1FA16300005166000006
:1078B000508DFF1FC17300005D7500002C8DFF1FF0
:1078C00089680000A1680000EC8EFF1F9568000029
:1078D000516C00000C8CFF1F696B0000856C000070
:1078E000A08FFF1FE5730000856E0000C08CFF1F96
:1078F00009740000F9680000C88BFF1FB163000025
:10790000796600000C90FF1F2D740000ED6E0000E2
:107910009C8CFF1FC1630000556F0000BC8DFF1FD2
:10792000D1630000C56F0000548CFF1FE1630000AD
:1079300059690000388BFF1FF1630000C16C000023
:10794000088DFF1F01640000C1710000C88EFF1F79
:1079500011640000F56C00009090FF1F216400008E
:107960002D7000005C8EFF1F3164000095700000D8
:107970005C8BFF1F41640000296D0000C48FFF1F56
:10798000896B0000FD700000A48EFF1F5164000091
:10799000DD740000808BFF1F616400005D6D0000DE
:1079A000148BFF1F71640000C56D0000808AFF1FEB
:1079B00081640000AD7400006090FF1F91640000BE
:1079C000B1690000308CFF1FA1640000096A00004B
:1079D000EC8AFF1FB1640000A48BFF1F588FFF1FAC
:1079E000616A0000C1640000B96A0000D16400004F
:1079F000116B0000C88AFF1FA48AFF1F8490FF1F1D
:107A00006D710000F16400009D71000001650000CF
:107A10009D7F0000E1640000F0B5461C83B00D4678
:107A20000127032336B22AB2044631468DE8880086
:107A30002448ADB204F032F80C23AA1C12B2009311
:107A40000197052321B21F4804F028F81E4A1F4B56
:107A500012881B68BA422AD023D3022A10D11C4CA8
:107A6000A3F6CA0384FB03241C44DB17C3EB2414D2
:107A70000A2CA8BF0A2424EAE474A2B223B202E0CA
:107A800000231A461C460D35AA1A012000930190C6
:107A900012B2314603230B4803F07EFF204603B0A9
:107AA000F0BD0C4CA3F6FC0384FB0324DDE7084C7B
:107AB000A3F6980384FB03241C44DB17C3EBE40404
:107AC000D6E700BFC09EFF1FAC9DFF1F309EFF1F6B
:107AD000898888881F85EB512DE9F0438FB283B0E8
:107AE000DFF84C80BD1D461D2DB204B236B24FF0FA
:107AF00001090AB22346314640460095CDF804906C
:107B000003F07CFF2A463346214640468DE820029A
:107B100003F074FF07F10C020095334612B22146C0
:107B2000CDF80490404603F069FF03B0BDE8F08350
:107B3000C09EFF1F2DE9F043804685B0002956D135
:107B40000121304804F0F0FA2F4998F8062098F8FF
:107B5000083011F80290994522DA4FEA89064D461D
:107B60000C24D8F80C3027489B595F6822B20021BA
:107B700004F0D6FA384609F043F93946024621485E
:107B800004F068FC1F4804F07BFC98F808300135CD
:107B90000934AB42A4B206F1040601DD422CE0D167
:107BA000B9F1000F13D109F1060999450CDA3C230C
:107BB00001213B22039102930093019239233F223A
:107BC0003A21104803F0D4FF05B0BDE8F0830F233D
:107BD00001213B22039102930093019239230C224D
:107BE0003A21084803F0C4FF98F80830DBE7002189
:107BF0003423009301913F230C22024803F0CCFE72
:107C00009EE700BFC09EFF1FB89EFF1F10B5104C1F
:107C10000121204604F08EFA2046012104F084FA66
:107C200020463422552104F07BFA204602220949DD
:107C300004F010FC20460522074904F00BFC204606
:107C400004F01EFC2046BDE8104003F08BBC00BFD2
:107C5000C09EFF1FAC250100B025010070B50D4688
:107C6000064609F0CDF800EB40008400002D36D028
:107C7000284609F0C5F800EB4000400023185B10CF
:107C800003F16001091A282209B21748C3F1600400
:107C900004F046FA0121144804F046FA284609F097
:107CA000AFF829460246104804F0D4FB0E4804F011
:107CB000E7FB02210C4804F037FA21B221220A48DE
:107CC00004F02EFA304609F09BF831460246064889
:107CD00004F0C0FB0448BDE8704004F0D1BB641060
:107CE000C4F16004E5E700BFC09EFF1F184B70B5EC
:107CF000B3F9003083EAE374A4EBE374002B82B0A1
:107D0000A1B21EDB68466D46012300E0134603EB7B
:107D1000830252009442F9DA0E4E91FBF3F286FB95
:107D200003E403FB1211DB173032D3EBA40389B257
:107D300005F8012BF1D119462B70FFF78FFF02B028
:107D400070BD2D238DF800300DF101056846DBE78D
:107D5000D09DFF1F6766666610B50D4B1B5C51F822
:107D60002340237884B013B1012004B010BD04AACD
:107D700001A942F8103D2046A3699847A38A9B07B2
:107D8000F2D401A80099FFF769FF012004B010BDEB
:107D9000A49EFF1F2DE9F04F2F4DDFF8CCB0DFF888
:107DA000C4A0DFF8C8900FCD91B003AC0FC40FCDC5
:107DB0000FC40FCD0FC42B6823600025A8462F46A3
:107DC0002E4600E09846BAF8003024495BF823209C
:107DD00028461123F8F730FE00EBC00400EB8400C6
:107DE00089FB00340444C017C0EB6434C4F13C0088
:107DF000C6F13C0207F14101012600B208F141033E
:107E000000901BB2019612B209B2154803F0F6FDBC
:107E100008EB060305F211153C2B2646ADB247468A
:107E2000D0D134226B210E4804F07AF900210C489D
:107E300004F07AF90B4B1B8810AA02EB830353F86A
:107E4000344C204608F0DCFF02460548214611B0BC
:107E5000BDE8F04F04F0FEBAC41D01003C1701005C
:107E6000C09EFF1F189CFF1FA01501000900028083
:107E700010B5424C424882B003F068FA2378C3B987
:107E800006213F4804F050F92378012B37D90A2204
:107E9000022B11463A486BD004F042F939490322CB
:107EA000374804F0D7FA364802B0BDE8104004F075
:107EB000E7BA354B1A7801210523002A35D1019103
:107EC000009311462E4803F0E9FD304B1A78002A42
:107ED00036D0052301220192009300220A2128486E
:107EE00003F05AFD2A4B1A78002A35D101210523C7
:107EF000019100931421224803F0D0FDC0E7254CE6
:107F00002388092B32D9632B8CBF0A211F210A2217
:107F10001B4804F005F92188194804F001FB1848B2
:107F200002B0BDE8104004F0ABBA0022019100930A
:107F30001146134803F030FD144B1A78002AC8D1BB
:107F400005230121019100930A210D4803F0A6FDAC
:107F50000F4B1A78002AC9D0012205230192009301
:107F600000221421064803F017FD89E73021CEE7EF
:107F700004F0D6F80322084992E700BF3B9FFF1F99
:107F8000C09EFF1FBC250100559EFF1F569EFF1F70
:107F9000579EFF1F7A9EFF1FB8250100F8B56D4D53
:107FA000287840B96C4B1B6899425CD36B4A01231B
:107FB00013702B70F8BD0C4600266948664F03F01D
:107FC000C5F904F6AC53324665483B6031212E704A
:107FD00004F0A6F801216248624D04F0ABF8314686
:107FE0005F4804F0A1F805225F495D4804F032FAC9
:107FF0005B4804F045FA0C221021594804F090F82F
:108000000B225A49564804F025FA0522584954488B
:1080100004F020FA524804F033FA564B50481C68DA
:10802000A4F69803C3EB031385FB03251D4410211D
:10803000DB172022C3EB652504F072F840F6CC3341
:108040009C4205F124054FF022014FF004000BDCA7
:10805000FFF7E2FC484B1C88064674B3012C46D05F
:10806000022C41D00120F8BDFFF736FD092243491B
:108070003B4804F0EFF92A221021394804F050F867
:108080003F4C374884FB0534EB17C3EBA40421466F
:1080900004F046FA01223B49314804F0DBF904EBD5
:1080A0008401A5EB41012E4804F03AFA0122364939
:1080B0002B4804F0CFF90120F8BD3449102228489C
:1080C00004F0C8F9264804F0DBF92A2210212448DC
:1080D00004F026F83146224804F022FA07222C49FF
:1080E0001F4804F0B7F9CBE70C222A49E7E70C2236
:1080F00029491B4804F0AEF9194804F0C1F92A22B5
:108100001021174804F00CF8314615481C4E04F0B5
:1081100007FA07221E49124804F09CF986FB05362F
:10812000EB17C3EBA60631460D4804F0F9F92246D9
:1081300014490B4804F08EF906EB8601A5EB4101CA
:10814000074804F0EDF922460F49054804F082F98A
:108150002046F8BD108BFF1F3C9FFF1F389FFF1F5D
:10816000C09EFF1F3B773B98C0250100C82501003A
:10817000B0250100309EFF1FAC9DFF1FD4250100DC
:1081800067666666082D0100782C0100E025010075
:10819000F42501000C260100FC2501002DE9F04129
:1081A000754C2278002A05460F4614BF4FF001088F
:1081B0004FF000084ED1714E3368CB1AB3F5FA6F09
:1081C00004D86B78A3B94046BDE8F0816C4B6D488C
:1081D0006D49DFF8D0E11A7001230370098823701C
:1081E00026208EF8002000F0F1FD6B78002BEAD0FD
:1081F0003760F9F789FC654A654B6649127828783B
:108200001B78097802EB4303421E03EB81030E2A1D
:10821000D9D801A151F822F009830000D5820000CD
:10822000C781000009830000C7810000C7810000EA
:10823000C7810000BD820000C78100006F8200007E
:10824000C7810000C7810000C7810000C78100000E
:108250006B820000AF215048484E02F027FEFFF726
:1082600007FE002337602370ABE705F00BFB4A489D
:1082700003F06CF80221484803F056FF0F22232137
:10828000454803F04DFF05224449434804F0E2F815
:10829000414804F0F5F81E2223213F4803F040FF37
:1082A00005223F493C4804F0D5F83B4804F0E8F883
:1082B000394803F057F900F0ADFC84E7394D2B78CD
:1082C000012B50D9304B2620198800F07FFD002368
:1082D0002B7078E7002B3FF476AF013B324A32F83F
:1082E0001330002B3FF46FAF274C304825492D4AFF
:1082F00023804FF001080023037081F8008082F88A
:108300000080FFF7B5FD5EE793B1013B264A32F8E6
:10831000131019B31C4B254D1A4C224A1980002604
:10832000012326202E702370137000F04FFD15E0FE
:10833000154C1E4922880B7004284FF6FF7002F17D
:10834000FF310CBF012202460A440E4E154D02F0C9
:108350007F0201320121228031702B70FFF788FDEE
:108360004FF001082FE70649064A01230020087054
:1083700013702370A6E700BF108BFF1F349FFF1FF1
:10838000389FFF1F0B9CFF1F7A9EFF1F559EFF1FEC
:10839000569EFF1F579EFF1FC09EFF1F1C260100F9
:1083A000242601003B9FFF1F8C9DFF1F7C9CFF1F0D
:1083B0002DE9F04F05468BB00F46AD48012116461A
:1083C00003F0B8FEAA8812F0010440F0B080DFF894
:1083D000CC8298F80030002B7DD1AB79A54AD15CD6
:1083E000A1B9DFF8BCA279781AF8039041B33978C3
:1083F0000139072900F2B780DFE811F0F1005401DC
:10840000B5006C01B500B500B500E9007C78002C22
:1084100000F0CA800139EC68387854F82170FC68A3
:10842000411EB4F80080072900F2A780DFE811F0B0
:1084300074015901A5006C01A500A500A5009F00CD
:10844000DFF854A2DAF80020B21AB2F5967F75D997
:10845000894A107801281ABF012010701170874ACC
:1084600018BF0146D05CC0EB0900C0B2FFF704F9A9
:108470000124CAF80060AB889B0770D57B78002B7D
:108480006DD0F9F741FB7E4B7E4A7F481B7812780E
:1084900039780078022515FB02330A2903EB8003A3
:1084A00000F04E810C295AD1002B58D003F119004D
:1084B000764E774A013B0021400080B226F8131027
:1084C0000123157088F8003000F080FC714B032206
:1084D00020461A702FE0664802F038FF01216448F8
:1084E00003F022FE62482246214603F019FEAB88C3
:1084F000580725D42C68204608F082FC2146024605
:108500005B4803F0A7FF5A4803F0BAFF0922012392
:108510008DE80C0000217F23554803F06FFA0021FD
:108520002846FFF707FB002388F8003055E7AB68C3
:108530003146384698470BB0BDE8F08F0846FAE759
:108540002B6804A8984704A808F05AFC04A902461E
:10855000474803F07FFF464803F092FFD6E72046E6
:108560000BB0BDE8F08F00240AF8039083E70021E8
:10857000D1543846FB699847FC68A4F8008000276E
:1085800025223C238DE8840041211822384803F03D
:1085900003FAE968A879FFF7DFFB374A3E4B17700B
:1085A0001E600BB0BDE8F08F3B490A68B21AB2F505
:1085B000967FD4D9304F0E603E78012E00F0B48003
:1085C000E968184601233B70FFF7C6FBB3E7304A62
:1085D000E9791170012288F800200024C4E72A7A82
:1085E000013A4A45BFDD09F10104E4B2A145BAD020
:1085F000224E16F803B0CBEB0900C0B20021FFF702
:108600003BF82B7A052BD9461BD9CBEB0402042A65
:1086100040F3AE80A4F1040BBBF1000FC0F2B080B8
:10862000063B5B45A8BF5B465FFA83F9AA7913480E
:10863000B15C994205D000F8029001212846FFF76D
:1086400079FAC9EB0400C0B201210B4EFFF714F810
:1086500000213423019100930548317040230B22FF
:108660003F21A14603F098F90124AB797CE700BFD4
:10867000C09EFF1F289FFF1F399FFF1FB89EFF1F2F
:10868000559EFF1F569EFF1F579EFF1F8C9DFF1F6D
:10869000389FFF1F3B9FFF1F249FFF1F108BFF1F53
:1086A000A49EFF1F0FFA89F1E868604C50F8216022
:1086B0002168049134785E4904980860002C71D0D8
:1086C000012C7FF450AF5B4A317A88F8004011707A
:1086D000002449E7B9F1000F50D009F1FF34E4B2AA
:1086E00084E7B98A01F0040189B200293FF440AF60
:1086F0003B6A03929847039A00283FF43DAFAB7959
:10870000FC680021D15438E77B8A43453CD908F105
:1087100001081FFA88F830E73B8A43453BD208F14D
:10872000FF381FFA88F828E725238DE8180042480B
:108730003C703C231822412103F02EF93046FAE622
:10874000002B3FF40CAF3D4A3D4E1188394A03F1EE
:108750001900013B400080B226F81310012388F86D
:108760000030157000F032FB364B20461D70E2E6FB
:10877000002A3FF755AF04F1FF3B4DE74C46F3E6C7
:108780004FF000094B4651E7BB8ADA077FF5F5AE9B
:10879000B7F81080F1E6BB8AD9077FF5EEAEB7F8DF
:1087A0001280EAE62849C85CC0EB090009F1010E15
:1087B000C0B201214FF0340B02F803E0FEF75CFF7A
:1087C000B6681D48019440230B223F210124CDF8B7
:1087D00000B003F0E1F840230B223F211648CDF80A
:1087E00000B0019403F05AF92146134803F09CFCB1
:1087F000304608F005FBA0EB800000F15F0109B2F4
:108800000F220D4803F08CFC304608F0F9FA31468F
:108810000246094803F01EFE074803F031FEE968EE
:10882000A879FFF799FAAB799EE600BF7C9FFF1FFE
:10883000249FFF1F389FFF1FC09EFF1F7A9EFF1FB0
:108840008C9DFF1F3B9FFF1FB89EFF1F2DE9F04728
:10885000DFF808926D4B99F800601B68DFF800A202
:1088600082B0003601934FF0030018BF0126019F2C
:108870009AF8008004F0BEFC0546042004F0BAFC1F
:108880000446052004F0B6FC800040EA44040620BB
:1088900004F0B0FC2C4364B25D4944EAC0000A789D
:1088A00080F00F03DBB29A425A4A3CD01760002294
:1088B00059480B7003788DF800808DF8012053B370
:1088C000564A12684EF66021BA1A8A4219D8022B0B
:1088D00059D0012B5FD0062B48D0032B63D0042B3B
:1088E00069D0052B77D0072B7DD0082B00F0838033
:1088F000092B68D016B14A4802F034FE02B0BDE838
:10890000F087484A484C002301212370037013600C
:10891000938089F800103A4669464448FFF748FDBD
:108920003043C6B2E6E71268BA1A1E2A6BD99AF823
:108930000020934222D0394C3D488AF80030012B68
:10894000276082EA030207609846B1D0042BAFD1BA
:1089500037480068381AB0F5C87FA9D9354C206867
:10896000381A3228A4D927601A46A1E73A46694640
:108970003148FFF71DFD3043C6B2BBE7012B4FF076
:108980000002E3D1E4E73A4669462C48FFF710FDC0
:108990003043C6B2AEE73A4669462948FFF708FDBC
:1089A0003043C6B2A6E73A4669462648FFF700FDBF
:1089B0003043C6B29EE73A4669462348FFF7F8FCC3
:1089C0003043C6B296E73A4669462048FFF7F0FCC6
:1089D0003043C6B28EE73A4669461D48FFF7E8FCC9
:1089E0003043C6B286E73A4669461A48FFF7E0FCCC
:1089F0003043C6B27EE73A4669461748FFF7D8FCCF
:108A00003043C6B276E7002252E700BF7C9FFF1FCB
:108A1000409FFF1FAC9EFF1F389FFF1F309FFF1F0F
:108A2000C09EFF1F289FFF1F3A9FFF1F302001009D
:108A3000449FFF1FB49EFF1F60240100881F010098
:108A40008C1E0100041E0100C82B01007C1E0100C9
:108A5000E41E01006C1F01008490FF1F108BFF1F9C
:108A6000B09EFF1F28B11028044BA8BF102018602B
:108A70007047024B01201860704700BF489FFF1FDE
:108A800038B50F4D2B78013B01381B02C4B203F4FB
:108A90007063200443F4404343F00C0300F4FE00F1
:108AA000184305F00FFD2868013860F03F00C0B2A0
:108AB00004F036FD2046BDE8384004F031BD00BF6B
:108AC000489FFF1F70B5124D2B78013B1B0203F42A
:108AD0007063064643F430430806320400F0FE405B
:108AE00043F00B03034302F4FE0018430C4605F069
:108AF000E9FC2868013860F04F00C0B204F010FDB6
:108B0000304604F00DFD2046BDE8704004F008BD7D
:108B1000489FFF1F70B5124D2B78013B1B0203F4D9
:108B20007063064643F410430806320400F0FE402A
:108B300043F00903034302F4FE0018430C4605F01A
:108B4000C1FC2868013860F06F00C0B204F0E8FC96
:108B5000304604F0E5FC2046BDE8704004F0E0BC7F
:108B6000489FFF1F38B5104D2B78013B1B0203F4C3
:108B70007063044643F41043000443F0090300F417
:108B8000FE00184305F09EFC2868013860F06F0075
:108B9000C0B204F0C5FC204604F0C2FC0020BDE8D1
:108BA000384004F0BDBC00BF489FFF1F38B50E4DD4
:108BB0002B78013B1B0203F47063044643F45043DB
:108BC000000443F00D0300F4FE00184305F07AFCA6
:108BD0002868013860F02F00C0B204F0A1FC2046E4
:108BE000BDE8384004F09CBC489FFF1F08B500203A
:108BF00005F032FD0028FAD108BD00BF08B5642198
:108C00000720FFF75FFF7F210B20BDE80840FFF73B
:108C100059BF00BF10B500217B20FFF753FF002490
:108C2000E0B2FFF79FFF0134022004F019FB802C13
:108C3000F6D110BD10B504464FF4406004F020FC9E
:108C400004F078FC2CB1102C044BA8BF10241C603D
:108C500010BD024B01241C6010BD00BF489FFF1FC8
:108C600010B5044641F0E00004F05AFC04F07F0027
:108C700004F056FCC4F3C610BDE8104004F050BC2C
:108C800038B5134D2B78044641F6FF72A0F500501D
:108C9000824203F1FF33A8BF02461B0202F50052D5
:108CA00003F47063100443F4604343F00E0300F4D4
:108CB000FE005204184302F0FE42104305F002FC8D
:108CC000296801392046C9B2BDE83840FFF7C8BF5E
:108CD000489FFF1F38B504460D46F02004F020FCE5
:108CE00035B1254414F8010B04F01AFCAC42F9D15B
:108CF000F720BDE8384004F013BC00BF00B50B4BB3
:108D000083B00246998818680090032AADF80410D1
:108D100002D903B05DF804FB684606218DF80520F2
:108D2000FFF7D8FF03B05DF804FB00BF382C01004B
:108D300000B50B4B024683B0186899880090131F4A
:108D40004C2BADF8041002D903B05DF804FB684663
:108D500006218DF80520FFF7BDFF03B05DF804FB89
:108D6000402C0100030203F4FE43C0F3C610184375
:108D7000704700BF03784078DB0103F47E5300F0B6
:108D80007F001843704700BF82B002AA114642F824
:108D9000040D002012F8013B03F07F03914243EAE7
:108DA0000020F7D102B07047003210B403884FF0B2
:108DB000010404FA01F418BF012202FA01F123EAC6
:108DC00004020A43028010BC704700BF70B5CEB2E7
:108DD0000C46054603F0D6FD864203D031462846B0
:108DE00003F0EAFD0135284603F0CCFD240A844255
:108DF00005D021462846BDE8704003F0DDBD70BDBA
:108E000038B5054603F0BEFD4FF0000460F30704DB
:108E1000681C03F0B7FD60F30F24A0B238BD00BF9B
:108E2000F8B504460020FFF7EBFF002C00F01B858F
:108E30004FF4AF610220FFF7C9FF4FF47A610420BD
:108E4000FFF7C4FF4FF496610620FFF7BFFF4FF412
:108E5000FA610820FFF7BAFF4FF4AF610A20FFF76D
:108E6000B5FF40F6FC010C20FFF7B0FF4FF4966110
:108E70002220FFF7ABFF4FF416612420FFF7A6FF77
:108E80007D212A20FFF7A2FF0C210E20FFF79EFF75
:108E900001211020FFF79AFF02211220FFF796FF11
:108EA00000211420FFF792FF00211620FFF78EFF0C
:108EB00002211820FFF78AFF01211A20FFF786FF01
:108EC00002211C20FFF782FF04211E20FFF77EFFF6
:108ED00014212020FFF77AFF01212620FFF776FFDB
:108EE00003212820FFF772FF04212C20FFF76EFFDB
:108EF00014212E20FFF76AFF00213020FFF766FFC4
:108F00000C213220FFF762FF00213420FFF75EFFC3
:108F100000213620FFF75AFF00213820FFF756FFC7
:108F200000213A20FFF752FF00213C20FFF74EFFBF
:108F300000213E20FFF74AFF00214020FFF746FFB7
:108F400000214220FFF742FF1F214420FFF73EFF90
:108F500013214620FFF73AFF0E214820FFF736FF86
:108F600011214A20FFF732FF0A214C20FFF72EFF84
:108F700000214E20FFF72AFF06215020FFF726FF91
:108F800002215220FFF722FF0C215420FFF71EFF81
:108F900000215620FFF71AFF00215820FFF716FF87
:108FA00001215A20FFF712FF03215C20FFF70EFF7B
:108FB0000A215E20FFF70AFF00216020FFF706FF6D
:108FC00004216220FFF702FF01216420FFF7FEFE6B
:108FD00000216620FFF7FAFE0B216820FFF7F6FE5E
:108FE0007F216A20FFF7F2FE00216C20FFF7EEFEE2
:108FF00000216E20FFF7EAFE00217020FFF7E6FE59
:1090000000217220FFF7E2FE00217420FFF7DEFE50
:109010001F217620FFF7DAFE13217820FFF7D6FE16
:109020000E217A20FFF7D2FE11217C20FFF7CEFE21
:109030000A217E20FFF7CAFE1F218020FFF7C6FE0F
:1090400013218220FFF7C2FE0E218420FFF7BEFE0F
:1090500011218620FFF7BAFE0A218820FFF7B6FE0D
:1090600000218A20FFF7B2FE01218C20FFF7AEFE1F
:1090700000219620FFF7AAFE00219820FFF7A6FE08
:1090800000219A20FFF7A2FE05219C20FFF79EFEFB
:1090900006219E20FFF79AFE0021A020FFF796FEF2
:1090A00027210020FFF792FE0220FFF7A9FEB0F56E
:1090B000805F034680F04785D24A04201380FFF783
:1090C0009FFEB0F5805F034680F03485CE4A0620CF
:1090D0001380FFF795FEA0F52F739BB2B3F57A6F5F
:1090E000024606D940F628210620FFF76FFE40F61B
:1090F0002822C64B08201A80FFF782FEA0F52F73A6
:109100009BB2B3F57A6F024606D940F6E4410820D7
:10911000FFF75CFE40F6E442BD4B0A201A80FFF7E1
:109120006FFEA0F5FA739BB240F6AC518B4202463B
:1091300006D94FF4AF610A20FFF748FE4FF4AF6243
:10914000B44B0C201A80FFF75BFEA0F5FA739BB2BC
:1091500040F6AC518B42024606D940F6FC010C2089
:10916000FFF734FE40F6FC02AB4B0E201A80FFF7EF
:1091700047FE1828034600F2D684A84A1020138020
:10918000FFF73EFE431E9BB20F2B024604D901217E
:109190001020FFF71BFE0122A14B12201A80FFF7BF
:1091A0002FFE0A28034600F2B7849E4A142013803B
:1091B000FFF726FE0128034604D900211420FFF7FB
:1091C00005FE0023984A16201380FFF719FE7F281A
:1091D000034600F29A84954A18201380FFF710FE88
:1091E0000428034600F28A84914A1A201380FFF76C
:1091F00007FE0C28034600F27A848E4A1C20138056
:10920000FFF7FEFD0428034600F26A848A4A1E2006
:109210001380FFF7F5FD0928034600F25A84874AB8
:1092200020201380FFF7ECFD4628034600F24A8415
:10923000834A22201380FFF7E3FDA0F5FA739BB267
:1092400040F6AC518B42024606D94FF4966122207B
:10925000FFF7BCFD4FF496627A4B24201A80FFF78B
:10926000CFFDA0F5FA739BB240F6AC518B4202469B
:1092700006D94FF416612420FFF7A8FD4FF41662BB
:10928000714B26201A80FFF7BBFD7F28034600F2B2
:1092900012846E4A28201380FFF7B2FD0628034689
:1092A00000F202846A4A2A201380FFF7A9FDA0F188
:1092B00032039BB2B3F5967F024604D97D212A2062
:1092C000FFF784FD7D22634B2C201A80FFF798FD69
:1092D0000C28034600F2E2835F4A2E201380FFF73A
:1092E0008FFD1E28034600F2D3835C4A3020138092
:1092F000FFF786FD0928034600F2C483584A32204E
:109300001380FFF77DFD1E28034600F2B583554A02
:1093100034201380FFF774FD7F28034600F2A683F4
:10932000514C36202380FFF76BFD7F28034600F267
:10933000978338206380FFF763FD7F28034600F2A0
:1093400089833A20A380FFF75BFD7F28034600F264
:109350007B833C20E380FFF753FD7F28034600F228
:109360006D833E202381FFF74BFD7F28034600F2EB
:109370005F8340206381FFF743FD7F28034600F2AF
:1093800051834220A381FFF73BFD384D28804420C4
:10939000FFF736FD3028034600F23E83344A46206C
:1093A0001380FFF72DFD3028034600F22F83314C48
:1093B00048202380FFF724FD3028034600F2208355
:1093C0004A206380FFF71CFD3028034600F2128319
:1093D0004C20A380FFF714FD3028034600F20483DD
:1093E0004E20E380FFF70CFD0128034604D900213D
:1093F0004E20FFF7EBFC00231F4A50201380FFF79D
:10940000FFFC3BE0B49CFF1F6A9EFF1F6A9CFF1F8E
:10941000449EFF1F149EFF1F309CFF1F049CFF1FD4
:10942000D09DFF1F049EFF1FA69CFF1F089CFF1FCF
:10943000B89CFF1F529CFF1F4A9CFF1F149CFF1FDC
:10944000509EFF1FC89DFF1FC49DFF1F7A9EFF1FD8
:10945000209EFF1F649EFF1F189CFF1FA09CFF1FE4
:10946000F49BFF1F469EFF1F8C9DFF1F289CFF1F24
:109470002A9CFF1F249EFF1F489CFF1F431E9BB278
:109480000B2B024604D906215020FFF79FFC062231
:10949000CD4B52201A80FFF7B3FC0428034600F29C
:1094A0009D82CA4A54201380FFF7AAFC431E9BB238
:1094B0001D2B024604D90C215420FFF787FC0C22F7
:1094C000C34B56201A80FFF79BFC0128034604D9A2
:1094D00000215620FFF77AFC0023BE4A5820138053
:1094E000FFF78EFC7F28034600F27282BA4A5A20A8
:1094F0001380FFF785FC431E9BB2092B024604D95B
:1095000001215A20FFF762FC0122B44B5C201A8033
:10951000FFF776FC431E9BB2102B024604D90321B1
:109520005C20FFF753FC0322AD4B5E201A80FFF74F
:1095300067FC431E9BB21D2B024604D90A215E2004
:10954000FFF744FC0A22A74B60201A80FFF758FC63
:109550000228034600F23682A34A64201380FFF7F4
:109560004FFC0128034604D901216420FFF72EFC9B
:1095700001239E4A62201380FFF742FCC31E9BB268
:10958000012B024604D904216220FFF71FFC0422AC
:10959000974B66201A80FFF733FC7F28034600F2C2
:1095A0000B82944A68201380FFF72AFC7F28034629
:1095B00000F2FC81904A6A201380FFF721FC7F288B
:1095C000034600F2ED818D4A6C201380FFF718FCF2
:1095D0000428034600F2DE81894A6E201380FFF7DB
:1095E0000FFC1928034600F2CF81864A70201380B1
:1095F000FFF706FC0228034600F2C081824A72206F
:109600001380FFF7FDFB0628034600F2B1817F4A75
:1096100074201380FFF7F4FB0428034600F2A281B4
:109620007B4A8A201380FFF7EBFB0A28034600F2EF
:109630009381784A8C201380FFF7E2FB04280346CD
:1096400000F28481744A98201380FFF7D9FB012827
:10965000034604D900219820FFF7B8FB00236F4A86
:109660009A201380FFF7CCFB0128034604D9002180
:109670009A20FFF7ABFB0023694A96201380FFF77F
:10968000BFFB0B28034600F25B81664A9C201380D7
:10969000FFF7B6FB831E9BB2032B024604D90521BC
:1096A0009C20FFF793FB05225F4B76201A80FFF783
:1096B000A7FB3028034600F23D815C4A78201380E6
:1096C000FFF79EFB3028034600F22E81584C7A208B
:1096D0002380FFF795FB3028034600F21F817C2092
:1096E0006380FFF78DFB3028034600F211817E2056
:1096F000A380FFF785FB3028034600F2038180201A
:10970000E380FFF77DFB3028034600F2F580494AED
:1097100082201380FFF774FB3028034600F2E680B6
:10972000454C84202380FFF76BFB3028034600F272
:10973000D78086206380FFF763FB3028034600F262
:10974000C9808820A380FFF75BFB3028034600F226
:10975000BB80A020E380FFF753FB0128034604D918
:109760000021A020FFF732FB0023344A9E20138003
:10977000FFF746FBC31E9BB20C2B04D99E2006218B
:10978000FFF724FB06202B88DFF8D0E02C4F2D4A72
:109790002D4D2E4E2E4C2F4903F0010CAEF800C07B
:1097A000C3F3400EA7F800E0C3F380071780C3F3AC
:1097B000C007294A2F70C3F30017C3F34015C3F342
:1097C0008013378025804BE0148AFF1F5E89FF1FBE
:1097D000168AFF1F929CFF1F129EFF1F009CFF1FF7
:1097E000648AFF1F5C89FF1FC09DFF1F1C9EFF1F17
:1097F000589CFF1F529EFF1F849CFF1F3E9CFF1F13
:10980000F09BFF1F969EFF1FAC9DFF1F709EFF1FCA
:109810003C9EFF1FD29DFF1FBA9DFF1F3C9CFF1F58
:10982000989CFF1F0C9EFF1F1E9CFF1F329CFF1F5A
:109830009C9DFF1F349CFF1FA49DFF1F8C9EFF1F3C
:10984000689CFF1FA29CFF1FB09DFF1FC29DFF1FB2
:109850001E9EFF1FD69DFF1FC089FF1F0E9EFF1F6C
:109860000B801080F8BD4FF6FF7398423FF4E0AADA
:1098700027283FF419AC17287FF6DAAA19287FF6B3
:1098800043AB1B287FF660AB1C283FF475AB1E284A
:109890007FF67AAB1F283FF47FAB20283FF498ABCC
:1098A00021283FF4A1AB22283FF4A6AB23283FF4A4
:1098B000AFAB24283FF4E0AB25283FF4E5AB2628E6
:1098C0007FF4EEABFFF7E4BB0A218820FFF77EFAB6
:1098D0000A233EE711218620FFF778FA112330E7AB
:1098E0000E218420FFF772FA0E2322E71321822033
:1098F000FFF76CFA132313E71F218020FFF766FAA6
:109900001F2304E70A217E20FFF760FA0A23F6E608
:1099100011217C20FFF75AFA1123E8E60E217A2064
:10992000FFF754FA0E23DAE613217820FFF74EFAF8
:109930001323CBE61F217620FFF748FA1F23BCE64E
:1099400000219620FFF742FA00239EE601218C2099
:10995000FFF73CFA012375E600218A20FFF736FA6B
:10996000002366E600217420FFF730FA002357E653
:1099700000217220FFF72AFA002348E60021702018
:10998000FFF724FA002339E600216E20FFF71EFAC4
:1099900000232AE600216C20FFF718FA00231BE6BB
:1099A0007F216A20FFF712FA7F230CE60B21682043
:1099B000FFF70CFA0B23FDE500216620FFF706FAFE
:1099C0000023EEE500216020FFF700FA0023C3E545
:1099D00000215820FFF7FAF9002387E502215220E1
:1099E000FFF7F4F902235CE50A214C20FFF7EEF9BA
:1099F0000A23F5E411214A20FFF7E8F91123E7E4EF
:109A00000E214820FFF7E2F90E23D9E41321462066
:109A1000FFF7DCF91323CAE41F214420FFF7D6F92E
:109A20001F23BBE400214020FFF7D0F90023A8E466
:109A300000213E20FFF7CAF900239AE400213C20D0
:109A4000FFF7C4F900238CE400213A20FFF7BEF9A8
:109A500000237EE400213820FFF7B8F9002370E4EA
:109A600000213620FFF7B2F9002362E40021342000
:109A7000FFF7ACF9002353E40C213220FFF7A6F9DD
:109A80000C2344E400213020FFF7A0F9002335E443
:109A900014212E20FFF79AF9142326E404212C2008
:109AA000FFF794F9042317E403212820FFF78EF928
:109AB0000323FFF7F7BB01212620FFF787F90123D6
:109AC000FFF7E7BB14212020FFF780F91423FFF7ED
:109AD000AFBB04211E20FFF779F90423FFF79FBBDA
:109AE00002211C20FFF772F90223FFF78FBB01212F
:109AF0001A20FFF76BF90123FFF77FBB0221182023
:109B0000FFF764F90223FFF76FBB00211620FFF770
:109B10005DF90023FFF75FBB02211220FFF756F922
:109B20000223FFF742BB0C210E20FFF74FF90C2355
:109B3000FFF723BB4FF47A610420FFF747F94FF496
:109B40007A63FFF7C3BA4FF4AF610220FFF73EF923
:109B50004FF4AF63FFF7B0BAF8B5B32006F0C8FB17
:109B6000204B214A054603CB1368C5F803001A0CA5
:109B7000A220C5F807102B80AA70FFF7F3F82E4635
:109B8000002426F80B0FA0B2FFF73AF9FFF7EAF826
:109B90000234A22C26F8020FF5D16C1E05F1AE0698
:109BA0004FF0FF3014F8013F082758400F4B40F3A7
:109BB00000017A1E0B4012F0FF0783EA5000F5D136
:109BC000B442EFD1C043FFF7DFF83A46C5F8AF0023
:109BD000B321284604F0C4FC2846BDE8F84006F04E
:109BE0008FBB00BF4C2C0100482C01002083B8ED36
:109BF000F0B50E4B0E4C054693E8070085B024687F
:109C00002E88AD7801AB83E80700270C18460022A8
:109C10000B21ADF804408DF80670ADF80C608DF89E
:109C20000E5004F09DFC05B0F0BD00BF582C0100A3
:109C3000482C0100F0B5124B124D1E68124F0FCD8B
:109C400087B06C460FC495E8030044F8040B3868ED
:109C50003B79CDF80D00320C272021808DF80220B1
:109C60008DF81130ADF80060FFF77CF80022ADF8F8
:109C70000B001221684604F073FC07B0F0BD00BF72
:109C8000482C0100642C0100B0250100002004F0E4
:109C9000E3BC00BF02F02EBE70B5124C82B00025AE
:109CA0004023064629462046009301958023202222
:109CB00001F072FE20222946204602F031FA2046A9
:109CC000012102F037FA304607F09AF83146024691
:109CD000204602F0BFFB204602B0BDE8704001F014
:109CE00041BC00BFC09EFF1FF0B5B22983B075D93B
:109CF0000546441E00F1AE064FF0FF3014F8012F68
:109D000008275040404A40F300017B1E0A4013F0F0
:109D1000FF0782EA5000F5D1B442EFD1C043FFF70C
:109D200033F80146D5F8AF000190019A914202D074
:109D3000B2F17F2F0BD105F10B00FFF71BF8A22822
:109D40000BD03248FFF7A8FF002003B0F0BD304829
:109D5000FFF7A2FF384603B0F0BD05F10D00FFF795
:109D600009F8272840D1002440F6AC5613E0042817
:109D70001AD0062821D008281FD00A2828D00C285D
:109D800022D1A1F5FA7292B2B24201D8FFF71EF8C1
:109D90000234A22C0ED004F10D002844FEF7EAFF95
:109DA000022C0146A0B2E2D1B1F5805FEED30234BD
:109DB000A22CF0D1012003B0F0BDA1F52F7292B218
:109DC000B2F57A6FE4D8E1E7222801D0242811D136
:109DD000A1F5FA7292B2B242DAD8D7E70D48FFF78E
:109DE0005BFF002003B0F0BD0B48FFF755FF0020DC
:109DF00003B0F0BD2A28C9D1A1F1320292B2B2F566
:109E0000967FC5D8C2E700BF2083B8EDA82C01001B
:109E1000942C01007C2C0100BC2C010003290CD9DE
:109E200070B5461C82B005460C46304603222A49CE
:109E300007F054F810B102B070BD70470B2C05D973
:109E400005222649281D07F049F840B12448FFF7AC
:109E500023FF244802B0BDE87040FFF7C9BE05F1FA
:109E60000901032201A807F089F801A803221E496D
:109E700007F034F8D8B103221C4901A807F02EF8E6
:109E800008B301A803221A4907F028F8B0B9194805
:109E9000FFF702FFA11E89B23046FFF725FF002819
:109EA000C9D0154802B0BDE87040FFF7F5BE1348B1
:109EB000FFF7F2FEFFF750FE1148F3E71148FFF7F6
:109EC000EBFE1148C6E71148FFF7E6FE02B0BDE819
:109ED0007040FFF7AFBE00BF482C0100D42C01003A
:109EE000DC2C0100F02C0100F42C01001C2D0100E1
:109EF000342D0100382D01004C2D0100F82C0100FB
:109F00000C2D0100602D0100742D0100202D010099
:109F10002DE9F043174D2B6883B081460F469046DC
:109F2000F3B1154E34880A1992B2184611463280A0
:109F300006F05CFD28603A464946204402F06CFD7C
:109F4000B8F1000F09D031882868FFF767FF28684B
:109F500006F0D6F900232B60338003B0BDE8F08310
:109F6000054E01930846318006F0C2F9019B286036
:109F70001C46E0E7509FFF1F4C9FFF1F10B51F4C72
:109F80004FF4FA70FCF776F8204601F0DFF9002272
:109F90001146204602F0C4F82046012102F0CAF81A
:109FA0002046002102F0C0F80B221549204602F09D
:109FB00051FA204602F064FA0F221249204602F0BC
:109FC00049FA204602F05CFA0F490722204602F0C7
:109FD00041FA204602F054FA204601F0C3FA0B4B36
:109FE0000B4A1A604FF4FA70FCF744F8FFF722FEB0
:109FF0000848BDE81040FFF74FBE00BFC09EFF1FDE
:10A00000782D0100842D0100942D010008A1FF1F6F
:10A01000119F00009C2D01000020704790F839200E
:10A0200090F83800101A704790F8383090F83920BE
:10A030009A4205D95A1C034480F83820187E70478C
:10A040004FF0FF30704700BF90F8383090F839205B
:10A050009A4286BF1B18187E4FF0FF30704700BF32
:10A06000704700BF38B50546B0F85E0090B195F86E
:10A070005D301446C3F1210294420CD805F13B0037
:10A080001844224602F0C8FC95F85D30234485F858
:10A090005D30204638BD012014462871EEE700BF30
:10A0A000B0F85E306BB190F85D30202B07D8C21845
:10A0B000013380F85D30012082F83B1070470123A6
:10A0C00003710020704700BF0023426980F83830D8
:10A0D00080F8393080F85C3080F85D3080F85E3090
:10A0E00080F85F3006CA30B40D68046943662A43BD
:10A0F00083660A60A370426990F86130164914685B
:10A1000013441D7A5B7B01EBC5051B026D6803F4EC
:10A11000E06343F064032B6090F8623013449D7C4D
:10A12000DB7D01EBC5011B02496803F4E06343F0EA
:10A1300064030B6021685368194205D00369272224
:10A140005A70036904229A71036920225A710369C3
:10A1500080229A7030BC7047D038010043690CCB24
:10A1600012681A420CD0094B99420AD9084B9942FD
:10A17000036994BF1A220D225A70036904229A714E
:10A180007047036927225A70F7E700BF7F1A06005D
:10A190003F420F0010B50269D378DBB2D9060446FE
:10A1A0003DD510215806D17038D503F0040303F0D3
:10A1B000FF02002B51D03D49626E00230B7084F8E2
:10A1C0005D30002A5BD0904794F85D30002B56D06C
:10A1D0002369D0229A70236994F83B201A7123696D
:10A1E000012284F85C200222DA7010BD304B84F822
:10A1F00060009C424AD02F4B9C4252D094F83910B8
:10A2000013791F29DBB207D82848007820B16018DD
:10A21000013184F8391003760223D37010BD59063A
:10A22000C3D4917801F0100101F0FF000029DDD0C6
:10A2300013F001031ED194F85C1094F85D0088427D
:10A2400081BF4B1C091984F85C3091F83B301371C5
:10A250002369D0229A702269DEE7236984F83920C5
:10A26000C0229A702369114A1979012111700222C2
:10A27000DA7010BDC023937022691379CCE70122F4
:10A28000002384F85D2084F83B30A1E7626994F8EC
:10A290006130094913440322187A02F043FD226910
:10A2A000ACE7626994F861300449F3E7549FFF1FFB
:10A2B000D090FF1F3C91FF1F1DA3000029A30000A9
:10A2C0000369DB7803F0200373B190F86030013349
:10A2D000DBB2012B80F860301AD9426990F8613006
:10A2E0001344187A02F09ABD70B5426903F0FF0575
:10A2F00090F8613013440446187A02F08FFDA36E83
:10A300005BB184F8385094F83900BDE870401847C4
:10A3100090F85F30002BE0D0704770BD0148FFF728
:10A32000CFBF00BFD090FF1F0148FFF7C9BF00BFDC
:10A330003C91FF1F2DE9F047374FDFF8E0903B6875
:10A34000026982B006460093DDF800800021A02556
:10A35000D3789B065BD53B680193019BC8EB030355
:10A360000F2BF5D949B1102BF2D000209070336932
:10A3700080229A7002B0BDE8F087726996F8613069
:10A3800013440521187A02F043FF726996F8613090
:10A390001344012193F812A0504602F039FF09241A
:10A3A0000021504602F020FF2B46013BFDD1012148
:10A3B000504602F019FF2B46013BFDD1013CEFD185
:10A3C000706996F8611001444FF4A0720C7A4B7BCF
:10A3D00009EBC4011B02496803F4E06343F0640322
:10A3E0000B6096F862300344997CDB7D09EBC10178
:10A3F0001B02496803F4E06343F064030B60013A15
:10A40000FDD13269D3789B064FF00101A3D401201E
:10A4100002B0BDE8F08700BF7C9FFF1FD03801006D
:10A42000F0B503691222DA700269937803F0200311
:10A4300085B004460D46002B5ED0B42393703C4992
:10A4400022690B680093009E05E00B680193019B55
:10A450009B1B042B42D8D37803F0200303F0FF00AA
:10A46000002BF2D094F85D30002B31D04FF0000E6D
:10A470004FF0020C04EB0E0393F83B3013710B68A2
:10A480000393039F206907E09B060DD50B68029399
:10A49000029BDB1B052B28D8C378DBB203F002023A
:10A4A00002F0FF06002AEFD080F803C02669F37897
:10A4B000DBB2DF0632462DD49F062BD5DB0731D425
:10A4C0000EF1010E94F85D305FFA8EFE7345D1D81F
:10A4D00000201DBB002384F85E3004E090702369E7
:10A4E00080229A70042005B0F0BD86702369802216
:10A4F00004209A7005B0F0BD03F0FF06FFF71AFFC5
:10A5000010B9042005B0F0BD236984F85F60B02263
:10A510009A7094E78023B3700420DAE726698023D9
:10A52000B370D7E7BEF1000F0CBF02200320F6E79F
:10A530007C9FFF1F2DE9F04106690025122780F856
:10A54000385080F83950F770D0F810C09CF802E00D
:10A550000EF0200E88B00446884615461E46BEF111
:10A56000000F49D0B4238CF80230784B21691A6867
:10A570000092DDF800E006E01A6801920198CEEB47
:10A580000000042830D8C87800F0200000F0FF0751
:10A590000028F1D04FEA480242F00102D2B20A711B
:10A5A0001A680292DDF808E0206906E01A68039252
:10A5B0000399CEEB010105292AD8C17801F00201E7
:10A5C00001F0FF070029F1D04FF0020C80F803C022
:10A5D0002269D17811F0110722D12DBB002E0CBFBA
:10A5E000A0238023937003E08F70236980229A70E8
:10A5F000384608B0BDE8F0810EF0FF07FFF79AFE7D
:10A600000028F5D0236984F85F70B0229A70ACE717
:10A6100087702369802238469A7008B0BDE8F081BF
:10A62000802393700027E3E7012D75D0A02191705E
:10A6300021690A79BE4667464FF0A80C1A68049251
:10A64000049805E01A680592059A121A052A4AD854
:10A65000CA7802F0020202F0FF08002AF2D0CF709E
:10A660002169CA78D2B212F0100F08465AD1920668
:10A6700058D5013DEDB2012D49D0BEF11F0F3BD998
:10A680000A79012DDAD11A680692069D05E01A684A
:10A690000792079A521B052A46D8C27802F0020296
:10A6A00002F0FF01002AF2D00223C3702269D3789E
:10A6B000DBB2D9063AD49B0634D5B023BEF11F0FC6
:10A6C00093703FD8226904EB0E0312791A760EF1CB
:10A6D000010E5FFA8EFE16B1236980229A7084F80B
:10A6E00039E0774684E781F80280236980229A70F6
:10A6F000774684F839E07BE704EB0E0291F804809A
:10A7000082F818800EF1010E5FFA8EFEB9E781F82B
:10A7100002C021690846B0E7A82191702069BE46B1
:10A720000279B0E7774663E78170DEE71021A02366
:10A73000D170013BFDD12269937803F0F70377468E
:10A74000937055E723691B79C5E700BF7C9FFF1F06
:10A750000148FFF71FBD00BFD090FF1F0148FFF762
:10A7600019BD00BF3C91FF1F704700BF38B5144CA6
:10A77000037801225B000546204684F83B3084F8CC
:10A780005E2084F85D20FFF78BFC20460021FFF758
:10A7900047FE0B4C2978012320461A46FFF7CAFED4
:10A7A0000128F6D194F8383094F839209A4205D926
:10A7B000E218013384F83830107E38BDFF2038BDF0
:10A7C000D090FF1F38B51B4C037801225B00054673
:10A7D000204684F83B3084F85E2084F85D20FFF743
:10A7E0005FFC20460021FFF71BFE124C2978204613
:10A7F00001230222FFF79EFE0228F6D194F83820AA
:10A8000094F839108A420FD2531CDBB2A018994237
:10A8100084F83830007E0AD9234402321B7E84F843
:10A82000382040EA032038BD4FF6FF7038BD40F4B1
:10A830007F4038BDD090FF1F0C2901D90020704700
:10A840000231490001F0FE01FFF7BCBF70B50C4CAE
:10A850000378164601255B00204684F83B3084F8D7
:10A860005E5084F85D50FFF71BFC31462046FFF731
:10A8700017FC29462046BDE87040FFF7D1BD00BF58
:10A88000D090FF1FF8B505460F46164641242146D5
:10A890003A462846FFF7DAFF611C0234C9B2324655
:10A8A0002846E4B2FFF7D2FF592CF0D1F8BD00BF23
:10A8B00038B504460D463548FFF706FC6322802173
:10A8C00020462570FFF7C2FF012002F0C9FC204698
:10A8D00000225E21FFF7BAFF20465D21FFF746FF09
:10A8E000242801D0002038BD204606220C21FFF785
:10A8F000C9FF204601222B21FFF7A8FF2046012295
:10A900002C21FFF7A3FF20460E222D21FFF79EFFEB
:10A91000204600222E21FFF799FF204601222F21F9
:10A92000FFF794FF204605223021FFF78FFF2046D6
:10A9300001223121FFF78AFF204600223221FFF752
:10A9400085FF204600223321FFF780FF20460022AA
:10A950003421FFF77BFF204600223521FFF776FFE9
:10A96000204600225B21FFF771FF204610225C2168
:10A97000FFF76CFF204620225D21FFF767FF20468E
:10A980008F225E21FFF762FF012038BDD090FF1FAC
:10A9900010B4047F4160022CC26002D010BC01F0F0
:10A9A000D7BB836810BC184790E80C00F0B41C6853
:10A9B00059682568164F174E29432160164D1749CF
:10A9C0001760D66015611160417A154A5C180A312A
:10A9D00094F8244053F8215002EBC40149680D60FB
:10A9E000017A5C1803EB8101247ECD6902EBC4017E
:10A9F00049680D60817A581803EB810390F83000A4
:10AA0000596B02EBC002F0BC53681960704700BF7D
:10AA100001401F00011000380110007800001F8065
:10AA2000D0380100704700BFF0B50C1EBDF81460AF
:10AA300034DBB0F906701919B942C4BF3B1B1BB215
:10AA4000002BA6461CDD002A1146B8BFD11D02F01E
:10AA50000705CC10826A012007FB04E1A840012E03
:10AA60000A44C0B21ED00CD3022E09D1013B12FA07
:10AA700083F3013A12F8011F41409A421170F9D153
:10AA8000F0BDC043013B12FA83F3C0B2013A12F8A1
:10AA9000011F014093421170F9D1F0BD23441BB254
:10AAA0000024C6E7013B12FA83F3013A12F8011FB2
:10AAB00001439A421170F9D1F0BD00BFF8B50D1EE7
:10AAC0000EDB14461F46064601F03AFBA84207DD9E
:10AAD000002C05DB304601F037FBA04201DCF8BD5D
:10AAE000F8BD304601F02AFB022853D003284BD092
:10AAF000012806D16540F3886C406540013B5D1B31
:10AB00002DB2012F03D02AD3022F14D0F8BD002C70
:10AB10002246B6F90630B06AB8BFE21D42F3CF0252
:10AB200002FB035504F00704435D012101FA04F41C
:10AB30001C434455F8BD002C2246B6F90630B06AD5
:10AB4000B8BFE21D42F3CF0202FB035504F0070435
:10AB5000435D012101FA04F45C404455F8BD002C2A
:10AB60002246B6F90630B06AB8BFE21D42F3CF0202
:10AB700002FB035504F00704435D012101FA04F4CC
:10AB800023EA04044455F8BD3389013B591B25468B
:10AB90000CB2B6E7F18832890139013A4D1B141B1A
:10ABA0002DB224B2ADE700BF2DE9F041079E9DF91B
:10ABB0001880089D04461F4600F0C0FF0D4B0E484C
:10ABC0000E4984F83380FF22002F08BF1F4684F807
:10ABD0002F20002384F8302084F8312084F832209C
:10ABE0002060A665E565676261652362A362204611
:10ABF000BDE8F081D090FF1F282E01000110013820
:10AC000010B50446806A034B236008B105F078FB59
:10AC1000204610BD282E0100F8B5436ADBB190F83C
:10AC20002C200125AA4083F83B2083F85E5083F84E
:10AC30005D500446406A03680E461B680021984731
:10AC4000606A036831461B6898472946606ABDE818
:10AC5000F840FFF7E5BBC26BC56C1368046A23EAD2
:10AC6000050313604CB122684FF00043D362516377
:10AC7000D36A002BFCDA936BF8BD836B466B082517
:10AC8000802410E03768426C3A4332601F68826C5F
:10AC90003A431A601A68876C013D22EA07024FEABC
:10ACA00054041A6007D02142ECD13268476C22EA82
:10ACB00007023260EAE7F8BD70B50446406A0D4607
:10ACC00000282BD0A16DFFF749FA002D20460CBFBC
:10ACD000A621A721FFF7A0FF606A20B1E16DBDE8C2
:10ACE0007040FFF73BBA216C226D0868236A02436B
:10ACF0000A6093B1DA7A82B1D00703D5224A996902
:10AD00001160DA7A910703D5204AD9691160DA7A9D
:10AD1000520702D51E4A1B6A136070BD236A002BBE
:10AD20002BD0D97A626DE1B172B6D97ACE0706D549
:10AD30001848D9680668314099610160D97A880756
:10AD400006D51548196906683140D9610160D97A7C
:10AD50004E0705D5114859690668314019620160EE
:10AD600062B61B68D968914207D00D4818600D493A
:10AD7000DA6042F0804018611960226C216D13681E
:10AD800023EA01031360A0E700E100E004E100E032
:10AD900008E100E080E100E084E100E088E100E01B
:10ADA00001403F0000003F80436A2DE9F041054625
:10ADB0000E469046002B3ED090F82C100124A14066
:10ADC00083F83B1083F85E4083F85D40406A036877
:10ADD00000211B6808F1FF379847FFB2B8F1000F58
:10ADE00023D03744A046013E686A16F8011F036865
:10ADF0001B6898470134B742E4B216D0202CF3D137
:10AE00000121686AFFF70CFB95F82C206B6A520051
:10AE100083F83B2083F85E8083F85D80686A03686E
:10AE200000211B6898470124DEE7686A0121BDE81C
:10AE3000F041FFF7F5BAC26BC16C136823EA010356
:10AE400006EB080413604FF00048A6420ED02B6AB0
:10AE500016F801EB63B11A68C2F82C80C2F834E02E
:10AE6000D36A002BFCDAA642936BF0D1BDE8F081E7
:10AE7000AB6BD5F834C008208021DCF800206F6C63
:10AE80001EEA010F14BF3A43BA43CCF800201A68F7
:10AE9000AF6C3A431A601A68AF6C013822EA0702B5
:10AEA0004FEA51011A60E8D1CFE700BF70B5044600
:10AEB000406A0D46002828D0A16DFFF74FF92046C3
:10AEC0002946FFF7A9FE606A20B1E16DBDE8704038
:10AED000FFF744B9216C226D0868236A02430A60B7
:10AEE00093B1DA7A82B1D00703D5234A9969116008
:10AEF000DA7A910703D5214AD9691160DA7A5207C3
:10AF000002D51F4A1B6A136070BD236A002B2BD029
:10AF1000D97A626DE1B172B6D97ACE0706D51948F1
:10AF2000D9680668314099610160D97A880706D5E9
:10AF30001548196906683140D9610160D97A4E0710
:10AF400005D512485969066831401962016062B638
:10AF50001B68D968914207D00D4818600D49DA6026
:10AF600042F0804018611960226C216D136823EA59
:10AF700001031360A3E700BF00E100E004E100E08B
:10AF800008E100E080E100E084E100E088E100E029
:10AF900001403F0000003F802DE9F041044686B0AB
:10AFA000806A9DF830801E460F461546B4F9083079
:10AFB000002800F04281DA1D48BF03F10E02B4F907
:10AFC0000630D21003FB02F2002105F0BDFCB4F9FB
:10AFD0000820202A00F39280B4F90610A34B012028
:10AFE000203A733902EBD27201EBD1714FF0200E8F
:10AFF000029073208DE8014042F34F0241F34F016C
:10B00000204600F051FE606A84F82D70002800F0A0
:10B010004D81002D40F08A80B4F90830202B14BFF8
:10B020003D253C2584F82C50B8F1000F40F0858078
:10B0300006B394F93300002818DBC0B2012102F0F6
:10B04000E7F8012194F8330002F0CEF8012002F075
:10B0500007F9002194F8330002F0C6F80A2002F044
:10B06000FFF8012194F8330002F0BEF8606A00286E
:10B0700000F08280A16DFFF771F804227C49204620
:10B08000FFF792FE217A0139C9B22046FFF7C4FDCD
:10B09000784904222046FFF787FE94F92D30012BD2
:10B0A00014BF142110212046FFF7B6FD0422724977
:10B0B0002046FFF779FEB4F90630802B00F092802D
:10B0C000602B00F0A680D9212046FFF7A5FD94F95A
:10B0D0002D30012B14BFF12122212046FFF79CFDCA
:10B0E000204606226549FFF75FFE606A50B3E16DB6
:10B0F000FFF734F8012006B0BDE8F081B4F906107E
:10B100005F4B0120403A52394FF0400E029002EB63
:10B11000D272522001EBD1718DE8014042F34F020F
:10B1200041F34F01204600F0BFFD6CE76DB284F89B
:10B130002C50B8F1000F3FF47BAFFEF7C5FF002E97
:10B1400094D076E7216C226D0868236A02430A6076
:10B1500073B1DA7A62B1D00703D54A4A99691160AE
:10B16000DA7A91077CD4520702D5474A1B6A1360EA
:10B17000012006B0BDE8F081236A002B2BD0D97ADC
:10B18000626DE1B172B6D97ACF0706D53F48D9686A
:10B190000568294099610160D97A8E0706D53C4837
:10B1A000196905682940D9610160D97A4D0705D52B
:10B1B00038485969056829401962016062B61B6800
:10B1C000D968914207D0344818603449DA6042F0B7
:10B1D000804018611960226C216D136823EA010315
:10B1E00013604AE7B4F90830202B00F08680402B2A
:10B1F0007FF469AF2A4920460322FFF7D5FD94F971
:10B200002D30012B14BFCF219F212046FFF704FDD5
:10B2100059E7B4F90830102B7FF455AF2149204687
:10B220000322FFF7C1FD94F92D30012B14BFAF218C
:10B2300010212046FFF7F0FC45E7DA1D48BF03F177
:10B240000E02B4F90630D21003FB02F2104605924A
:10B2500005F04EF8A06200283FF44DAF059AB3E622
:10B26000114AD9691160DA7A7DE700BF802E0100AA
:10B270006030010064300100683001006C30010072
:10B280007430010000E100E008E100E080E100E04E
:10B2900084E100E088E100E001403F0000003F80E1
:10B2A0007C2E01003433010004E100E0012194F818
:10B2B0003100244F01F0ACFF94F83200012101F07D
:10B2C000A7FF94F9312094F9323057F83220E26325
:10B2D00057F83330206A23640125E56425651A6830
:10B2E0002A431A6078B1B8F1000F3FF428AFFFF796
:10B2F0005BFB002E3FF4BAAE9BE6042212492046C7
:10B30000FFF752FDDFE6294694F82F0001F080FF99
:10B31000294694F8300001F07BFF94F92F2094F92E
:10B32000303057F83220626357F833306564A564D3
:10B330001A68A36322F001021A60002E3FF496AE51
:10B3400077E600BFD0380100782E0100B0F9082060
:10B35000D31D48BF02F10E03B0F90620806ADB104E
:10B3600002FB03F2002105F0EFBA00BFF0B500299F
:10B37000BDF814502EDBB0F90660B1422ADA002A7B
:10B3800059DBB0F9087014461C44BC42C4BFBB1A58
:10B390001BB2002B1EDDD2B2D408D0F828E016FB79
:10B3A000041112F00702DBB20EEB010421D0C2F14E
:10B3B0000807FAB2374F9342BF5C0CD2C3EB020CC2
:10B3C000FF2646FA0CF6012D07EA06073FD005D303
:10B3D000022D36D0F0BD012D39D030D21EF80160DB
:10B3E00026EA07070EF801709342F3D3B0F906106E
:10B3F0000C449A1AD2B2072A10D9022D36D0002D49
:10B4000014BFFF26002613462670083BB0F906102D
:10B41000DBB2072B0C44F7D802F00702002AD9D080
:10B420001D4B012D9B5C1DD017D3022DD2D122784C
:10B4300053402370F0BD13441BB20022A1E7022D3C
:10B4400025D11EF8016077400EF80170CCE71EF898
:10B45000016037430EF80170C6E7227822EA030341
:10B460002370F0BD227813432370F0BD114623787A
:10B47000DB4323700839B0F90630C9B207291C44F0
:10B48000F5D812F00702A5D0034B9B5CCFE73444FC
:10B49000AFE700BF182E0100082E010070B4C47D74
:10B4A000BDF80C50022C18D0032C1FD0012C0BD04F
:10B4B000002A03DBB0F90840944201DC70BC7047FD
:10B4C000039570BCFFF7B0BAC4880395013CA41A79
:10B4D0000A4621B270BCFFF749BF0689C488013E05
:10B4E000641AB21AE41A12B221B2E1E70489039590
:10B4F000E41A641A114622B270BCFFF737BF00BFCE
:10B5000070B4C57DBDF80C60022D1AD0032D12D089
:10B51000012D03D0039670BCFFF728BFC488E41A3E
:10B52000A41A0A4621B2002A03DBB0F9084094426B
:10B5300013DC70BC70470489013C641A114622B2C6
:10B54000F1E7C48805890396013CAD1AED1A621A29
:10B5500011B22AB270BCFFF709BF039670BCFFF7A7
:10B5600063BA00BF2DE9F8430446406A002863D05F
:10B57000A16DFEF7F3FD052274492046FFF714FC88
:10B58000A1790139C9B22046FFF746FBB4F908207A
:10B59000E588A66AD31D48BF02F10E03DB10626A7C
:10B5A00015FB03F51FFA85F8002A7BD094F82C30A0
:10B5B0000125AB4082F83B3082F85E5082F85D5046
:10B5C000606A036840211B6808F1FF379847BFB2E3
:10B5D000B8F1000F23D03744A846013E606A16F840
:10B5E000011F03681B6898470135B742EDB216D0BA
:10B5F000202DF3D10121606AFEF712FF94F82C2070
:10B60000636A520083F83B2083F85E8083F85D8094
:10B61000606A036840211B6898470125DEE7012125
:10B62000606AFEF7FDFE606A002800F08D80E16D23
:10B63000BDE8F843FEF792BD236A002B2BD0D97AE0
:10B64000626DE1B172B6D97ACE0706D54048D968A5
:10B650000568294099610160D97A8D0706D53D4872
:10B66000196905682940D9610160D97A480705D56B
:10B6700039485969056829401962016062B61B683A
:10B68000D968914207D0354818603549DA6042F0F0
:10B69000804018611960226C216D136823EA010350
:10B6A000136068E7E26BE36C1168276A0B4306EBF3
:10B6B000080913604FF0004E4E450DD016F801CB2F
:10B6C0002FB33A68C2F82CE0C2F834C0D36A002B1A
:10B6D000FCDA4E45936BF1D1226C236D11680B435C
:10B6E000136097B1FB7A83B1D90703D51D4BBA69B3
:10B6F0001A60FB7A9A0703D51B4BFA691A60FB7A2A
:10B700005B0702D5194B3A6A1A60BDE8F883A36B50
:10B71000D4F8348008208021D8F80020656C1CEA19
:10B72000010F14BF2A43AA43C8F800201A68A56C69
:10B730002A431A601A68A56C013822EA05024FEA0A
:10B7400051011A60E8D1B7E7276AC5E7102E01005A
:10B7500080E100E084E100E088E100E001403F009A
:10B7600000003F8000E100E004E100E008E100E0CB
:10B770002DE9F04F85B09946BDF93870BDF83CA071
:10B78000BB1AC1EB090B002BB8BF5B42BBF1000F2A
:10B79000B8BFCBF1000B5B450D46164600938046C3
:10B7A00048DC4D453A4633464CDC194613460A46BA
:10B7B000C5EB09019B1A89B2002B0CB2B8BF5B42E2
:10B7C00004EBD474BE42ACBF4FF0FF3201224D45B2
:10B7D000039102924FEA640429DC9BB201930DE0CD
:10B7E000D8F80070BF69B847019BE41AA3B21CB235
:10B7F0000135002C2DB211DBA94518DB009B5B4500
:10B800002A46534631464046EADCD8F800205346E3
:10B810009769294632464046B847E5E7029A1644FA
:10B82000039AA94502EB030436B224B2E6DA05B066
:10B83000BDE8F08F4A462B46B94635464D4517467A
:10B840001E46B2DD304629463E464D4607468946ED
:10B85000AEE700BF10B404682469A44610BC60477A
:10B8600030B40468BDF808500295A46BA44630BCFF
:10B87000604700BF30B40468BDF808500295E46B1F
:10B88000A44630BC604700BF70B40468BDF90C60CA
:10B89000BDF8105003960495246CA44670BC604714
:10B8A000704700BF10B582B0B0F90C20019101685B
:10B8B000009200220C6CB0F90A301146A04702B089
:10B8C00010BD00BF704700BF01F003010129C17521
:10B8D00006D0032904D0C28803894281838170473E
:10B8E0000289C38842818381704700BF2DE9F041FE
:10B8F0000568134E6F6986B0B7420446BDF83080C4
:10B9000010D1013B13441BB20093CDF804800B46C9
:10B91000AD6A2046A8472368DB6AB3420AD106B065
:10B92000BDE8F081059304920391B84703A9256807
:10B930000EC9E6E7204606B0BDE8F041184700BF53
:10B94000A1B800002DE9F0410568124E6F6986B07C
:10B95000B7420446BDF830800FD1013BCDF80480DA
:10B960000B4400921BB2AD6A2046A8472368DB6AED
:10B97000B3420AD106B0BDE8F08105930492039169
:10B98000B84703A925680EC9E7E7204606B0BDE819
:10B99000F0411847A1B800002DE9F04F0568DFF825
:10B9A00058B06F6985B05F450646BDF93890BDF85F
:10B9B0003CA00C46904615D11F19BC420CDACDF8BC
:10B9C00000A0214601342D6A4B464246304624B23F
:10B9D000A847BC423568F2DBEB6A5B4507D105B08E
:10B9E000BDE8F08F0393B8473568039BE4E7304622
:10B9F00005B0BDE8F04F1847A1B800002DE9F043AD
:10BA000087B099420546BDF93840BDF83C6025D065
:10BA1000A24212D00768DFF88080D7F81490C145A1
:10BA200032D18DE850002846BC6AA0472B68DB6AFB
:10BA3000434524D107B0BDE8F083994202DD0846B2
:10BA40001946034628680E96C46B01335B1A1BB275
:10BA50002846A44607B0BDE8F0436047A24202DD95
:10BA6000134622461C4628680E96631C846B9B1A5C
:10BA70001BB22846A44607B0BDE8F04360472846FD
:10BA800007B0BDE8F0431847059304920391C847F7
:10BA900003A92F680EC9C4E7A1B800002DE9F04F33
:10BAA000D0F800E0DFF89090DEF814B083B0CB451A
:10BAB0000446BDF93080BDF834A00D4617461E4639
:10BAC00031D1CDF800A0DEF824B0294633463A46FD
:10BAD0002046D8472368CDF800A008F1FF323A4449
:10BAE000D3F824B0294612B233462046D8472368FB
:10BAF000CDF800A02946D3F820B03A464346204668
:10BB0000D8472068CDF800A0711E29444346056A35
:10BB100009B23A462046A8472368DB6A4B4506D15E
:10BB200003B0BDE8F08FD847D4F800E0C9E720465D
:10BB300003B0BDE8F04F1847A1B80000F0B40024EE
:10BB400001264FF6FF75094F07600471C475C48163
:10BB500004824476C4618675067685824582C180FA
:10BB6000028141818281F0BC704700BF40330100F7
:10BB70002DE9F04F85B00668BDF84450BDF9388016
:10BB8000CDF8008004460195D6F848B00392BDF97F
:10BB90003C60BDF9407089469A46D84723680195B4
:10BBA000009742465146D3F8488020463346C04766
:10BBB0002068039B0E930F95856C4B463A463146A1
:10BBC0002046AC4605B0BDE8F04F60472DE9F04F88
:10BBD00087B01746BDF9404000912546E91D059301
:10BBE00044BF2B4603F10E010268BDF8486053695B
:10BBF0000294C91003912B49BDF9444001968B4230
:10BC0000824645D1002C3CDD029B3C445E1EB6B210
:10BC10004FF0000923B2049301364D46029B002BDE
:10BC200028DD059B002403EB090806E0EDB22B0696
:10BC300004F1010411D4A6421CD0A1B211F0070FE7
:10BC400023B24FEA4505F1D1002BB8BF0733DB1013
:10BC5000013418F803502B06EDD5009BD2F818B02C
:10BC600019443A4609B2019B5046D847A642DAF831
:10BC70000020E2D1039B01379944049B3FB2BB42B1
:10BC8000CCD1D36A074A934206D107B0BDE8F08F02
:10BC90009847DAF80020B5E7504607B0BDE8F04F06
:10BCA000184700BFA1B8000070B4BDF90C60BDF921
:10BCB0001050BDF8144003960495059470BCFFF72E
:10BCC00085BF00BF2DE9F04F93B090460591C16943
:10BCD0001090BDF870000790BDF874909DF878A0A2
:10BCE0000493002900F0CD800A7A0AC98946049994
:10BCF0008A1AD2B203EBC203BAF1010FDA780B92BF
:10BD000093F905201E8893F802B00F9293F906402C
:10BD100079D913B2099323B20C93109B1A68A94BDB
:10BD20001193194653698B4240F0A6800B9B002B60
:10BD300055D01FFA88F300210D93C8462344DDF83F
:10BD4000409006910E930F460C46BBF1000F3FD07A
:10BD5000BDF818100C9B03971FFA8AF0CB1813FB41
:10BD600000F304900E9801440D98034409B21BB2ED
:10BD70000A910893002505E00135EBB264009B456C
:10BD8000E4B222D9039B2B44590703D1731C18F842
:10BD900006409EB22306EFD5099BBDF81000E918B6
:10BDA00011FB00F10598BAF1010F0FFA8AF3014473
:10BDB0001CD0079801900093D26909B217464846F3
:10BDC000089AB847D9F80020D6E7039F5F44FFB22E
:10BDD000069B0B9901330693DBB29942B5D8D36A1F
:10BDE000119A934243D113B0BDE8F08F0F9B1918FD
:10BDF00093690A9A29441F4609B2079B4846B847E7
:10BE0000D9F80020B8E700230C93099385E70A9A34
:10BE10000D9B0132013B52B213F0FF030A920D93C6
:10BE20006FD1DDF81890079BDDF83C80DDF820A08D
:10BE30004B4517D0BAF1010F00F0C8800B9A109D46
:10BE4000CDF804900BEB8B014FEACB030A4400932F
:10BE50001146DEF81C405346424609B22846A04728
:10BE6000D5F800E0DEF82C30119A9342BBD0109840
:10BE700013B0BDE8F04F1847109D284698472A6830
:10BE800054E7109A0598B2F90A308342ABDDB2F953
:10BE90000C304345A7DD062313FB0A03002BA2DD6C
:10BEA00008EBCA03002B9EDD537E2BB9049BAF2BFE
:10BEB00002D90133DBB20493109BD3F800E0414B6D
:10BEC00011931A46DEF81430934240F08E801FFA28
:10BED00088F30E9308339BB2BDF814200593052315
:10BEE0000D9300230A93CDF83C800FFA8AF3DDF816
:10BEF0004080CDF818900B921FFA8AFBCDF820A055
:10BF000099460A9ABDF810000B9C0E9D0523194610
:10BF100011FB00232C481146C75C039702FB0B4220
:10BF200014FA81F312B21BB209920C932C462E46DE
:10BF30001CE0089B0999012B2AB24B4640462DD0A4
:10BF4000079F0197CDF80090DEF81CA0D047D8F8E5
:10BF500000E0039B5B0801340393059BA4B25D449E
:10BF60005E44A342ADB2B6B23FF451AF039BD807D3
:10BF7000DFD4079B069A9342EBD0089B012B16D087
:10BF8000069B0193CDF80090DEF81CA009994B4662
:10BF900032B24046D047D8F800E0DAE7DEF818A021
:10BFA000079B0C9922B2D047D8F800E0D1E7DEF821
:10BFB00018A00C991346404622B2D047D8F800E0AA
:10BFC000C7E700BFA1B80000903301000B99109D96
:10BFD000CDF800900531DEF8204009B24246082332
:10BFE0002846A047D5F800E03CE7109C204698473B
:10BFF000D4F800E06BE700BFF0B5C36985B0044634
:10C000002BB30A2968D00D294AD01A7A914247D316
:10C01000587A884244D35D688A1A05EBC205AA782B
:10C02000002A50D0E87800284DD0207E00283AD051
:10C0300095F905E0B4F90E00A67DB4F90A707244D2
:10C0400006FB0202BA4262DCB4F9102030E00A2991
:10C0500056D00D2924D0027E002A4BD0B0F90E0014
:10C06000A57DB4F90A60062212FB0502B2423EDD4C
:10C07000228AE38102EBC50212B218462282A78A05
:10C08000668A02950B468DE8C00001462046FFF700
:10C0900019FEA37DE28903EB430302EB4303E38133
:10C0A000012005B0F0BDA67DB4F90E00B4F9102052
:10C0B000B4F814E0678A02960B468DE8804001468A
:10C0C0002046FFF7FFFD2979E389A27D012001FBCE
:10C0D0000233E38105B0F0BD0022C2819A7A817DEE
:10C0E000038A01FB02330382012005B0F0BDB4F9DD
:10C0F0001020C4E7857DB4F91020B0F90E00BEE72A
:10C10000028A817DC38102EBC1030382C8E700205C
:10C11000E0819B7A228A03FB062212B22282C7E7C1
:10C12000C1810282704700BF002908BF01218175CB
:10C13000704700BF81824182704700BFC07D704759
:10C14000B0F90A00704700BFB0F90C00704700BF9B
:10C1500010B4EFF3108272B6437F33B9017F012927
:10C1600007D003290FD00123437702B962B610BC70
:10C170007047124C2168A1B1114943610B6883617A
:10C1800008605861EFE70F4C216881B10E494361A7
:10C190000B688361086058610C4B4FF08051196047
:10C1A000E1E7074B4161816120601860DBE7064BE6
:10C1B0004161816120601860EEE700BF689FFF1F4A
:10C1C000649FFF1F589FFF1F5C9FFF1F04ED00E04F
:10C1D00070B5EFF3108272B60C4C206880B10C4E33
:10C1E00000254369236073B19D6102B962B645774A
:10C1F00083689847EFF3108272B620680028F0D168
:10C2000002B962B670BD3360EFE700BF589FFF1FF1
:10C210005C9FFF1FFFF7DCBF184A30B41468002C86
:10C2200027D0036821688B420ED2CB1A002184608C
:10C23000C1602360E06010600223037530BC70476A
:10C2400011688B42144608D3A2685B1A0360002A67
:10C25000F6D18260C460A060EEE7D268C2608460FC
:10C26000E060C568CB1A0222A8602360027530BC6A
:10C2700070478460C4601060DEE700BF609FFF1FEE
:10C28000F8B5224E34682CB32368002B3AD1204FE6
:10C290001D4604E03468ECB12368002B32D1A3685A
:10C2A00003B1DD6020693360036825751B68BB42FC
:10C2B00021D1037F4560022BC46020D0FFF748FFE7
:10C2C0006368002BE6D023602046FFF7A5FF3468A3
:10C2D000002CE1D1EFF3108372B60E4A00211068F2
:10C2E000116003B962B628B18468FFF795FF204654
:10C2F0000028F9D1F8BD224600219847E0E783687D
:10C300009847DDE7013B2360E4E700BF609FFF1F24
:10C3100091A90000709FFF1F024A13680133136048
:10C32000FFF7AEBF7C9FFF1F704700BF0368F0B4EC
:10C33000FBB1002501249D60DC601B4C1A601C448D
:10C34000241104F144056A11032692009E60174FE0
:10C350000679174B47F8241002F1604202F561425A
:10C3600005F01F05012000FA05F5E6541560F0BC44
:10C370007047104C236843F40003236000BF0E4B4A
:10C380000E4DA4F58734A4F59E7401261E60234645
:10C3900004609C68002CD0D01033AB420360F8D10D
:10C3A000002303601846E2E7008FFCBFA891FF1F3F
:10C3B00044E400E03C8004400070034040710340CE
:10C3C0000168A9B10B4BF0B40B441B110A4E0B4F83
:10C3D0000B4D46F8237003F1440202F01F040123C1
:10C3E0005211A340002445F822308C600460F0BC58
:10C3F000704700BF008FFCBFA891FF1F29C300003A
:10C4000080E100E0024A034B012111601B681847DC
:10C410000C710340A891FF1F024A034B01211160D8
:10C420005B6818471C710340A891FF1F024A034B29
:10C43000012111609B6818472C710340A891FF1FD0
:10C44000024A034B01211160DB6818473C7103402D
:10C45000A891FF1FF8B50E4671B17AB10746144690
:10C4600000253B6816F8011B1B6838469847013CBD
:10C470000544F6D12846F8BD0846F8BD1046F8BD7B
:10C4800000B5064A036812885B6883B001A9ADF85D
:10C4900004200222984703B05DF804FB90380100A5
:10C4A000F0B507468BB0002A33D0012A08BF0A2214
:10C4B00051B3212400E0F4B2B1FBF2F502FB1511F7
:10C4C000C8B2092900F1300198BFC8B20AA988BFD3
:10C4D0003730214488BFC0B201F8240C661E2946BB
:10C4E000002DE8D133B1013CE4B20AAB23442D2244
:10C4F00003F8242C3B6801AA11195B683846C4F183
:10C50000220298470BB0F0BD30228DF8252021245F
:10C51000E8E70368C9B21B6898470BB0F0BD00BFDD
:10C520000029BABF49422D2300230A22FFF7B8BFD2
:10C53000374A384913681B06FCD40B6813F0800394
:10C54000F8D172B634490A78002A5FD0334A3448A9
:10C55000F0B4344C176806682568D4680C303E4443
:10C56000143200681268304F35442C442044024491
:10C57000C2F34E022D4E2E482E4D2F4C42F4004257
:10C580003A60376806682D682C4A24680C303E44AF
:10C59000006812682A4F35442C4420440244C2F3F8
:10C5A0004E02284E2848294D294C42F400423A6058
:10C5B000376806682D68274A24680C303E440068B6
:10C5C0001268254F35442C4420440244C2F34E02E5
:10C5D000224E2348234D244C42F400423A603768EF
:10C5E00006682D68214A24680C303E4400681268B1
:10C5F00035442C4420440244C2F34E021C4842F409
:10C60000004202600B7062B6F0BC704762B67047C1
:10C6100024B0034024B00B40759FFF1F38B0034087
:10C620003CB0034040B003402CB0034058B003403E
:10C630005CB0034060B0034064B003406CB00340A2
:10C6400030B0034038B00B403CB00B4040B00B4022
:10C6500044B00B404CB00B402CB00B4058B00B40DA
:10C660005CB00B4060B00B4064B00B406CB00B4052
:10C6700030B00B4030B42948294A2A4B2A4D602457
:10C68000E121047011701B78284C082B30D00A2B44
:10C690002748284937D00C2B0CBF35223D221223C6
:10C6A0002A60236002600B60234B24491B78244AD4
:10C6B000BBB101230B601360224B23491B78234A33
:10C6C000012B26D9042B0FD9082B1ED9102B94BF70
:10C6D000862387230B6013601D4B01221A7030BC28
:10C6E00070470B601360E7E784230B601360F3E788
:10C6F00000F58E200F490830012213232A602360A1
:10C7000002600B60D0E73922F7E785230B601360E6
:10C71000E2E780230B601360DEE700BF00400740C4
:10C7200001400740B891FF1F08B003400CB0034020
:10C7300008B00B400CB00B40789FFF1F20B00340A7
:10C7400020B00B40B991FF1F24B0034024B00B4030
:10C75000759FFF1F0C2830B417D91023984228BFAB
:10C7600018461C46104A114D1178181A8C42287030
:10C7700018D00F4913700B7823B10E490E4A0023CD
:10C780000B60136030BCFFF775BF0A2802D90C2379
:10C790001C46E7E7082802D90A231C46E2E70823DB
:10C7A0001C46DFE730BC7047B891FF1F749FFF1F26
:10C7B000759FFF1F24B0034024B00B4028282FD8BA
:10C7C000334B2DE9F0411E5CFF2E2BD0314B1B78F3
:10C7D000002B2AD132062CD472B62F4D2F4C2F4667
:10C7E000012326602B7062B672B623681B060CD438
:10C7F0003B781BB9F4E72B78002BF1D062B602F03E
:10C800009BF972B623681806F5D5254B1B680022E4
:10C810002A7062B6234A107843FA00F0BDE8F0812E
:10C82000002070470020BDE8F081FFF781FE32064E
:10C83000D2D572B61C4DDFF87C801C4C06F0400748
:10C84000FFB206F03F06D8F80030DFB123F0100346
:10C85000C8F8003001232660134A2B7062B672B606
:10C86000236819060CD413781BB9ECE72B78002B3E
:10C87000E9D062B602F060F972B623681B06F5D5FE
:10C880000B4BC3E743F01003C8F80030E2E700BFEA
:10C8900094380100759FFF1F779FFF1F00B0034072
:10C8A00010B00340749FFF1F769FFF1F00B00B4026
:10C8B00010B00B400CB00B400A4A0B49136843F40C
:10C8C000805313600B7843B9084BC0221A70084B91
:10C8D00080F30C0000B218807047044B80221A705D
:10C8E000F5E700BF2C800440789FFF1F21C00C405B
:10C8F00000C00C40F0B51B4B1B4E596818689A6875
:10C90000DB6885B06C460FC4337899071DD5174A8C
:10C91000174C1378174913F0700318BF1370164A99
:10C92000164B8027177000263320032226706D4691
:10C9300008701A7072B6043C45F001052046A847FD
:10C9400062B6237813F0700309D10D4B064901E05C
:10C95000013B02D00A78D207FAD505B0F0BD2370AA
:10C9600005B0F0BDC03801000100024000000240E7
:10C97000040002400B000240070002400A0002408F
:10C98000410D0300B0F5006F0AD210B5094B1B78BA
:10C99000DB07044606D504F1A0500078C0B210BDF4
:10C9A00000207047FFF7A6FF04F1A0500078C0B246
:10C9B00010BD00BF01000240B0F5006F17D238B5BE
:10C9C0000F4B1B78DA070D46044611D504F1A05031
:10C9D0000378AB420AD00B4A137813F0700318BFE8
:10C9E0001370074A05701378DB07FCD538BD704714
:10C9F000FFF780FF04F1A0500378AB42EBD1F5E7DD
:10CA0000010002400000024008B5F3F74DFEF5F7C3
:10CA100057FD02F091F8FAE7844641EA000313F06B
:10CA200003036DD1403A41D351F8043B40F8043B35
:10CA300051F8043B40F8043B51F8043B40F8043BF8
:10CA400051F8043B40F8043B51F8043B40F8043BE8
:10CA500051F8043B40F8043B51F8043B40F8043BD8
:10CA600051F8043B40F8043B51F8043B40F8043BC8
:10CA700051F8043B40F8043B51F8043B40F8043BB8
:10CA800051F8043B40F8043B51F8043B40F8043BA8
:10CA900051F8043B40F8043B51F8043B40F8043B98
:10CAA00051F8043B40F8043B403ABDD2303211D338
:10CAB00051F8043B40F8043B51F8043B40F8043B78
:10CAC00051F8043B40F8043B51F8043B40F8043B68
:10CAD000103AEDD20C3205D351F8043B40F8043B38
:10CAE000043AF9D2043208D0D2071CBF11F8013B36
:10CAF00000F8013B01D30B8803806046704700BFFC
:10CB0000082A13D38B078DD010F003038AD0C3F10A
:10CB10000403D21ADB071CBF11F8013B00F8013BEC
:10CB200080D331F8023B20F8023B7BE7043AD9D3AB
:10CB3000013A11F8013B00F8013BF9D20B78037080
:10CB40004B7843708B7883706046704708B5104C03
:10CB500008E0236859050DD423681A050FD423680B
:10CB6000DB0411D423685803F3D500F08DFE23684D
:10CB70005905F1D502F044F823681A05EFD502F003
:10CB8000D5F82368DB04EDD500F0F0FCEAE700BF40
:10CB90003480044008B5FFF7D9FF00BF014B1022D5
:10CBA0001A80704700200540704700BF094908B54A
:10CBB0000B6830B16A461844A2F58052904202D206
:10CBC0000860184608BD03F065FB0C2303604FF0B6
:10CBD000FF3008BDBC91FF1FFEE700BFEFF31380DD
:10CBE00070B9EFF310836BB9EFF305825AB94FF4C4
:10CBF0008070EFF311832BB1984228BF184670471D
:10CC00004FF0FF3070470F2A01D81846F1E7014B6B
:10CC1000D05CEEE7F0E300E0F0B44D1E2E460024B9
:10CC200000E00134B0FBF2F302FB1300092800F12D
:10CC300030078ABF3730F8B2C0B206F8010F184685
:10CC4000002BEED10A1953704CB1107815F8016F12
:10CC500028700133E01A834202F80169F5DB0846C7
:10CC6000F0BC7047704700BF10B40F4B53F8302032
:10CC700092F880422CB1012369B182F8803010BC57
:10CC8000704703EBC0035B681A6841B922F00202E7
:10CC90001A6010BC704782F8003110BC704742F037
:10CCA00003021A6010BC7047D03801001C4A02EB26
:10CCB000C00301295B6811D004291BD052F8300051
:10CCC000002280F8802229B1022920D0032922D015
:10CCD0001A6070474FF480721A60704752F8300043
:10CCE0004FF4A27280F880121A601A6822F02002B3
:10CCF0001A60704752F830104FF4A272012081F888
:10CD000080021A601A6842F020021A60704740F2EE
:10CD100003121A6070474FF481721A60704700BFA7
:10CD2000D0380100212848D8F8B5042A44D8DFE8D3
:10CD300002F0484B4E0345004FF410262B4B03EBFB
:10CD4000C0030D465C68216811F4E06148D0284BAF
:10CD5000284A2949C3F89C2104F140422748C3F8D6
:10CD6000A411A2F59221264FC3F8A0017C292548E1
:10CD7000C3F8A871C3F8AC012CD9A2F594237C2B7D
:10CD80002AD9A2F596237C2B28D9A2F598237C2BAF
:10CD900029D9A2F59A227C2A27D81B4872B6236883
:10CDA00023F4702343F08072C4F38401164323609C
:10CDB00040F82150266062B6F8BD70474FF4302627
:10CDC000BCE74FF40026B9E74FF44026B6E74FF42E
:10CDD0002026B3E70D48E1E70D48DFE70D48DDE722
:10CDE000FFF764FFB3E70C48D8E7F8BDD03801007F
:10CDF0000082FF1FF188FF1F9988FF1FC588FF1F52
:10CE00006D88FF1F4188FF1F9892FF1FC091FF1F71
:10CE1000F891FF1F4892FF1F7892FF1F1A4B03EBF8
:10CE2000C00010B4426802F14043A3F592217C296E
:10CE300023D9A3F594217C290DD9A3F596217C292A
:10CE40001FD9A3F598217C2919D9A3F59A237C2B06
:10CE500011D80E4C00E00E4C72B613680D4823F04A
:10CE60008773C2F3840123F4803343F0807313602B
:10CE700044F8210062B610BC7047074CECE7074C41
:10CE8000EAE7074CE8E700BFD03801009892FF1F9F
:10CE9000F891FF1F65CC0000C091FF1F7892FF1F23
:10CEA0004892FF1F30B4054B054D064C002210215F
:10CEB0001A602A602060196030BC704714D00340AB
:10CEC00004D0034000D00340282838B52ED00029D4
:10CED00004464FDD5F4B1B78012505FA03F28A42B9
:10CEE00002D8212837D938BD0338C2B2012A3AD92D
:10CEF000202C4AD0192C48D0574A126802FB011244
:10CF000022FA03F31D2800F29B80DFE800F0928BE9
:10CF1000847D9999766F9999999999999999996830
:10CF2000615A53994C99999999999945494B1B780C
:10CF30000B2B08D90C2B1CBF0C3B19410846BDE834
:10CF40003840FFF7B9BCC3F10C0399400846BDE86F
:10CF50003840FFF7B1BC2946FFF786FE2946BDE8F9
:10CF60003840FFF7A3BE3D4A126802FB011222FAC5
:10CF700003F3C7E72128B6D80021FFF775FE204646
:10CF80000121BDE83840FFF791BE354A126802FB27
:10CF9000011222FA03F3B5E73249334A0B604FF42A
:10CFA0005173136038BD3149314A0B604FF45173EE
:10CFB000136038BD2F49304A0B6040F24443136080
:10CFC00038BD2E492E4A0B6040F24443136038BDF1
:10CFD0002C492D4A0B6040F24443136038BD2B4965
:10CFE0002B4A0B6040F24443136038BD29492A4A5A
:10CFF0000B6040F24443136038BD2849284A0B6057
:10D0000040F24443136038BD2649274A0B6040F282
:10D010004443136038BD2549254A0B6040F2444320
:10D02000136038BD2349244A0B604FF451731360D9
:10D0300038BD2249224A0B604FF45173136038BD4A
:10D04000212C3FF650AF7F29D4BF0021012120467B
:10D0500093E700BFA092FF1F0880034008900340A1
:10D0600008800B4010800B4048A0044018800B4003
:10D070004CA004401880034008B0044010800340D6
:10D0800004B004404080034018C00440388003408E
:10D0900014C004402880034010B0044020800340A6
:10D0A0000CB004403080034010C00440488003406E
:10D0B0001CC004401890034034900440109003407A
:10D0C0003090044038B1102828BF1020044AC3B261
:10D0D000107813707047024A01231078137070475C
:10D0E000A092FF1F2DE9F8430E4680463249334D8A
:10D0F000304603F055F847F6122300281ABF1D46A4
:10D100004FF002094FF00109002425FA04F002F063
:10D1100051FE4FF05E51074602F0A4FE0146304634
:10D1200003F052F830B90134072CEED1E80902F0CF
:10D1300041FE07463146384602F048FF4FF07C5129
:10D1400002F086FD03F07AF84FF6FF729042A8F1E4
:10D15000030328BF1046012B29D9B8F1170F17D8A0
:10D16000174B23FA08F303F0010383F0010223B9FC
:10D17000B8F1190F0FD0BDE8F883124B124D1349C7
:10D180001A6044EAC9042A6008601C60BDE8F8839C
:10D19000B8F1200FECD10E4B0E4D0F49002244EA9E
:10D1A000C9041A602A6008601C60BDE8F8830B4B54
:10D1B0000B4D0C49F2E700BF001BB740006CDC02CE
:10D1C0006006F000008003400480034008800340B4
:10D1D00000800B4004800B4008800B40009003400F
:10D1E0000490034008900340212801D8FFF73CBD7C
:10D1F000704700BF212806D8044B53F8303093F80D
:10D200000002C0B270470020704700BFD038010054
:10D21000212801D8FFF74ABD704700BF72B60C49FC
:10D220000C4B0D4A1B680868126862B6520102D5A1
:10D23000322B88BF01300949C3F5BB334FF47A72F2
:10D24000FF33A1FB031302FB00F000EB93107047C8
:10D250007C9FFF1F18E000E004ED00E0ABAAAAAA43
:10D260002DE9F843054672B6204F214B214A1B6831
:10D270003C68126862B6520102D5322B88BF013475
:10D2800095B3C3F5BB331C4EDFF86490DFF86480C0
:10D29000FF334FF47A72A6FB031302FB04F404EB92
:10D2A000931472B6D9F800103A68D8F800E062B664
:10D2B000C1F5BB33FF33A6FB03031EF0806FC4EB45
:10D2C00093134FF47A7002D0322988BF013200FBE9
:10D2D0000233B3F57A7F04D3013D05D004F57A74A7
:10D2E000DFE701F029FCDCE7BDE8F8837C9FFF1F46
:10D2F00018E000E004ED00E0ABAAAAAAF8B52D4BB7
:10D300002D49DFF8D0E0DFF8D0C02C4E2C4D2D4C4D
:10D310002D4A2E4F4FF4000018604FF080701860B7
:10D320004FF0007018604FF0806018604FF00060A0
:10D3300018600020086028234BF6FF71CCF800101D
:10D34000CEF80030336013602B6023603B60B36223
:10D350009362092245F8242CC4F8D80F05F57F659F
:10D36000C7F8D41F07F5FF2707F5FA67C6F8F83F97
:10D370002B6006F5FF26C4F8D42F05F5FD2504F52E
:10D38000FF24386006F2F4761148316005F5FF6538
:10D3900004F5FD642B6023600260FFF76BF9192030
:10D3A000FFF75EFF00F0B6FF40F21310BDE8F84053
:10D3B000FFF756BF08E100E00480034014800340FB
:10D3C000248003402C8003401C80034034800340B1
:10D3D00000800B400C800340088003402DE9F84F8B
:10D3E000214B1B6807460BB101221A70DFF88890A9
:10D3F0001E4D99F80040DFF884801D4E0134272C23
:10D400008ABF4FF0000A5FFA84FA5446AB462B7885
:10D41000A34216D1FFF7E2FB40281FDC33791B063D
:10D42000F5D59BF800300133272B86BF0022134629
:10D43000DAB218F80330DBB2F3712A702B78A3420A
:10D44000E8D00C490A4BFFB208F804700120AC2266
:10D45000087089F800A0DA70BDE8F88FFF28D6DDE3
:10D4600001F06AFBD3E700BFF49FFF1FF19FFF1F8E
:10D4700000C00640F09FFF1FF89FFF1F889FFF1FFF
:10D480001C4BDFF894C01A681B49F0B542F4805277
:10D490001A4D1A60DFF884E0194F1A4E1A4C002317
:10D4A0008CF800304FF451722B701F2840F2133566
:10D4B0008EF800303B70337025600A6012D8194630
:10D4C0000124124A124D11701248547000212C2769
:10D4D000402693724FF4003491701174D7702E70FF
:10D4E0000460F0BDC0F34431C0F3471400F01F03E3
:10D4F000E7E700BF348004400CC00440859FFF1F55
:10D50000F19FFF1FF09FFF1F08C0044000C00640AE
:10D5100031E400E004E100E0849FFF1FF89FFF1F5B
:10D52000034B1B68DB0401D5FFF758BF704700BFF2
:10D530003480044010B5044C237823B101F0FCFA88
:10D540002378002BFAD110BDF09FFF1F054A064B30
:10D5500010781B78C0B2DBB2984238BF4030C01A96
:10D56000704700BF849FFF1F859FFF1F30B42B4B68
:10D570001A7994061FD52A48DA79037829490133A4
:10D580003F2B0978C8BF00238B42D2B203D0264C70
:10D59000D9B2E2540170254A116861B1244A127867
:10D5A000D2B2934236BFC2F140029B1A9B18272B7E
:10D5B000C4BF01230B70194AD378DBB2180611D40B
:10D5C0005A060DD5154B1B795B0609D5194B1A491F
:10D5D0001B6800220A7003B11A70104B2C22DA70FB
:10D5E00030BC704711790906EAD5144910480C7807
:10D5F0000178C9B28C420DD04A1C272A84BF002171
:10D600000A460F4D054C98BFD1B2AA5CD2B2E27166
:10D610000170D5E76C21D170D2E700BF00C0064091
:10D62000849FFF1F859FFF1FB09FFF1F809FFF1FCD
:10D63000F19FFF1FF49FFF1FF09FFF1FF89FFF1F29
:10D64000889FFF1F21282FD8184B195CFF292BD04A
:10D65000174B184ADFF870C003EBC000F0B5436801
:10D66000DFF868E0144F154D154E00241C60DEF8FD
:10D670000030012043F020038840CEF800301460D1
:10D680004FF4A07338602E60C2F800C0013BFDD19A
:10D6900013689B05FCD42023013BFDD1094B09B243
:10D6A00033F8110080B2F0BD00207047E03901006E
:10D6B000D038010000500440085004400450044099
:10D6C000000002030051044080014A0038800440F9
:10D6D000431E032B14D872B60A4951F8230068B1CF
:10D6E00070B4094C058834F81320466841F823606B
:10D6F000521B24F8132062B670BC704762B67047A4
:10D700000020704754A0FF1F98A2FF1F0138032874
:10D710000BD872B6074B53F8203043B100205B683A
:10D720000130002BFBD162B67047002070471846CD
:10D73000F9E700BFA8A0FF1F30B472B62B4A1378D8
:10D740001D0706D52A4B196A002936D0996A002987
:10D7500041D053781C0706D5254B196C00293ED0C3
:10D76000996C002939D09378190705D5204B196E8B
:10D77000002936D0996E89B1D3781B0707D51C4B89
:10D78000D3F880207AB3D3F8882011213AB162B659
:10D79000184B00221A7030BC00F04ABE0D21154C07
:10D7A000154D227843F8315003EBC1030830013A9C
:10D7B0005860227062B630BC704704220D4C0F4D89
:10D7C000217843F8325003EBC20308304A1E5860F8
:10D7D000227062B6EFE70521E1E70921DFE70822C1
:10D7E000ECE70C22EAE71022E8E700BF043A010068
:10D7F0000080FF1FD1A0FF1FC8004000880040002C
:10D80000431E032B1DD81B4A400140F0100030B4CA
:10D81000104472B6184CE25C032A1BD8DFE802F011
:10D820000212151703220D88E25410F0080F14BFDE
:10D83000C823882343EA054308310360416062B688
:10D8400030BC704708300222EDE70522EBE70830D4
:10D850000422E8E7094A52F8230038B1084A52F88E
:10D860002300416042F8231062B6E9E742F8231032
:10D87000034AF7E70080FF1FE0A0FF1FA8A0FF1FDB
:10D88000B8A0FF1F00BE70472DE9F04FDFF818B3B6
:10D89000DFF818A387B044E0AD4F4FEA930807EBD9
:10D8A000C809013ED9F8042003F00803F6B2A2F13A
:10D8B000080003F0FF04002B40F0018157F83830D6
:10D8C0001B0C99B222F8081C002B00F0EF80A14B32
:10D8D00022F8064C42F8044C53F82620002A00F0A7
:10D8E000CF819D4D55F8263058609C4C45F8260058
:10D8F00034F81630194424F8161000F079FD002889
:10D9000000F0C281964A974B19F0080F00F1080009
:10D9100018BF1346C9F8040047F8383008238BF8BD
:10D9200000309BF80040E4B265071CD58E4B1B7895
:10D93000B3B18E490A7802F0FF0322B1013BDBB29A
:10D940000B7003B900BE8A490A7802F0FF032AB1BE
:10D95000013BDBB20B70002B00F0688100F066FE2B
:10D9600004238BF8003004F0080303F0FF02002BBF
:10D9700000F0C9809AF80030DBB21E098CD19A08F9
:10D98000DFF8CC9159F8321009EBC200C1F38301E2
:10D99000013940680C2900F28580DFE801F07A7ACD
:10D9A0008383838383834683838307000168714D68
:10D9B0004068714F714E6860296088B240F28161A1
:10D9C0000024674B49F832304FF0010E88423C602A
:10D9D000C9F81040C9F8184086F800E05C4A00F227
:10D9E000E780B0F5D06F80F01B82B0F5817F00F04A
:10D9F000D98100F26981802800F02A82822840F0D3
:10DA0000D781A98801F07F01042900F2D1815C4807
:10DA10005C4A890008441470547001788C0740F106
:10DA2000608382F800E0022173E1534F3A682AB321
:10DA3000554B524E554819883478057840298E4602
:10DA400045F0020828BF4FF0400E002C84F001047E
:10DA50003470CEEB01010CBF8824C82409EBC80642
:10DA600089B285F0010544EA0E447260198049F8D4
:10DA7000384072440570002965D03A603D4B1A88E1
:10DA8000B2F5A06F0ED100219A785970404B1A70F0
:10DA900008E038493F4C0D68A54200F098803049B5
:10DAA00049F832103C4A0123137037E72C4A2D4BBA
:10DAB00019F0080F18BF134647F838302EE700F06A
:10DAC000B7FC364A364952F82630002B00F0E38086
:10DAD00058688C5D42F8260003F10802C9F804205A
:10DAE000032C05D8DFE804F02C02292602228A55EF
:10DAF0001A8819F0080F0CBF8823C82343EA024391
:10DB000047F838300AE7E00700F19380210600F17A
:10DB1000D180A20706D5234A234913780220DBB21D
:10DB200013700870E30602D51F4B10221A7007B05D
:10DB3000BDE8F08F04228A55DAE705228A55D7E737
:10DB400003228A55D4E7BEF1400F18BF002294E7A4
:10DB50000080FF1F54A0FF1F00A0FF1F98A2FF1FFF
:10DB6000C800400088004000DCA0FF1F65A0FF1F28
:10DB700050A1FF1FC8A0FF1FFC9FFF1F64A0FF1F35
:10DB8000C0200740D4A0FF1F10A0FF1FD0A0FF1F80
:10DB9000982007402109000394200740A8A0FF1FF8
:10DBA000E0A0FF1F8820074080200740902007400A
:10DBB000B0F5106F00F07C8140F2A38040F6211296
:10DBC000904240F07B82A54A012313706AE74C68BB
:10DBD000A3498C427FF463AF0178A9297FF45FAF3A
:10DBE000417845297FF45BAF8178C2297FF457AF34
:10DBF000C1786B297FF453AF9A489B4E01783478F3
:10DC000081F00105002C41F0020105700CBF882055
:10DC1000C82084F0010449F8310009EBC1019348A0
:10DC20003470002505244D60047038E700F064FF6F
:10DC300094E68F4B89488B491A614FF0020E80F8A9
:10DC400000E08C4F0A708C49196099608B4E8C4DA6
:10DC50008C4C9A610D213970FF213170DFF84CE254
:10DC600029702270884D894A8EF800109F27012460
:10DC700006F8047C5D600470DA6007B0BDE8F08FE0
:10DC800043F82600824D30E6824A47F83800137880
:10DC90000133137042E68B5D032B00F2BA8001A2C0
:10DCA00052F823F01DD900001DD90000FDDC000052
:10DCB000F7DC00006F49724B80220D2008701A704B
:10DCC000A2077FF52FAF26E740F20232904240F0E4
:10DCD000ED81AA8802F07F02042A69D86D88002DA0
:10DCE00066D16449CDF804E0920011440A7842F00C
:10DCF00002020A70C1E101238B550FE600238B5508
:10DD00000CE6B0F5086F53D16349644A0978117085
:10DD10007146ED888D4280F0E88252480478402DAB
:10DD2000AE4644F0020C28BF4FF0400E02EB0E034B
:10DD300009EBCC01029301234A604FEA0E48CEEB77
:10DD4000050101930025C82242EA080384F001027C
:10DD500049F83C3035700270DFF814C1424BDFF8EF
:10DD6000048149BBBEF1400F7FF42DAF42F0020C9D
:10DD700009EBCC03029ADFF8F8E05A608DBB0D0482
:10DD800045F088059DF804304EF83C500A44337045
:10DD90000470134640297FF416AF0021404A3B60CF
:10DDA000118010E7AA8802F07F02042A40F28B81DA
:10DDB000304A0F23137006E74029D7D942F00202F8
:10DDC0000CEBC200029E4660BDB19DF80450354880
:10DDD0001D703346403988F8004040334CF832001B
:10DDE000DCE79DF8043033700D04029B047045F0AD
:10DDF000C8050B444EF83C50CCE79DF804501D700C
:10DE0000029B1D4888F80040403940334CF83200EE
:10DE1000C4E719F0080F0CBF022303238B557DE5DF
:10DE200021494A68002AC3D06C88B5F804E003E0B1
:10DE30000C314A68002ABBD00B88A342F8D14B882A
:10DE40007345F5D1240A032C0CBF1178098960E7CA
:10DE5000124A0221147054705BE700BF94200740FF
:10DE600001000400D0A0FF1F64A0FF1F65A0FF1FDA
:10DE70000080FF1FC0200740880040008820074026
:10DE8000802007409820074014A0FF1F68A0FF1FB4
:10DE900000A0FF1FD1A0FF1FDCA0FF1FD4A0FF1F09
:10DEA00010A0FF1FC8004000083A01008C20074066
:10DEB000B248116AAC7804700C0600F19881D9F868
:10DEC0002820AF49100600F1DB81D9F83020AC4999
:10DED000120600F1D081D9F83820A949130600F1C3
:10DEE000C581D9F84020A649150600F1BA81D9F8B4
:10DEF0004820A349140600F1AF81D9F85020A04969
:10DF0000100600F1A481D9F858209D49120600F1AD
:10DF10009981D9F860209A49130600F18E81D9F8C9
:10DF200068209749150600F18381D9F8702094493B
:10DF3000140600F17881D9F878209149100600F193
:10DF40006D81D9F880208E49120600F16181D9F8DF
:10DF500088208B49130600F15581D9F89020884913
:10DF6000150600F14981D9F898208549140600F179
:10DF7000FF808448844A854901908548854D864CB8
:10DF8000049700230596029580460F4616461D46C7
:10DF90000394306828B1446800F04AFA2046002C07
:10DFA000F9D100233360029B38681A46002342F8F7
:10DFB000253028B1446800F03BFA2046002CF9D106
:10DFC00000223A60019A98F800301146002241F888
:10DFD000042B039A0191023B4FF0000122F8151027
:10DFE000032B07D8DFE803F05D025D024FF0010369
:10DFF00088F800300135042D06F1040607F1040706
:10E0000008F10108C5D1654C654D2278654B049F28
:10E01000059E0021100729701A7000F19280624954
:10E0200062780A700021C9F83010C9F83810110759
:10E03000DFF84C816ED4A2785C49DFF844810A7025
:10E0400000211207C9F85010C9F858104BD4E278D3
:10E0500057494B4C0A7013074FF00001C9F8701074
:10E06000C9F8781000F1AE8033780193002283F074
:10E070000105C9F89020C9F898200021029188462E
:10E080008E460A464B48047844F0020C09EBCC0358
:10E090000393019B002B039B5A600CBF8822C8226C
:10E0A00052E64FF0000388F80030A3E7B0F5A06F08
:10E0B0007FF47EAE012300250193DEE740F62122A6
:10E0C0009042F7D074E66D88002D7FF471AE3A4926
:10E0D000CDF804E0920011440A7822F002020A709E
:10E0E000CBE7022115E600F083F9002800F0EB8071
:10E0F0000830324AC8F86400C8F8602000F078F9A7
:10E10000002800F0DA8008302D4AC9F86C00C9F800
:10E1100068209CE700F06CF9002800F0E0800830EF
:10E12000264AC8F84400C8F8402000F061F90028E9
:10E1300000F0CF800830224AC9F84C00C9F84820C6
:10E1400079E700F055F9002800F0A58008301B4A57
:10E15000C9F82400C9F8202000F04AF9002800F08E
:10E1600094800830164AC9F82C00C9F8282056E7D0
:10E17000D1F89C00083800F05BF9FAE6DCA0FF1F3C
:10E180000080FF1FB8A0FF1F54A0FF1FA8A0FF1F03
:10E19000E0A0FF1F00A0FF1F98A2FF1F043A01008C
:10E1A000D1A0FF1FC4200740C8200740CC20074053
:10E1B000D0200740D0A0FF1FC020074088004000AB
:10E1C000C800400000F014F9002870D008304F4A11
:10E1D000C4F88400C4F8802000F00AF9002860D058
:10E1E00008304B4AC9F88C00C9F888203CE7506ACF
:10E1F000083800F01DF962E6D1F89400083800F004
:10E2000017F9B0E6D1F88C00083800F011F9A4E64F
:10E21000D1F88400083800F00BF998E6C86F083888
:10E2200000F006F98DE6486F083800F001F982E643
:10E23000C86E083800F0FCF877E6486E083800F041
:10E24000F7F86CE6C86D083800F0F2F861E6486D42
:10E25000083800F0EDF856E6C86C083800F0E8F829
:10E260004BE6486C083800F0E3F840E6C86B083825
:10E2700000F0DEF835E6486B083800F0D9F82AE6F9
:10E28000C86A083800F0D4F81FE62A78C9F82800D0
:10E2900001322A70C3E62A78C9F8200001322A70B8
:10E2A0005AE72A78C9F8880001322A70DCE62A7811
:10E2B000C4F8800001322A708EE72A78C9F8680015
:10E2C00001322A70C3E62A78C8F8600001322A7049
:10E2D00014E72A78C9F8480001322A70ABE62A7898
:10E2E000C8F8400001322A701FE740298E4628BF37
:10E2F0004FF0400E02EB0E0302930123CEEB01011F
:10E300004FEA0E4800250193BCE600BF880040009C
:10E31000C8004000F8B500F08FFD294B29482A4C71
:10E320002A4F2B4DDFF8BCC0DFF8BCE0294E00229D
:10E330001A605A609A60DA601A615A619A61DA6109
:10E340001A625A629A62DA621A635A639A63DA63E9
:10E350001A645A649A64DA641A655A659A65DA65C9
:10E360001A665A669A66DA661A675A679A67DA67A9
:10E37000C3F880200168C3F8842041F48021016043
:10E38000C3F307212170C3F30740134938701B0EF4
:10E390002B70FF238CF80030104D8EF800301048A1
:10E3A0000B700123337084F8642070264FF40074DE
:10E3B000102207F82C3C2E70046081F8F820F8BD7C
:10E3C0000080FF1F348004409C200740B02007409D
:10E3D000B4200740942007401020074049E400E0A3
:10E3E00008E100E08020074088200740704700BF18
:10E3F00072B60D480268B2FA82F30F2B10DC4FF0B0
:10E400000041D94022EA0102026062B6074803EBEC
:10E41000C303DB00C2180021C15010465160704791
:10E4200062B60020704700BFA492FF1FBC83FF1F8D
:10E430000D4B0E4AC31AA2FB03231B090F2B0CD84A
:10E440000B4A127852B972B60A484FF0004102687E
:10E4500021FA03F31A43026062B67047064A127843
:10E46000002AF0D0FFF768B9BC83FF1F398EE3386C
:10E47000D1A0FF1FA492FF1FDCA0FF1F38B50E4BD9
:10E480000E4C1B68218805468BB1B1F5917F05D2F2
:10E490000B4A4B1C55549BB2238038BD00220848C0
:10E4A00098470021064A55540123238038BDB1F511
:10E4B000917FEDD338BD00BF08A1FF1FA2A2FF1FAF
:10E4C000A8A2FF1F2DE9F843214E224F31680123F6
:10E4D00080463B70B1B1204D4B8801EB8302013384
:10E4E00000240F2BC2F808802C7004D84B80002326
:10E4F0003B70BDE8F88340230B800320FFF780F9D1
:10E500003460F4E7DFF8549099F80030002BF0D035
:10E51000114D45F6215408E0013C12D02B7883B907
:10E5200000F00AFB99F800307BB10320FFF7EEF80A
:10E530000528F1D8FFF75CFF014630600028EBD0DA
:10E54000CAE701232B70BDE8F883BDE8F88300BF5C
:10E5500024A1FF1FF8A0FF1F28A1FF1FDCA0FF1FA1
:10E560001201F8B5D5B2A1B3012943D043780446CE
:10E5700000781B0643EA004040F4704045F0040672
:10E580008F1E3043FFF79EFF022F04F1020314D9C0
:10E59000053414F8023C14F8032C14F8010C1B0485
:10E5A00043EA0223334343EA0060033FFFF78AFF55
:10E5B000022F234604F10304EBD8022F23D0012FAE
:10E5C0000DD045F4774040F00500BDE8F840FFF776
:10E5D00079BF14482843BDE8F840FFF773BF1878A7
:10E5E00045F4770545F0060545EA0020BDE8F8400A
:10E5F000FFF768BF03780C4845EA03452843BDE8A8
:10E60000F840FFF75FBF1A78587845F0774545F036
:10E61000070545EA022545EA0040BDE8F840FFF756
:10E6200051BF00BF06F0F70007F000F738B5084B00
:10E630001C7824B9074D296809B14B8803B938BD46
:10E640009B000B800320FFF7DBF82C6038BD00BF78
:10E65000F8A0FF1F24A1FF1F2DE9F041AD4E336844
:10E660000746002B00F092801D885A88910803EB22
:10E6700081010432AA428C6842D25A8004F00F060B
:10E680004FEA1428A449A6F1080208F00F00C4F3C9
:10E690000313062A00F101050B701AD9B31E012BD2
:10E6A0005FFA88F04ED9052E48D0042E00F0A481E0
:10E6B000731F022B7FD90F2E0ED1F72842D8F028D6
:10E6C00002D0964B1B883BB1FFF7D8FE0020BDE877
:10E6D000F08127B1BD4202D00020BDE8F081082EB4
:10E6E000C4F3033300F08780092E11D00A2E40F0C6
:10E6F00094800A2BF0D18A4B8A4A1B68A02181E0C2
:10E700001846FFF795FE0420FEF7E2FF3060B5E7FC
:10E71000092BE1D1270E00F07B81834B814A1B68D6
:10E720009021C4F307461170EDB2FCB2002B00F04B
:10E730009D80224631462846984797E0F02843D9E5
:10E74000F72841D0F1380E28C6D801A353F820F09D
:10E7500007E90000EBE80000D9E80000D9E6000076
:10E76000D9E60000CBE80000D9E60000ABE90000E4
:10E77000D9E6000075E900008FE90000B3E8000069
:10E78000D9E600009BE800007FE80000674B1B789B
:10E79000002BA1D00420FEF79BFF03463060002829
:10E7A0009AD00588002D7FF460AFFFF741FE3560F9
:10E7B0002846BDE8F081FFF761FEC4F30740FFF78C
:10E7C0005DFE072E02D1200EFFF758FE534B584A2C
:10E7D000198858481468584D524A017000270E0A8B
:10E7E000F0201F802E7010700CB301225348A047F8
:10E7F0000120BDE8F081082B7FF46EAF504B494AF1
:10E800001B688021C4F307461170EDB2240E6BB370
:10E81000284622463146984728E00B2E11D10B2B73
:10E820007FF45AAF474B3F4A1B68B021EAE7464B9B
:10E830001B68002B00F0FB80404898470120BDE892
:10E84000F0810C2E40F000810C2B7FF445AF3F4B44
:10E85000344A1B68C0211170EDB2C4F30746002B87
:10E8600000F0C88028463146240E98473849314A7E
:10E87000314B0D7016701C700120BDE8F081354BD6
:10E880001B68002B00F0D6809847C4F30746254B41
:10E89000EDB2240E83F80080E8E72F4B1B68002BB5
:10E8A000F2D12E4B1B68A3B1FE209847C4F3074654
:10E8B000EDE72B4B1B68002BE6D1284B1B6843B1BF
:10E8C000FC209847C4F30746E1E7264B1B68002B62
:10E8D000DAD1C4F30746DAE7234B1B68C4F30746D3
:10E8E000002BD4D030469847D1E7204B1A68002A35
:10E8F000EFD0260C630C06F07F0003F47E53184320
:10E90000F6B29047C3E71A4B1B68C4F30746002BC7
:10E91000E8D1BCE730A1FF1FA6A2FF1FA2A2FF1FE4
:10E920000CA1FF1FA0A2FF1F40A1FF1FDCA0FF1F23
:10E9300008A1FF1FA4A2FF1FA5A2FF1FA8A2FF1FDF
:10E9400038A1FF1F3CA1FF1F20A1FF1FFCA0FF1F3C
:10E95000A7A2FF1FE8A0FF1FECA0FF1FF0A0FF1F52
:10E960002CA1FF1F1CA1FF1F34A1FF1F04A1FF1F2B
:10E9700018A1FF1F3F4B1B68002B85D13E4B1B6826
:10E98000002BA6D0FA209847C4F307467FE73B4BFD
:10E990001B68002B7FF478AF374B1B68002B98D097
:10E9A000FB209847C4F3074671E7354B1B68002BE3
:10E9B0007FF46AAF304B1B68002B8AD0F820984751
:10E9C000C4F3074663E70E2B7FF486AE2D4A2E4B29
:10E9D0001268E0211970002A47D0260C610C06F05D
:10E9E0007F0301F47E511943EDB2A1F50051284691
:10E9F0009047F6B2240E39E7FFF740FDC4F3074015
:10EA0000FFF73CFD200EFFF739FD0020BDE8F08147
:10EA10001E4B1D4A1B6880211170EDB2C4F30746DE
:10EA200083B1314628463A4698473C461EE70120C6
:10EA3000BDE8F081104B1B68002B3FF44AAFFF206C
:10EA4000984746E71C4611E70D2EBCD10D2B7FF4ED
:10EA500043AE0F4B0C4A1B68D0211170EDB2C4F3CA
:10EA60000746002B7FF4FEAEC4E7C4F30746EDB2C1
:10EA7000240EFBE614A1FF1FF0A0FF1FF4A0FF1F50
:10EA8000E4A0FF1F00A1FF1FA0A2FF1F38A1FF1FCE
:10EA900010A1FF1F38B5164D2868E0B101884488E1
:10EAA000A14213DD03191B7A83B104F10803C218D4
:10EAB0000C1B002302E012F8011F21B10133A34215
:10EAC000F9D1204638BD1C46204638BDFFF7B0FCC2
:10EAD0000020286038BD074B1B780BB9002038BDDB
:10EAE0000220FEF7F5FD28600028D7D1F6E700BF29
:10EAF0004CA1FF1FDCA0FF1F0D4B1B78BBB910B54D
:10EB00000C4C216803F0FF024B883F2B07DC0733D6
:10EB10000B4401F1470003F8012F8342FBD140234E
:10EB20000B800120FEF76CFE0023236010BD7047B0
:10EB300044A1FF1F48A1FF1F38B5224C237803B121
:10EB400038BD01232370FFF7A5FF70BB00F048F824
:10EB500040BB00F0DBF810BBFEF7F8FCE0B9002387
:10EB60002370EFF30583002BEAD1EFF3108172B627
:10EB7000154B1868E0B1154C2278CAB945691D607B
:10EB800001232370C5B1AA6101B962B6002545779A
:10EB9000836898472570D3E700F020F8DFE700F09E
:10EBA0001BF8D9E700F016F8D3E7FFF71FFCCDE715
:10EBB0000029C5D162B638BD054B1D600029E5D1DD
:10EBC000E3E700BF51A1FF1F689FFF1F6C9FFF1F5E
:10EBD000649FFF1F704700BF704700BF704700BFB2
:10EBE000054A064B10781B78C0B2DBB2984238BF9A
:10EBF0004030C01A704700BF58A1FF1F59A1FF1F26
:10EC0000F0B4384B1A7912F0300F2CD072B6997DCF
:10EC100001F0FF0200293DD062B6334F3349387806
:10EC20000D78334E1C46C0B2EDB2431C402BE17947
:10EC300028BF0023AB4202F1FF32C9B21CBFF1541E
:10EC4000184612F0FF02F0D12A4B1B68C2B23A708C
:10EC50004BB1A84236BFC5F14005401B40192728DB
:10EC6000C4BF01221A701F49CA78D2B2150616D441
:10EC700052060DD51B4B1B795B0609D51E4B1F4950
:10EC80001B6800220A7003B11A70164B3C22DA701E
:10EC9000F0BC70474022D9795A7462B6E3E70B7929
:10ECA0001C06E5D5164B174E1C783378E4B2DBB260
:10ECB0009C420ED0144D01E0A3420AD00133402BF8
:10ECC00028BF00230879E85CC0B2C871087D072816
:10ECD000F2D9DBB2034933700B79180644BF7C23A9
:10ECE000CB70C5E700A0064058A1FF1F59A1FF1F28
:10ECF0009CA1FF1F54A1FF1FE0A1FF1FDCA1FF1F6C
:10ED0000E4A1FF1FDDA1FF1F5CA1FF1F054A064B09
:10ED100010781B78C0B2DBB2984238BF4030C01ABE
:10ED2000704700BF58A2FF1FEDA1FF1FF0B4384B82
:10ED30001A7912F0300F2CD072B6997D01F0FF02D3
:10ED400000293DD062B6334F334938780D78334EC1
:10ED50001C46C0B2EDB2431C402BE17928BF002312
:10ED6000AB4202F1FF32C9B21CBFF154184612F097
:10ED7000FF02F0D12A4B1B68C2B23A704BB1A842D5
:10ED800036BFC5F14005401B40192728C4BF0122EA
:10ED90001A701F49CA78D2B2150616D452060DD57C
:10EDA0001B4B1B795B0609D51E4B1F491B680022B4
:10EDB0000A7003B11A70164B3C22DA70F0BC70472F
:10EDC0004022D9795A7462B6E3E70B791C06E5D57F
:10EDD000164B174E1C783378E4B2DBB29C420ED04F
:10EDE000144D01E0A3420AD00133282B28BF002391
:10EDF0000879E85CC0B2C871087D0728F2D9DBB297
:10EE0000034933700B79180644BF7C23CB70C5E7E8
:10EE100000B0064058A2FF1FEDA1FF1F18A2FF1F60
:10EE2000E8A1FF1F5CA2FF1FECA1FF1F60A2FF1F54
:10EE300059A2FF1FF0A1FF1F70B584B072B6194B25
:10EE4000194D1A48702241260F2480211A702E7005
:10EE50001A460470197013781B06FCD5144B1868F9
:10EE600062B6144B144C984298BF00EB800001A985
:10EE700098BF40000A22FDF7CFFE01A920460023DB
:10EE800011F8012B01333AB10A2B20F8022FF7D1E8
:10EE90001623237004B070BD5B00DBB2237004B096
:10EEA00070BD00BF000002400700024006000240A3
:10EEB000080002407F9698007093FF1FFFFFFFFF3E
:10EEC0002DE9F043DFF8EC808BB006460F4600F0EA
:10EED00073F898F90030013304460D4637D03046B8
:10EEE000394600F0DFF9002831D02BA3D3E9002305
:10EEF0003046394600F026FE814668BB28A3D3E998
:10EF000000233046394600F0FFFD00B398F9003089
:10EF1000254ACDF82090042400200021022BCDE9C1
:10EF20000467CDE9026700940192CDE906012CD077
:10EF3000684600F0BDF940B3089B1BB101F0AAF987
:10EF4000089B0360DDE906010BB0BDE8F0832046B5
:10EF500029460BB0BDE8F083134A98F900300192BE
:10EF600003210022CDE90467CDE9026700910892F0
:10EF70002BB90E4B4FF06042CDE90623D8E70C4980
:10EF80000020022BCDE90601D2D101F083F9222322
:10EF90000360D1E7AFF30080EF39FAFE422E8640DE
:10EFA00051302DD5104987C0743A0100FFFFEF475B
:10EFB0000000F07F8693FF1F2DE9F04FB04F21F046
:10EFC0000042BA4283B00C464FEAD17605460DD9CD
:10EFD000AC4FBA4225D9C1F31303034340F0EF808D
:10EFE0000EB10020014603B0BDE8F08FA64B9A4257
:10EFF00000F2CC80A54B9A4200F2DE808AA3D3E9CE
:10F00000002300F05DF90022A14B00F09BFD0028D9
:10F0100000F005812846214600229D4B00F050F962
:10F02000E1E783A3D3E9002300F08CFD002840F042
:10F03000CB802846214680A3D3E9002300F064FD5D
:10F040000028CED1934B284603EBC60821467CA36B
:10F05000D3E9002300F0E6FAD8E9002300F030F904
:10F0600000F07AFD804600F077FA77A3D3E9002319
:10F0700006460F4600F0D6FA02460B4628462146C1
:10F0800000F01CF972A3D3E90023CDE9000130465A
:10F09000394600F0C7FA82468B4652465B46DDE9A8
:10F0A000000100F00BF905460C462A462346284687
:10F0B000214600F0B7FA68A3D3E9002306460F46BD
:10F0C00000F0B0FA66A3D3E9002300F0F7F8324667
:10F0D0003B4600F0A7FA64A3D3E9002300F0F0F860
:10F0E00032463B4600F09EFA61A3D3E9002300F0CC
:10F0F000E5F832463B4600F095FA5FA3D3E90023DA
:10F1000000F0DEF832463B4600F08CFA02460B4631
:10F110002846214600F0D2F806460F4628462146EA
:10F1200032463B46B8F1000F56D000F07BFA32462B
:10F1300004460D463B4600204FF0804100F0BEF8EB
:10F1400002460B462046294600F096FB02460B4637
:10F150005046594600F0B2F8DDE9002300F0AEF861
:10F160000B4602464A49002000F0A8F86FF47F736E
:10F1700098454FDA08F57A7801EB085100224FF0F4
:10F18000B87300F04FFA03B0BDE8F08F424B9A42DB
:10F190003FF658AF414BF4002344D3E9002300F07D
:10F1A0008DF83F4BC6F101081C44CDE90001D4E9BC
:10F1B00000ABC6EB080870E74FF0000875E70246A1
:10F1C0000B4600F07DF80EE717A3D3E900231046A5
:10F1D000194600F027FA06E700F024FA00228046DC
:10F1E00089464FF080433046394600F067F80246C2
:10F1F0000B464046494600F03FFB2A46234600F0B6
:10F200005DF802460B460020214900F057F803B094
:10F21000BDE8F08F01EB085103B0BDE8F08F8046E8
:10F2200043E700BFAFF300809C7500883CE4377E65
:10F23000EF39FAFE422E864051302DD5104987C055
:10F24000FE822B654715F73F0000E0FE422EE63FA9
:10F25000763C7935EF39EA3DD0A4BE726937663E17
:10F26000F16BD2C541BDBB3E2CDE25AF6A56113FC6
:10F2700093BDBE166CC1663F3E5555555555C53FAD
:10F28000412E8640FFFFEF7F422ED63FFFFF2F3EED
:10F290000000F03F783A0100B1A2F03F983A010037
:10F2A000883A010041F0004101F58010C00F70471D
:10F2B0000020704781F0004102E000BF83F000436E
:10F2C00030B54FEA41044FEA430594EA050F08BF01
:10F2D00090EA020F1FBF54EA000C55EA020C7FEAC5
:10F2E000645C7FEA655C00F0E2804FEA5454D4EB42
:10F2F0005555B8BF6D420CDD2C4480EA020281EA0C
:10F30000030382EA000083EA010180EA020281EA43
:10F310000303362D88BF30BD11F0004F4FEA013195
:10F320004FF4801C4CEA113102D0404261EB4101A4
:10F3300013F0004F4FEA03334CEA133302D052422A
:10F3400063EB430394EA050F00F0A780A4F10104E6
:10F35000D5F1200E0DDB02FA0EFC22FA05F2801820
:10F3600041F1000103FA0EF2801843FA05F3594106
:10F370000EE0A5F120050EF1200E012A03FA0EFC85
:10F3800028BF4CF0020C43FA05F3C01851EBE371AF
:10F3900001F0004507D54FF0000EDCF1000C7EEBCC
:10F3A00000006EEB0101B1F5801F1BD3B1F5001F0A
:10F3B0000CD349085FEA30004FEA3C0C04F1010429
:10F3C0004FEA445212F5800F80F09A80BCF1004F52
:10F3D00008BF5FEA500C50F1000041EB045141EAD4
:10F3E000050130BD5FEA4C0C404141EB010111F4D5
:10F3F000801FA4F10104E9D191F0000F04BF014680
:10F400000020B1FA81F308BF2033A3F10B03B3F15D
:10F4100020020CDA0C3208DD02F1140CC2F10C02ED
:10F4200001FA0CF021FA02F10CE002F11402D8BF4B
:10F43000C2F1200C01FA02F120FA0CFCDCBF41EA17
:10F440000C019040E41AA2BF01EB0451294330BDE6
:10F450006FEA04041F3C1CDA0C340EDC04F11404C3
:10F46000C4F1200220FA04F001FA02F340EA03009A
:10F4700021FA04F345EA030130BDC4F10C04C4F1E0
:10F48000200220FA02F001FA04F340EA03002946C0
:10F4900030BD21FA04F0294630BD94F0000F83F40A
:10F4A000801306BF81F480110134013D4EE77FEAED
:10F4B000645C18BF7FEA655C29D094EA050F08BF39
:10F4C00090EA020F05D054EA000C04BF194610461A
:10F4D00030BD91EA030F1EBF0021002030BD5FEA5E
:10F4E000545C05D14000494128BF41F0004130BD86
:10F4F00014F580043CBF01F5801130BD01F00045DA
:10F5000045F0FE4141F470014FF0000030BD7FEA4C
:10F51000645C1ABF194610467FEA655C1CBF0B4647
:10F52000024650EA013406BF52EA033591EA030F5E
:10F5300041F4002130BD00BF90F0000F04BF002156
:10F54000704730B54FF4806404F132044FF0000589
:10F550004FF0000150E700BF90F0000F04BF002102
:10F56000704730B54FF4806404F1320410F0004568
:10F5700048BF40424FF000013EE700BF42004FEA63
:10F58000E2014FEA31014FEA02701FBF12F07F43E0
:10F5900093F07F4F81F06051704792F0000F14BFDD
:10F5A00093F07F4F704730B54FF4607401F0004521
:10F5B00021F0004120E700BF50EA010208BF704778
:10F5C00030B54FF000050AE050EA010208BF70476D
:10F5D00030B511F0004502D5404261EB41014FF4D6
:10F5E000806404F132045FEA915C3FF4DCAE4FF0DA
:10F5F00003025FEADC0C18BF03325FEADC0C18BFC1
:10F60000033202EBDC02C2F1200300FA03FC20FA11
:10F6100002F001FA03FE40EA0E0021FA02F114445E
:10F62000C1E600BF70B54FF0FF0C4CF4E06C1CEA73
:10F6300011541DBF1CEA135594EA0C0F95EA0C0FE8
:10F6400000F0DEF82C4481EA030621EA4C5123EA5B
:10F650004C5350EA013518BF52EA033541F480118A
:10F6600043F4801338D0A0FB02CE4FF00005E1FB3D
:10F6700002E506F00042E0FB03E54FF00006E1FB87
:10F6800003569CF0000F18BF4EF0010EA4F1FF04CA
:10F69000B6F5007F64F5407404D25FEA4E0E6D410A
:10F6A00046EB060642EAC62141EA55514FEAC5201B
:10F6B00040EA5E504FEACE2EB4F1FD0C88BFBCF597
:10F6C000E06F1ED8BEF1004F08BF5FEA500E50F148
:10F6D000000041EB045170BD06F0004646EA01010E
:10F6E00040EA020081EA0301B4EB5C04C2BFD4EB40
:10F6F0000C0541EA045170BD41F480114FF0000E39
:10F70000013C00F3AB8014F1360FDEBF002001F0A6
:10F71000004170BDC4F10004203C35DA0C341BDC20
:10F7200004F11404C4F1200500FA05F320FA04F0F2
:10F7300001FA05F240EA020001F0004221F0004126
:10F7400010EBD37021FA04F642EB06015EEA430E99
:10F7500008BF20EAD37070BDC4F10C04C4F12005C9
:10F7600000FA04F320FA05F001FA04F240EA02007C
:10F7700001F0004110EBD37041F100015EEA430E4D
:10F7800008BF20EAD37070BDC4F1200500FA05F26D
:10F790004EEA020E20FA04F301FA05F243EA0203EC
:10F7A00021FA04F001F0004121FA04F220EA0200FB
:10F7B00000EBD3705EEA430E08BF20EAD37070BD41
:10F7C00094F0000F0FD101F00046400041EB010121
:10F7D00011F4801F08BF013CF7D041EA060195F003
:10F7E000000F18BF704703F00046520043EB0303BD
:10F7F00013F4801F08BF013DF7D043EA06037047AA
:10F8000094EA0C0F0CEA135518BF95EA0C0F0CD0B4
:10F8100050EA410618BF52EA4306D1D181EA0301FA
:10F8200001F000414FF0000070BD50EA410606BFF4
:10F830001046194652EA430619D094EA0C0F02D139
:10F8400050EA013613D195EA0C0F05D152EA03367E
:10F850001CBF104619460AD181EA030101F000419C
:10F8600041F0FE4141F470014FF0000070BD41F0E5
:10F87000FE4141F4780170BD70B54FF0FF0C4CF4BF
:10F88000E06C1CEA11541DBF1CEA135594EA0C0FDE
:10F8900095EA0C0F00F0A7F8A4EB050481EA030E2B
:10F8A00052EA03354FEA013100F088804FEA033312
:10F8B0004FF0805545EA131343EA12634FEA0222E0
:10F8C00045EA111545EA10654FEA00260EF00041A1
:10F8D0009D4208BF964244F1FD0404F5407402D2F3
:10F8E0005B084FEA3202B61A65EB03055B084FEA84
:10F8F00032024FF480104FF4002CB6EB020E75EB81
:10F90000030E22BFB61A754640EA0C005B084FEAA8
:10F910003202B6EB020E75EB030E22BFB61A754625
:10F9200040EA5C005B084FEA3202B6EB020E75EB70
:10F93000030E22BFB61A754640EA9C005B084FEAE8
:10F940003202B6EB020E75EB030E22BFB61A7546F5
:10F9500040EADC0055EA060E18D04FEA051545EAE4
:10F9600016754FEA06164FEAC30343EA52734FEA8D
:10F97000C2025FEA1C1CC0D111F4801F0BD141EA06
:10F9800000014FF000004FF0004CB6E711F4801F6B
:10F9900004BF01430020B4F1FD0C88BFBCF5E06F4B
:10F9A0003FF6AFAEB5EB030C04BFB6EB020C5FEA5B
:10F9B000500C50F1000041EB045170BD0EF0004EB0
:10F9C0004EEA113114EB5C04C2BFD4EB0C0541EAE2
:10F9D000045170BD41F480114FF0000E013C90E6DF
:10F9E00045EA060E8DE60CEA135594EA0C0F08BFA3
:10F9F00095EA0C0F3FF43BAF94EA0C0F0AD150EAA2
:10FA000001347FF434AF95EA0C0F7FF425AF104634
:10FA100019462CE795EA0C0F06D152EA03353FF45C
:10FA2000FDAE1046194622E750EA410618BF52EAD9
:10FA300043067FF4C5AE50EA41047FF40DAF52EAAD
:10FA400043057FF4EBAE12E74FF0FF3C06E000BF4A
:10FA50004FF0010C02E000BF4FF0010C4DF804CD57
:10FA60004FEA410C7FEA6C5C4FEA430C18BF7FEA17
:10FA70006C5C1BD001B050EA410C0CBF52EA430C45
:10FA800091EA030F02BF90EA020F0020704710F1C5
:10FA9000000F91EA030F58BF994208BF90422CBF54
:10FAA000D8176FEAE37040F0010070474FEA410C4D
:10FAB0007FEA6C5C02D150EA013C07D14FEA430C6B
:10FAC0007FEA6C5CD6D152EA033CD3D05DF8040BDC
:10FAD000704700BF8446104662468C46194663460E
:10FAE00000E000BF01B5FFF7B7FF002848BF10F1E5
:10FAF000000F01BD4DF808EDFFF7F4FF0CBF01202A
:10FB000000205DF808FB00BF4DF808EDFFF7EAFFA5
:10FB100034BF012000205DF808FB00BF4DF808ED60
:10FB2000FFF7E0FF94BF012000205DF808FB00BF55
:10FB30004DF808EDFFF7CEFF94BF012000205DF8DF
:10FB400008FB00BF4DF808EDFFF7C4FF34BF0120EC
:10FB500000205DF808FB00BF4FEA410212F50012D9
:10FB600015D211D56FF47873B3EB625212D94FEA04
:10FB7000C12343F0004343EA505311F0004F23FAEE
:10FB800002F018BF404270474FF00000704750EA43
:10FB9000013005D111F0004008BF6FF00040704700
:10FBA0004FF00000704700BF4FEA4102B2F1E0435E
:10FBB00024BFB3F5001CDCF1FE5C0DD901F0004C54
:10FBC0004FEAC0024CEA5070B2F1004F40EB8300A4
:10FBD00008BF20F00100704711F0804F21D113F1D0
:10FBE0003872BCBF01F00040704741F480114FEA09
:10FBF0005252C2F11802C2F1200C10FA0CF320FA92
:10FC000002F018BF40F001004FEAC1234FEAD323AE
:10FC100003FA0CFC40EA0C0023FA02F34FEA430318
:10FC2000CCE77FEA625307D150EA01331EBF4FF0A1
:10FC3000FE4040F44000704701F0004040F0FE40BC
:10FC400040F40000704700BF80F0004002E000BFB9
:10FC500081F0004142001FBF5FEA410392EA030FB7
:10FC60007FEA226C7FEA236C6AD04FEA1262D2EB01
:10FC70001363C1BFD218414048404140B8BF5B4206
:10FC8000192B88BF704710F0004F40F4000020F09F
:10FC90007F4018BF404211F0004F41F4000121F0B5
:10FCA0007F4118BF494292EA030F3FD0A2F10102FF
:10FCB00041FA03FC10EB0C00C3F1200301FA03F13D
:10FCC00000F0004302D5494260EB4000B0F5000F60
:10FCD00013D3B0F1807F06D340084FEA310102F11F
:10FCE0000102FE2A51D2B1F1004F40EBC25008BFD1
:10FCF00020F0010040EA03007047490040EB00009B
:10FD000010F4000FA2F10102EDD1B0FA80FCACF1C9
:10FD1000080CB2EB0C0200FA0CF0AABF00EBC250C8
:10FD200052421843BCBFD0401843704792F0000FB6
:10FD300081F4000106BF80F400000132013BB5E709
:10FD40004FEA41037FEA226C18BF7FEA236C21D07F
:10FD500092EA030F04D092F0000F08BF08467047E4
:10FD600090EA010F1CBF0020704712F07F4F04D1B2
:10FD7000400028BF40F00040704712F100723CBFC5
:10FD800000F50000704700F0004343F0FE4040F4EF
:10FD9000000070477FEA226216BF08467FEA2363AD
:10FDA0000146420206BF5FEA412390EA010F40F498
:10FDB000800070474FF0000304E000BF10F00043E4
:10FDC00048BF40425FEA000C08BF704743F09643CB
:10FDD00001464FF000001CE050EA010208BF7047E6
:10FDE0004FF000030AE000BF50EA010208BF70476D
:10FDF00011F0004302D5404261EB41015FEA010C82
:10FE000002BF84460146002043F0B64308BFA3F179
:10FE10008053A3F50003BCFA8CF2083AA3EBC2535B
:10FE200010DB01FA02FC634400FA02FCC2F120027A
:10FE3000BCF1004F20FA02F243EB020008BF20F0B1
:10FE40000100704702F1200201FA02FCC2F1200217
:10FE500050EA4C0021FA02F243EB020008BF20EA0C
:10FE6000DC7070474FF0FF0C1CEAD0521EBF1CEA3A
:10FE7000D15392EA0C0F93EA0C0F6FD01A4480EA28
:10FE8000010C400218BF5FEA41211ED04FF0006311
:10FE900043EA501043EA5111A0FB01310CF000403D
:10FEA000B1F5000F3EBF490041EAD3715B0040EA63
:10FEB000010062F17F02FD2A1DD8B3F1004F40EB33
:10FEC000C25008BF20F00100704790F0000F0CF006
:10FED000004C08BF49024CEA502040EA51207F3ACA
:10FEE000C2BFD2F1FF0340EAC250704740F40000A5
:10FEF0004FF00003013A5DDC12F1190FDCBF00F096
:10FF000000407047C2F10002410021FA02F1C2F143
:10FF1000200200FA02FC5FEA310040F1000053EADF
:10FF20004C0308BF20EADC70704792F0000F00F02D
:10FF3000004C02BF400010F4000F013AF9D040EA33
:10FF40000C0093F0000F01F0004C02BF490011F4C7
:10FF5000000F013BF9D041EA0C018FE70CEAD153C5
:10FF600092EA0C0F18BF93EA0C0F0AD030F0004C45
:10FF700018BF31F0004CD8D180EA010000F00040F9
:10FF8000704790F0000F17BF90F0004F084691F0B7
:10FF9000000F91F0004F14D092EA0C0F01D14202F1
:10FFA0000FD193EA0C0F03D14B0218BF084608D1BA
:10FFB00080EA010000F0004040F0FE4040F4000004
:10FFC000704740F0FE4040F4400070474FF0FF0C97
:10FFD0001CEAD0521EBF1CEAD15392EA0C0F93EADE
:10FFE0000C0F69D0A2EB030280EA010C49024FEA30
:10FFF000402037D04FF0805343EA111143EA1013E9
:020000021000EC
:100000000CF000408B4238BF5B0042F17D024FF4A0
:10001000000C8B4224BF5B1A40EA0C00B3EB510F7B
:1000200024BFA3EB510340EA5C00B3EB910F24BF64
:10003000A3EB910340EA9C00B3EBD10F24BFA3EBE9
:10004000D10340EADC001B0118BF5FEA1C1CE0D1B1
:10005000FD2A3FF650AF8B4240EBC25008BF20F064
:10006000010070470CF0004C4CEA50207F32C2BFB8
:10007000D2F1FF0340EAC250704740F400004FF055
:100080000003013A37E792F0000F00F0004C02BF86
:10009000400010F4000F013AF9D040EA0C0093F050
:1000A000000F01F0004C02BF490011F4000F013BAA
:1000B000F9D041EA0C0195E70CEAD15392EA0C0F12
:1000C00008D142027FF47DAF93EA0C0F7FF470AF4A
:1000D000084676E793EA0C0F04D14B023FF44CAF8D
:1000E00008466EE730F0004C18BF31F0004CCAD122
:1000F00030F000427FF45CAF31F000437FF43CAF5E
:100100005FE700BF4FF0FF3C06E000BF4FF0010C7F
:1001100002E000BF4FF0010C4DF804CD4FEA400261
:100120004FEA41037FEA226C18BF7FEA236C11D0AB
:1001300001B052EA530C18BF90EA010F58BFB2EB5E
:10014000030088BFC81738BF6FEAE17018BF40F0DE
:10015000010070477FEA226C02D15FEA402C05D192
:100160007FEA236CE4D15FEA412CE1D05DF8040B17
:10017000704700BF844608466146FFE70FB5FFF7AA
:10018000C9FF002848BF10F1000F0FBD4DF808ED62
:10019000FFF7F4FF0CBF012000205DF808FB00BF53
:1001A0004DF808EDFFF7EAFF34BF012000205DF8AD
:1001B00008FB00BF4DF808EDFFF7E0FF94BF0120FA
:1001C00000205DF808FB00BF4DF808EDFFF7D2FFF7
:1001D00094BF012000205DF808FB00BF4DF808ED3A
:1001E000FFF7C8FF34BF012000205DF808FB00BF07
:1001F0004FEA4002B2F1FE4F0FD34FF09E03B3EB34
:1002000012620DD94FEA002343F0004310F0004F73
:1002100023FA02F018BF404270474FF000007047C9
:1002200012F1610F01D1420205D110F0004008BF68
:100230006FF0004070474FF00000704742000ED250
:10024000B2F1FE4F0BD34FF09E03B3EB126209D411
:100250004FEA002343F0004323FA02F070474FF0C7
:100260000000704712F1610F01D1420202D14FF03C
:10027000FF3070474FF00000704700BF0B4601464B
:10028000184600F001B800BF13460A460146022096
:1002900000F0A8BE014B1868704700BFB097FF1F61
:1002A00070B50F4E0F4D761BB61018BF002405D049
:1002B000013455F8043B9847A642F9D10A4E0B4D3C
:1002C000761B03F0F3FBB61018BF002406D00134F0
:1002D00055F8043B9847A642F9D170BD70BD00BFE8
:1002E000B83A0100B83A0100CC3A0100B83A01002E
:1002F000024B0146186800F00BB800BFB097FF1F13
:10030000024B0146186800F031BF00BFB097FF1FD5
:100310002DE9F04F01F10B05162D83B0064640F292
:100320009F8035F0070500F1BF80A94200F2BC8034
:1003300000F058FBB5F5FC7FC0F09C826B0A00F022
:10034000BA80042B00F28381A80900F1390E4FEA2C
:100350004E033830C44F07EB8303A3F108015C68F8
:10036000A14207D1ACE0002A80F2AC80E468A1424F
:1003700000F0A680636823F003035A1B0F2AF2DD06
:10038000B9493C6901F1080E744500F0B381636816
:1003900023F003035A1B0F2A00F39981002AC1F8A6
:1003A00014E0C1F810E080F29E80B3F5007F80F089
:1003B0006781DB0803F1010C01229B1002FA03F3B1
:1003C0004A6851F83C80C4F8088001EBCC091A4314
:1003D000A9F10803E3604A6041F83C40C8F80C40CA
:1003E000831001249C40944200F28A80144206D17A
:1003F00020F003006400144200F10400FAD007EB7F
:10040000C009CC468046DCF80C108C4507D173E15E
:10041000002A80F28181C9688C4500F06D814B68AB
:1004200023F003035A1B0F2AF2DD0C46D1F80CC04F
:1004300054F8088F4B1945F001054D6042F0010159
:10044000C8F80CC03046CCF808807B613B61C3F82B
:100450000CE0C3F808E059609A5000F0C5FA1FE0BC
:10046000102921D800F0BEFA1025062302207E4F65
:1004700007EB8303A3F108025C68944200F0458116
:100480006368E168A56823F00303234430465A6893
:10049000E96042F001028D605A6000F0A5FA08346C
:1004A000204603B0BDE8F08F00240C2320463360C3
:1004B00003B0BDE8F08F80234FF0400E3F2049E7A6
:1004C00070465DE72344E1685A68A56842F001027E
:1004D000E96030468D605A6000F086FA08342046A4
:1004E00003B0BDE8F08F234430465A6842F0010261
:1004F0005A6000F079FA0834204603B0BDE8F08F66
:10050000BC68636823F00308A84504D3C5EB08035F
:100510000F2B00F38C80554BDFF860911A68D9F8E7
:10052000003001332A4404EB080A00F0608102F530
:1005300080520F3222F47F6222F00F0211463046C1
:10054000019200F04BFCB0F1FF3F8346019A00F0AE
:100550005881824500F2FC80454B1968DA45114408
:10056000196000F05381D9F80000DFF810E1013084
:100570001BBFCAEB0B0A5144CEF800B019601BF048
:10058000070100F01781C1F10800C1F580518344D3
:1005900008315A44C2F30B02C2EB01094946304606
:1005A000019300F01BFC431C019B00F03F81CBEB4F
:1005B00000024A4442F001021968C7F808B04944F1
:1005C000BC42CBF804201960DFF8A49016D0B8F133
:1005D0000F0F40F2FD806268A8F10C0323F00703BF
:1005E000E01802F001024FF0050E1A430F2B626073
:1005F000C0F804E0C0F808E000F21C811D4BBC68A4
:100600001A68914288BF19601B4B1A689142626850
:1006100088BF196022F003029542A2EB050301D8BE
:100620000F2B04DC304600F0DFF9002438E76219B4
:1006300043F0010345F0010565603046BA60536040
:1006400000F0D2F90834204603B0BDE8F08F142B37
:1006500071D9542B00F2A480280B00F16F0E4FEAE1
:100660004E036E3076E600BFB497FF1F6CA2FF1FEB
:1006700070A2FF1F68A2FF1F64A2FF1FC09BFF1F85
:100680005A0A042A5ED9142A00F2B38002F15C01EE
:1006900049005B3207EB810C57F82110DFF8DC8151
:1006A000ACF1080C8C4500F088804A6822F0030207
:1006B000934202D289688C45F7D1D1F80CC07A6890
:1006C000C4F80CC0A160CCF80840CC6088E663197F
:1006D00042F0010745F00105656030464B610B6152
:1006E000C3F80CE0C3F808E05F609A50083400F0EB
:1006F0007BF9D5E64A6873E608F1010818F0030FA4
:100700000CF1080C7FF47FAE30E0DC68A34208BF38
:1007100002303FF435AEB3E60B440C465A68C96864
:1007200054F8085F42F001025A603046E9608D607B
:1007300000F05AF9B4E603F15C0E03F15B004FEAF6
:100740004E0307E69A0902F1390149003832A1E760
:10075000BC424A4B3FF400AF9C68626822F003023F
:100760005AE759F80839994540F0828010F0030F94
:1007700000F1FF30F5D17B6823EA04037B6064005D
:100780009C423FF6BDAE002C3FF4BAAE1C42404640
:100790007FF435AE64001C4200F10400FAD02EE66E
:1007A000B3F5AA7F18D8E80B00F1780E4FEA4E0394
:1007B0007730CFE54FF48051EBE60121D8F80430D3
:1007C000921001FA02F21A43C8F80420614677E752
:1007D0000123CBF8043025E740F25452934220D84D
:1007E000A80C00F17D0E4FEA4E037C30B2E51032CA
:1007F000A4E6542A26D81A0B02F16F0149006E3282
:1008000048E7BC68626822F0030205E7CAF30B0000
:1008100000287FF4A8AE4244BB6842F001025A604F
:10082000ECE6FE234FF07F0E7E2093E501224FF091
:100830000009C1E604F10801304600F097FCD9F840
:100840000010DBE6B2F5AA7F05D8DA0B02F17801D9
:10085000490077321EE740F254518A4205D89A0C7B
:1008600002F17D0149007C3214E7FE217E2211E76E
:100870007B6884E7E808431C5B00F8E5B497FF1F3A
:100880008842F0B50DD98B1898420AD28118002AF7
:1008900051D09A1A13F8014D01F8014D9342F9D144
:1008A000F0BD0F2A48D941EA00039B0746D100F169
:1008B000100401F11003154653F8106C44F8106C45
:1008C00053F80C6C44F80C6C53F8086C44F8086C42
:1008D000103D53F8046C44F8046C0F2D03F1100321
:1008E00004F11004E8D8A2F1100323F00F0302F082
:1008F0000F0E1033BEF1030F1944034421D91E1FFC
:100900000D467446043C55F8047B46F8047F032CDE
:10091000F8D8AEF1040424F0030404342344214441
:1009200002F0030262B1013B0A4411F8014B03F8E3
:10093000014F8A42F9D1F0BD0346F3E70346F2E7DF
:10094000F0BD7246EEE700BF70B4840746D0541E77
:10095000002A41D0CDB2034602E0621EE4B3144641
:1009600003F8015B9A07F8D1032C2ED9CDB245EAE2
:1009700005250F2C45EA054519D903F11002264635
:10098000103E0F2E42F8105C42F80C5C42F8085CF6
:1009900042F8045C02F11002F2D8A4F1100222F035
:1009A0000F0204F00F041032032C13440DD91E461D
:1009B0002246043A032A46F8045BFAD8221F22F0A2
:1009C00003020432134404F003042CB1C9B21C44E2
:1009D00003F8011BA342FBD170BC704714460346C9
:1009E000C2E700BF704700BF704700BF024B0A4616
:1009F0000146186800F002B8B097FF1F2DE9F04FCC
:100A0000174683B0002900F0C1800E46814607F1E9
:100A10000B05FFF7E7FF56F804EC162D2EF0030444
:100A2000A6F1080840D810221546AF4241D894429A
:100A300075DAC94B996808EB04008842416800F0F8
:100A4000D98021F0010303445B68DB077DD51EF0EC
:100A5000010F35D039464846FFF75AFC0746E0B14A
:100A600056F8043C23F001034344A0F108029A42E3
:100A700000F04481221F242A00F23181132A00F25F
:100A800004810346324611681960516859609268C2
:100A90009A603146484600F069FB4846FFF7A4FFDC
:100AA000384603B0BDE8F08F25F00705002D2A4633
:100AB000BBDA0C230020C9F8003003B0BDE8F08F8A
:100AC00056F8083CC3EB080ADAF8043023F0030CAC
:100AD00004EB0C039342BDDB5746DAF80C1057F8D1
:100AE000080F221F242AC160886000F21781132A90
:100AF00040F212813168CAF808107168CAF80C1007
:100B00001B2A00F22B8108360AF1100231681160AD
:100B100071685160B16891603E461C46D046631BC7
:100B20000F2B1DD8D8F8043003F0010323434444AD
:100B3000C8F80430636843F0010363604846FFF778
:100B400053FF304603B0BDE8F08F21F0030121448C
:100B5000914221DBC36882680C46D3609A60DEE76D
:100B6000D8F8042008EB050102F00102154343F018
:100B700001020B44C8F804504A605A6842F001026E
:100B800008315A60484600F0F1FAD7E7114603B041
:100B9000BDE8F04FFFF7BCBB1EF0010F7FF45AAF6A
:100BA00056F8083CC3EB080ADAF8043023F0030CCB
:100BB00001EB0C0E96458BDBC36882685746D36009
:100BC0009A6057F8081FDAF80C30CB60221F242AED
:100BD000996000F29980132A62D93368CAF8083004
:100BE0007368CAF80C301B2A00F2A08008360AF19C
:100BF000100356E021F0030BA34405F110008345D8
:100C000059DA1EF0010F7FF425AF56F8081CC1EB2E
:100C1000080ADAF8041021F0030CE34458453FF7C2
:100C200057AF5746DAF80C1057F8080F221F242A3E
:100C3000C160886000F2B480132A40F2A580316858
:100C4000CAF808107168CAF80C101B2A00F2AF80AD
:100C500008360AF110023168116071685160B1689C
:100C600091600AEB0501C5EB0B0242F001029960AD
:100C70004A60DAF8043003F001031D434846CAF81D
:100C80000450FFF7B1FE38465CE7336803607368D1
:100C900043601B2A27D800F1080306F10802F2E698
:100CA0003B4632681A6072685A60B2689A603E4683
:100CB0007446D04633E708EB0501C5EB0B0B4BF050
:100CC000010299604A6056F8043C03F001031D4399
:100CD000484646F8045CFFF787FE304632E7314667
:100CE000FFF7CEFDD5E6B3688360F368C360242ABE
:100CF00028D000F1100306F11002C4E650F8043CBD
:100D000023F003031C440AE7314638467446D046B4
:100D1000FFF7B6FD3E4602E73A46F7E6314638466B
:100D20001C46D046FFF7ACFD3E46F8E6B368CAF86D
:100D30001030F368CAF81430242A1BD010360AF198
:100D40001803AEE7336903617369436106F1180262
:100D500000F1180397E600BFB497FF1FB168CAF807
:100D60001010F168CAF81410242A0FD010360AF1B6
:100D70001802CBE63369CAF818307369CAF81C3018
:100D800018360AF120038CE73A4664E73269CAF85C
:100D900018207269CAF81C2018360AF12002B5E63C
:100DA000314638460193FFF76BFD019B59E7B16867
:100DB000CAF81010F168CAF81410242A03D01036AB
:100DC0000AF1180247E73269CAF818207269CAF8AE
:100DD0001C2018360AF120023DE700BF38B5074C49
:100DE0000023054608462360FBF7E0FE431C00D0C5
:100DF00038BD2368002BFBD02B6038BDCCA3FF1F70
:100E000090F800F06DE9024520F007016FF0000C4A
:100E100010F0070491F820F040F049804FF00004F2
:100E20006FF00700D1E9002391F840F000F10800CD
:100E300082FA4CF2A4FA8CF283FA4CF3A2FA8CF305
:100E40004BBBD1E9022382FA4CF200F10800A4FA6C
:100E50008CF283FA4CF3A2FA8CF3E3B9D1E90423C0
:100E600082FA4CF200F10800A4FA8CF283FA4CF3F7
:100E7000A2FA8CF37BB9D1E9062301F1200182FAB1
:100E80004CF200F10800A4FA8CF283FA4CF3A2FAB7
:100E90008CF3002BC6D0002A04BF04301A4612BAC5
:100EA000B2FA82F2FDE8024500EBD2007047D1E9C8
:100EB000002304F00305C4F100004FEAC50514F057
:100EC000040F91F840F00CFA05F562EA05021CBF28
:100ED00063EA050362464FF00004A9E7002A41D007
:100EE00040EA010313F00303F0B425D1032A23D908
:100EF00004680D68AC421FD1043A35D0A4F1013525
:100F000025EA040414F0803F31D1071D0D1D0DE0CA
:100F100057F8043B0E68A3F10134B34224EA0304FA
:100F20000AD1043A20D014F0803F23D1032A294665
:100F3000384605F10405EBD803780C789C4202F1A1
:100F4000FF320CD182B114B916E06AB17BB110F84E
:100F5000013F11F8014FA34202F1FF32F5D0181BF7
:100F6000F0BC7047104670471046F0BC70471846FA
:100F7000F0BC70470020F3E72046F1E740EA0103A8
:100F80009B0770B42BD1032A29D90C46034621466E
:100F900054F8046BA6F1013525EA060515F0803FEB
:100FA00006D1043A032A43F8046B2146EFD8A2B1D4
:100FB0000C781C70013A013301313CB16AB111F86F
:100FC000014B03F8014B013A002CF7D12AB11A4426
:100FD000002103F8011B9A42FBD170BC7047034605
:100FE000E5E700BF2DE9F047254C2568D5F84841D5
:100FF0000646884692469946C4B360681F2817DCA7
:10100000431C76B104EB80050122C5F888A0D4F812
:10101000881182401143022EC4F88811C5F8089146
:101020001ED00230636044F820800020BDE8F087C5
:10103000144B03B34FF4C870FFF75AF90446D0B10C
:10104000D5F84831002780E88800C5F8484138467F
:101050000123C4F88871C4F88C71002EE1D0D1E767
:10106000D4F88C110A43C4F88C21DAE705F5A6748C
:10107000C5F84841C1E74FF0FF30BDE8F08700BF39
:10108000A83A0100F1020100024B13B1024800F03E
:1010900005B8704700000000A910010000230146B8
:1010A0001A461846FFF79EBF38B5074D074C2C1B54
:1010B000A41005D0013C55F8043D9847002CF9D107
:1010C000BDE8384002F002BD000000000000000052
:1010D000F8B5234F0C460646FFF784FCBB685D68F5
:1010E00025F00305291B01F6EF7121F47F6121F042
:1010F0000F01A1F58054B4F5805F07DB0021304675
:10110000FFF76CFEBB682B44984204D03046FFF7D3
:101110006BFC0020F8BD61423046FFF75FFE0130F6
:101120000DD0104BBA6819682D1B45F001053046EB
:10113000091B55601960FFF757FC0120F8BD00211D
:101140003046FFF74BFEBA68831A0F2BDEDD064CE4
:101150000449246843F00103001B53600860D5E78D
:10116000B497FF1F70A2FF1FC09BFF1F002945D02F
:101170002DE9F0410D468046FFF734FC55F8047C1C
:101180006A4927F00103A5F10804E2188E68506847
:10119000B24220F0030062D0FE0750600BD455F835
:1011A000087CE41B01F1080EA56875453B446FD02F
:1011B000E768EF60BD6015186D68ED0742D543F034
:1011C00001026260E350B3F5007F18D2DB085A1CBD
:1011D0004D6851F83270A76001209B1000FA03F3AC
:1011E00001EBC2001D430838E0604D6041F8324019
:1011F000FC604046BDE8F041FFF7F6BB70475A0A75
:10120000042A53D89A0902F139077F0002F1380500
:1012100001EB870051F827204449083890424DD00F
:10122000516821F003018B4202D292689042F7D1BB
:10123000D068E060A2608460D4604046BDE8F041C0
:10124000FFF7D2BB95683A4FBD4203443FD0D06808
:10125000E86043F0010285606260E350B3E7FF0796
:10126000034407D455F8082CA41A1344A068E26874
:10127000C26090602F4A126843F0010093426060A0
:101280008C60B6D32C4B40461968FFF721FFB0E7BE
:1012900011184968C90744D49168D268CA600344E8
:1012A00043F0010091606060E350A2E7142A17D870
:1012B00002F15C077F0002F15B05A9E7AA104B6809
:1012C000012505FA02F213434B600246B1E743F0F1
:1012D00001024C610C61E560A5606260E35088E743
:1012E000542A06D81A0B02F16F077F0002F16E052F
:1012F0008EE7B2F5AA7F06D8DA0B02F178077F00F5
:1013000002F1770584E740F25450824206D89A0CE5
:1013100002F17D077F0002F17C0579E7FE277E253B
:1013200076E743F001026260E35062E7B497FF1F83
:10133000BC97FF1FBC9BFF1F6CA2FF1F000078051E
:101340003408540B800C3C0F5C12E015FA19141E83
:101350006022AC265C2B0C30BC34023AFF3FFFFF0E
:10136000FDFFFFFFFBFFFFFFF8FFFFFFFDFFFFFF9C
:10137000FBFFFFFFF8FFFFFFFDFFFFFFFAFFFFFF8F
:10138000F7FFFFFFFDFFFFFFFBFFFFFFF7FFFFFF83
:10139000FCFFFFFFFBFFFFFFF7FFFFFFFDFFFFFF6E
:1013A000FAFFFFFFF7FFFFFFFDFFFFFFFBFFFFFF60
:1013B000F8FFFFFFFDFFFFFFFBFFFFFFF8FFFFFF51
:1013C000FDFFFFFFFAFFFFFFF7FFFFFFFCFFFFFF3F
:1013D000FBFFFFFFF7FFFFFFFDFFFFFFFBFFFFFF2F
:1013E000F7FFFFFFFDFFFFFFFAFFFFFFF7FFFFFF24
:1013F000FDFFFFFFFBFFFFFFF7FFFFFFFDFFFFFF0D
:10140000FBFFFFFFF7FFFFFFFDFFFFFFFAFFFFFFFF
:10141000F7FFFFFFFDFFFFFFFAFFFFFFF8FFFFFFF2
:10142000FDFFFFFFFAFFFFFFF7FFFFFFFDFFFFFFDD
:10143000FAFFFFFFF7FFFFFFFDFFFFFFFAFFFFFFD0
:10144000F8FFFFFFFDFFFFFFFAFFFFFFF8FFFFFFC1
:10145000FDFFFFFFFAFFFFFFF7FFFFFFFCFFFFFFAE
:10146000FBFFFFFFF7FFFFFFFDFFFFFFFAFFFFFF9F
:10147000F7FFFFFFFDFFFFFFFAFFFFFFF7FFFFFF93
:10148000FEFFFFFFFBFFFFFFF8FFFFFFFEFFFFFF79
:10149000FBFFFFFFF8FFFFFFFDFFFFFFFAFFFFFF6E
:1014A000F7FFFFFFFCFFFFFFFAFFFFFFF7FFFFFF64
:1014B000FCFFFFFFFAFFFFFFF7FFFFFFFDFFFFFF4E
:1014C000FAFFFFFFF7FFFFFFFDFFFFFFF9FFFFFF41
:1014D000F7FFFFFFFDFFFFFFF9FFFFFFF7FFFFFF34
:1014E000FDFFFFFFFAFFFFFFF7FFFFFFFDFFFFFF1D
:1014F000FAFFFFFFF7FFFFFFFDFFFFFFFAFFFFFF10
:10150000F6FFFFFFFDFFFFFFFAFFFFFFF7FFFFFF03
:10151000FEFFFFFFFBFFFFFFF7FFFFFFFEFFFFFFE9
:10152000FBFFFFFFF7FFFFFFFDFFFFFFFAFFFFFFDE
:10153000F7FFFFFFFDFFFFFFFBFFFFFFF8FFFFFFD0
:10154000FDFFFFFFFBFFFFFFF8FFFFFFFDFFFFFFBA
:10155000FAFFFFFFF7FFFFFFFCFFFFFFF9FFFFFFB1
:10156000F7FFFFFFFCFFFFFFF9FFFFFFF7FFFFFFA4
:10157000FDFFFFFFFAFFFFFFF7FFFFFFFDFFFFFF8C
:10158000FAFFFFFFF7FFFFFFFDFFFFFFF9FFFFFF80
:10159000F6FFFFFFFDFFFFFFFAFFFFFFF7FFFFFF73
:1015A000501C01002C1C0100081C0100E41B010060
:1015B0003C170100F81501001C160100401601003F
:1015C00018170100D4150100601A01003C13010036
:1015D000901801000000580246056608540BD80E0A
:1015E0005C127017FC21F82A70305834DC37663AE8
:1015F0008C3C803EFF3FFFFF000058024605660816
:10160000540BD80E5C12E015FA19141E6022AC2699
:101610005C2B0C30BC34023AFF3FFFFF000090010E
:1016200020031405D0075A0AAC0DCC10B4146A1864
:10163000E81C342180252A2B70301437FF3FFFFF30
:101640000000C800F4018403140508072E091C0CCF
:10165000D80EF811AE159619401F1C25F22B5834E0
:10166000FF3FFFFFFBFFFFFFF8FFFFFFF4FFFFFF60
:10167000FAFFFFFFF7FFFFFFF4FFFFFFFDFFFFFF94
:10168000F9FFFFFFF4FFFFFFFAFFFFFFF7FFFFFF88
:10169000F4FFFFFFFCFFFFFFF7FFFFFFF4FFFFFF7B
:1016A000FBFFFFFFF8FFFFFFF4FFFFFFFDFFFFFF62
:1016B000FAFFFFFFF4FFFFFFFDFFFFFFF9FFFFFF52
:1016C000F4FFFFFFFDFFFFFFF8FFFFFFF4FFFFFF49
:1016D000FCFFFFFFF7FFFFFFF4FFFFFFFBFFFFFF34
:1016E000F8FFFFFFF4FFFFFFFCFFFFFFF7FFFFFF27
:1016F000F4FFFFFF40067805B004E80384032003ED
:10170000BC025802F40190012C01FA00C8009600B6
:10171000640032001900FFFF00006400C80090015F
:10172000BC021A04DC059E07F609800CA00F2413E6
:10173000A2174C1D5424442FFF3FFFFF0000FF035E
:10174000FF07FF0BFF0FFF13FF17FF1BFF1FFF23F9
:10175000FF27FF2BFF2FFF33FF37FF3BFF3FFFFF2D
:101760000102010100010101020101020101010167
:101770000101020101020101020101010000010257
:101780000101020101010100010201010201010048
:101790000202010201010201000202020102010132
:1017A0000200010202020102010100000002020225
:1017B0000102010101000002020201020100020215
:1017C00002020202010200020201020202020102FE
:1017D00000020202010202020101000202020202F0
:1017E00002020100000202000202020200020102E3
:1017F00002020202020200020002020202020202CD
:10180000FBFFFFFFF7FFFFFFF4FFFFFFFBFFFFFF03
:10181000F7FFFFFFF4FFFFFFFDFFFFFFF7FFFFFFF5
:10182000F4FFFFFFFDFFFFFFF8FFFFFFF4FFFFFFE7
:10183000FAFFFFFFF7FFFFFFF4FFFFFFFBFFFFFFD4
:10184000F7FFFFFFF4FFFFFFFBFFFFFFF7FFFFFFC7
:10185000F4FFFFFFFBFFFFFFF7FFFFFFF4FFFFFFBA
:10186000FDFFFFFFF8FFFFFFF4FFFFFFFDFFFFFF9E
:10187000F8FFFFFFF4FFFFFFFDFFFFFFF8FFFFFF93
:10188000F4FFFFFFFAFFFFFFF8FFFFFFF4FFFFFF8A
:101890000000D007800CD80E0010C012EC130C17FB
:1018A000FA19141E6022AC265C2B0C30BC34023AB0
:1018B000FF3FFFFF00000000070000000C000000D9
:1018C0001000000013000000180000001C000000C1
:1018D00000000000070000000C00000013000000E2
:1018E000180000001F00000024000000000000009D
:1018F0000C00000018000000240000003000000070
:101900003C0000004800000000000000FBFFFFFF5B
:10191000F4FFFFFFEFFFFFFFE8FFFFFFE3FFFFFF25
:10192000DCFFFFFF00000000F4FFFFFFE8FFFFFF08
:10193000DCFFFFFFD0FFFFFFC4FFFFFFB8FFFFFF8B
:10194000FBFFFFFFF8FFFFFFF4FFFFFFFAFFFFFFC2
:10195000F7FFFFFFF4FFFFFFFDFFFFFFF9FFFFFFB2
:10196000F4FFFFFFFAFFFFFFF7FFFFFFF4FFFFFFAA
:10197000FCFFFFFFF7FFFFFFF4FFFFFFFBFFFFFF91
:10198000F8FFFFFFF4FFFFFFFDFFFFFFFAFFFFFF80
:10199000F4FFFFFFFBFFFFFFF8FFFFFFF4FFFFFF78
:1019A000FDFFFFFFF8FFFFFFF4FFFFFFFCFFFFFF5E
:1019B000F7FFFFFFF4FFFFFFFBFFFFFFF8FFFFFF55
:1019C000F4FFFFFFFCFFFFFFF7FFFFFFF4FFFFFF48
:1019D000FBFFFFFFF8FFFFFFF6FFFFFFFAFFFFFF30
:1019E000F8FFFFFFF6FFFFFFFDFFFFFFFBFFFFFF1D
:1019F000F9FFFFFFFDFFFFFFF9FFFFFFF7FFFFFF0D
:101A0000FEFFFFFFFCFFFFFFF7FFFFFFFBFFFFFFF6
:101A1000F8FFFFFFF6FFFFFFFCFFFFFFFAFFFFFFEE
:101A2000F6FFFFFFFDFFFFFFFBFFFFFFF9FFFFFFDB
:101A3000FCFFFFFFFAFFFFFFF6FFFFFFFEFFFFFFC8
:101A4000FCFFFFFFF7FFFFFFFBFFFFFFF8FFFFFFBC
:101A5000F6FFFFFFFEFFFFFFFCFFFFFFF7FFFFFFAB
:101A60000000580246056608540BA00FD41728231F
:101A7000F82A442F643284354038663A8C3C803EE4
:101A8000FF3FFFFF2C011301FA00E100C800AF0087
:101A900096007D0064004B00320019000000000039
:101AA000CDCC4C3DCDCCCC3D9A99193ECDCC4C3EC5
:101AB0000000803E9A99993E3333B33ECDCCCC3E64
:101AC0006666E63EFBFFFFFFF7FFFFFFF6FFFFFF47
:101AD000FBFFFFFFF7FFFFFFF6FFFFFFFBFFFFFF2F
:101AE000F7FFFFFFF6FFFFFFFDFFFFFFFCFFFFFF1C
:101AF000F8FFFFFFFDFFFFFFFCFFFFFFF8FFFFFF09
:101B0000FDFFFFFFFCFFFFFFF8FFFFFFFBFFFFFFF5
:101B1000F7FFFFFFF6FFFFFFFBFFFFFFF7FFFFFFF2
:101B2000F6FFFFFFFBFFFFFFFAFFFFFFF8FFFFFFDE
:101B3000FCFFFFFFF9FFFFFFF8FFFFFFFDFFFFFFC7
:101B4000FCFFFFFFF8FFFFFFFCFFFFFFFAFFFFFFB7
:101B5000F7FFFFFFFBFFFFFFF7FFFFFFF4FFFFFFB4
:101B6000FBFFFFFFF7FFFFFFF4FFFFFFFBFFFFFFA0
:101B7000F7FFFFFFF4FFFFFFFDFFFFFFF8FFFFFF91
:101B8000F4FFFFFFFDFFFFFFF8FFFFFFF4FFFFFF84
:101B9000FDFFFFFFF8FFFFFFF4FFFFFFFBFFFFFF6D
:101BA000F7FFFFFFF4FFFFFFFBFFFFFFF7FFFFFF64
:101BB000F4FFFFFFFBFFFFFFF8FFFFFFF4FFFFFF56
:101BC000FCFFFFFFF9FFFFFFF4FFFFFFFDFFFFFF3B
:101BD000F8FFFFFFF4FFFFFFFCFFFFFFF7FFFFFF32
:101BE000F4FFFFFF00007805220B0410B414321933
:101BF000B01DFC214826FE29822D38312634463777
:101C0000663A223DFF3FFFFF0000D007100E881309
